:100000000C940B110C9404140C942F140C945A148B
:100010000C9485140C94B0140C94DB140C940615F9
:100020000C9431150C943B110C943B110C943B1126
:100030000C943B110C943B110C943B110C943B1110
:100040000C943B110C94C32F0C943B110C943B115A
:100050000C943B110C943B110C94FE230C943D1119
:100060000C943B110C9454170C9400180C943B11F5
:100070000C943B110C943B110C943B110C943B11D0
:100080000C943B110C943B110C943B110C943B11C0
:100090000C943B110C943B110C943B110C943B11B0
:1000A0000C943B110C943B110C943B110C943B11A0
:1000B0000C943B110C943B110C943B110C943B1190
:1000C0000C943B110C943B110C943B110C943B1180
:1000D0000C943B110C943B110C943B110C943B1170
:1000E0000C943B117A127F1284128E129812111303
:1000F000A212AA12B212BC12C612D012DF12E91258
:100100001113F312FD1207133513381327132B1392
:1001100031136F133C13401346134A134E135413F9
:1001200058135C136F13621366136A1387178D17C6
:100130009E17A917B117C617B517C617B917BD1758
:10014000C617C317421F421F491F491F491F501F8F
:10015000501F501F5D1F571F571F571F084AD73B7F
:100160003BCE016E84BCBFFDC12F3D6C74319ABD86
:1001700056833DDA3D00C77F11BED9E4BB4C3E91AA
:100180006BAAAABE000000803F05A84CCDB2D44E99
:10019000B93836A9020C50B9918688083CA6AAAA9B
:1001A0002ABE000000803F004E414E494E4954593E
:1001B000494E46CDCCCC3D0AD7233C17B7D1387732
:1001C000CC2B329595E6241FB14F0A000020410048
:1001D00000C84200401C4620BCBE4CCA1B0E5AAE92
:1001E000C59D7400000A0B02090C0D0E08070304DC
:1001F00001000000000000000000000000000000FE
:1002000000000000000000000000000000000012DC
:1002100011100000000000000000000000000000BD
:10022000000000000000000000010210202008086B
:100230001020401020408002010201080402010148
:100240000204081020408080402010080402018031
:100250000402018040201008040201080402010188
:10026000020408102040800102040810204080058C
:10027000050505070508080808020202020A0A081F
:100280000804040404010101010101010103030345
:100290000303030303040707070C0C0C0C0C0C0CE2
:1002A0000C0202020206060606060606060B0B0BE9
:1002B0000B0B0B0B0B000020002300260029002C49
:1002C000002F0032000001000003010601090100B7
:1002D000002200250028002B002E003100340002EF
:1002E000010000050108010B010000210024002786
:1002F000002A002D00300033000101000004010736
:10030000010A014F4646004F4E006563686F3A0090
:100310004572726F723A004572726F72207772691D
:1003200074696E6720746F20454550524F4D210A05
:100330000063616E63656C00706F7765726F6666EF
:10034000002F2F616374696F6E3A0020573A0020C6
:10035000573A00202F002042403A0020403A0054F3
:100360006865726D616C2052756E617761790045C8
:100370003120544845524D414C2052554E41574131
:10038000590042454420544845524D414C20525555
:100390004E4157415900202D20496E76616C6964A9
:1003A000206578747275646572206E756D62657211
:1003B00020210A0048656174696E67206661696C76
:1003C0006564004265642068656174696E672066D3
:1003D00061696C65640048656174696E6720666177
:1003E000696C65640045312048656174696E6720F9
:1003F0006661696C6564004D494E54454D502074EA
:100400007269676765726564004531204572723AAA
:10041000204D494E54454D50004572723A204D4989
:100420004E54454D5020424544004D415854454D91
:1004300050207472696767657265640045312045B4
:1004400072723A204D415854454D50004572723AEF
:10045000204D415854454D5020424544006265644A
:100460000A002C2073797374656D2073746F70703B
:10047000656421204865617465725F49443A2000D3
:1004800023646566696E652044454641554C545F5A
:10049000004B6420004B6920004B70200000626517
:1004A0006400504944204175746F74756E65206610
:1004B000696E69736865642120507574207468657D
:1004C000206C617374204B702C204B6920616E642A
:1004D000204B6420636F6E7374616E747320667258
:1004E0006F6D2062656C6F7720696E746F20436F4B
:1004F0006E66696775726174696F6E2E680A005066
:100500004944204175746F74756E65206661696C2D
:100510006564212074696D656F75740A005468659F
:10052000726D616C2052756E617761790045312082
:10053000544845524D414C2052554E415741590067
:1005400042454420544845524D414C2052554E415D
:100550005741590048656174696E67206661696C2E
:1005600065640045312048656174696E6720666185
:10057000696C6564004265642068656174696E67D2
:10058000206661696C656400504944204175746F50
:1005900074756E65206661696C6564212054656DB3
:1005A000706572617475726520746F6F2068696719
:1005B000680A00204B643A2000204B693A20002052
:1005C0004B703A20000A20436C61737369632050BA
:1005D0004944200A002054753A2000204B753A20E7
:1005E00000206D61783A2000206D696E3A2000206D
:1005F000643A200020626961733A20005049442027
:100600004175746F74756E652073746172740A003D
:10061000504944204175746F74756E652066616938
:100620006C6564212054656D7065726174757265C6
:1006300020746F6F20686967680A001000AD03308E
:10064000016A0150022B0170030A019004F500B009
:1006500005E500D006D800F007CE001009C500302F
:100660000ABE00500BB700700CB100900DAB00B08B
:100670000EA600D00FA200F0109D001012990030BD
:100680001395005014920070158E0090168B00B0D8
:10069000178700D0188400F0198100101B7E0030ED
:1006A0001C7B00501D7900701E7600901F7300B0F7
:1006B000207000D0216E00F0226B00102469003001
:1006C000256600502663007027610090285E00B008
:1006D000295C00D02A5900F02B5600102D54003010
:1006E0002E5100502F4E0070304B0090314800B01A
:1006F000324500D0334200F0343E0010363B00302B
:100700003737005038330070392E00903A2900B046
:100710003B2300D03C1B00F03D1100103F0100F0D6
:100720003F00001000C90210012C0140012201709D
:10073000011801B0010E01F00104015002FA00B0ED
:1007400002F0003003E600D003DC009004D2007019
:1007500005C800A006BE000008B400B009AA00D079
:100760000BA000600E960060118C00001582002026
:10077000197800C01D6E00A0226400B0275A0090B6
:100780002C500000314600E0343C0010383200901C
:100790003A2800603C1E00A03D1400803E0A002064
:1007A0003F00006F70656E005452494747455245FF
:1007B00044003A20007A5F6D6178007A5F6D696E5F
:1007C00000795F6D617800795F6D696E00785F6DAB
:1007D000617800785F6D696E005265706F72746940
:1007E0006E6720656E6473746F70207374617475C6
:1007F000730A00205A3A0020593A0020583A0065FE
:100800006E6473746F7073206869743A2000486F67
:100810006D696E67206661696C656400496E76611A
:100820006C69642065787472756465720A0045307D
:100830003A20005A3A2000593A20004D53312C4DAD
:1008400053322C4D53332050696E730A583A2000AE
:100850004D6963726F737465707320756E61766134
:10086000696C61626C650A00205A3A0020593A00AE
:1008700020436F756E7420583A00C23100001C2668
:100880000000F4190000D80F0000EB080000C004BD
:100890000000750200004001000024F4D43050C371
:1008A0008E20C2A24017828B7011127A910D816C3A
:1008B000D90AA861E108C7586607615143061E4B73
:1008C0005D05C145A7041A411104093D980371391A
:1008D00031034036DB0265339102D4305402802E5E
:1008E0001D02632CEE01752AC501B028A001102756
:1008F00081018F2564012B244B01E0223401AC21BE
:100900001F018D200D01801FFC00841EED00971D2E
:10091000DF00B81CD200E61BC600201BBC00641A16
:10092000B200B219A8000A19A0006A189900D117DC
:10093000910040178B00B516840031167E00B31568
:1009400079003A157300C7146F0058146A00EE134B
:1009500066008813630025135E00C7125B006C12EB
:10096000570015125400C111510070114F00211190
:100970004B00D61049008D1047004610440002106D
:100980004200C00F4000800F3E00420F3C00060FA7
:100990003B00CB0E3800930E37005C0E3500270E5F
:1009A0003400F30D3200C10D3100900D3000600DA8
:1009B0002E00320D2D00050D2C00D90C2B00AE0C95
:1009C0002900850C29005C0C2700350C27000E0C33
:1009D0002600E80B2400C40B2400A00B23007D0B91
:1009E00023005A0B2100390B2100180B2000F80AB4
:1009F0001F00D90A1E00BB0A1E009D0A1D00800AA6
:100A00001D00630A1C00470A1B002C0A1B00110A68
:100A10001A00F7091A00DD091900C4091900AB0909
:100A20001900920917007B091800630917004C0987
:100A3000160036091600200916000A091500F508E7
:100A40001500E0081400CC081400B8081400A4082D
:100A50001400900813007D0812006B08130058085A
:100A60001200460812003408110023081100120871
:100A7000110001081100F0071000E0071000D00776
:100A80001000C0071000B0070F00A1071000910769
:100A90000E0083070F0074070F0065070E0057074D
:100AA0000E0049070E003B070D002E070E00200721
:100AB0000D0013070D0006070D00F9060C00ED06EA
:100AC0000D00E0060C00D4060C00C8060C00BC06A5
:100AD0000C00B0060C00A4060B0099060C008D0655
:100AE0000B0082060B0077060B006C060B006106FC
:100AF0000A0057060B004C060A0042060A00380698
:100B00000A002E060A0024060A001A060A00100629
:100B1000090007060A00FD050900F4050900EB05B8
:100B20000900E2050900D9050900D0050900C7053B
:100B30000900BE050900B5050800AD050800A505BA
:100B400009009C050800940508008C050800840530
:100B500008007C050800740508006C0507006505A1
:100B600008005D050700560508004E05070047050B
:100B700007004005080038050700310507002A0571
:100B80000700230507001C050600160507000F05D2
:100B900007000805060002050700FB040600F5042F
:100BA0000700EE040600E8040600E2040700DB0488
:100BB0000600D5040600CF040600C9040600C304DD
:100BC0000600BD040600B7040600B1040500AC042D
:100BD0000600A6040600A00405009B040600950478
:100BE0000500900406008A040500850405008004C1
:100BF00006007A04050075040500700405006B0406
:100C0000050066040500610405005C040500570446
:100C10000500520405004D04050048040500430486
:100C200005003E0404003A040500350405003004C4
:100C300004002C04050027040400230405001E04FE
:100C400004001A04040016040500110404000D0435
:100C50000400090405000404040000040400FC036B
:100C60000400F8030400F4030400F0030400EC03A0
:100C70000400E8030400E4030400E0030400DC03D0
:100C80000400D8030400D4030400D0030400CC0300
:100C90000400C8030300C503030024F404D9201B87
:100CA000C40C5C0E9804C4095F0265077101F40569
:100CB000F900FB04B30048048700C103690058032E
:100CC000550003034500BE023A008402310053027E
:100CD0002A002902250004022000E4011C00C801AA
:100CE0001900AF011700980114008401130071016D
:100CF00010006101100051010E0043010D0036018A
:100D00000B002B010B0020010B00150109000C0149
:100D1000090003010800FB000800F3000800EB00D5
:100D20000700E4000600DE000600D8000600D2003E
:100D30000600CC000500C7000500C2000500BD008C
:100D40000400B9000400B5000400B1000400AD00C7
:100D50000400A9000400A5000300A20003009F00F6
:100D600004009B000300980003009500020093001C
:100D70000300900003008D0002008B000300880038
:100D800002008600020084000300810002007F0050
:100D900002007D0002007B00020079000200770063
:100DA0000100760002007400020072000100710070
:100DB00002006F0002006D0001006C0002006A007A
:100DC0000100690002006700010066000100650083
:100DD0000100640002006200010061000100600087
:100DE00001005F0002005D0001005C0001005B008B
:100DF00001005A000100590001005800010057008D
:100E0000010056000100550001005400010053008C
:100E10000000530001005200010051000100500089
:100E200001004F0001004E0000004E0001004D0087
:100E300001004C0001004B0000004B0001004A0083
:100E4000010049000100480000004800010047007F
:100E5000010046000000460001004500000045007A
:100E60000100440001004300000043000100420073
:100E7000000042000100410000004100010040006C
:100E800001003F0000003F0001003E0000003E0066
:100E900001003D0000003D0001003C0000003C005E
:100EA00000003C0001003B0000003B0001003A0054
:100EB00000003A000100390000003900010038004C
:100EC0000000380000003800010037000000370043
:100ED0000100360000003600000036000100350039
:100EE000000035000000350001003400000034002F
:100EF0000000340001003300000033000000330024
:100F00000100320000003200000032000100310018
:100F1000000031000000310001003000000030000E
:100F20000000300001002F0000002F0000002F0003
:100F300000002F0001002E0000002E0000002E00F7
:100F400001002D0000002D0000002D0000002D00EC
:100F500001002C0000002C0000002C0000002C00E0
:100F600001002B0000002B0000002B0000002B00D4
:100F700001002A0000002A0000002A0000002A00C8
:100F800001002900000029000000290000002900BC
:100F900000002900010028000000280000002800AF
:100FA00000002800000028000100270000002700A2
:100FB0000000270000002700000027000100260095
:100FC0000000260000002600000026000000260089
:100FD000010025000000250000002500000025007C
:100FE000000025000000250001002400000024006E
:100FF0000000240000002400000024000100230061
:101000000000230000002300000023000000230054
:101010000000230000002300010022000000220045
:101020000000220000002200000022000000220038
:10103000010021000000210000002100000021002B
:10104000000021000000210000002100010020001C
:101050000000200000002000000020000000200010
:1010600000002000000020000000200001001F0000
:1010700000001F0000001F0000001F0000001F00F4
:1010800000001F0000001F0001001E0000001E00E5
:1010900000001E0000001E0000003A0A0020286D1B
:1010A0006D2900204500205A0020204D393037207E
:1010B000580053746570706572206D6F746F722084
:1010C00063757272656E74733A0A0020204D393070
:1010D00030204B004C696E65617220416476616E10
:1010E00063653A0A0020204D383531205A005A2DC8
:1010F00050726F6265204F6666736574002044000D
:1011000020490020204D333034205000204400205E
:10111000490020204D333031205000504944207385
:10112000657474696E67733A0A0020204D3432305A
:101130002053004175746F20426564204C657665CC
:101140006C696E673A0A00204500205A0020590059
:1011500020580020540020530020204D32303520EC
:10116000420020453C6D61785F655F6A65726B3E49
:101170000020583C6D61785F785F6A65726B3E2035
:10118000593C6D61785F795F6A65726B3E205A3CAD
:101190006D61785F7A5F6A65726B3E00416476616B
:1011A0006E6365643A20423C6D696E5F7365676D7E
:1011B000656E745F74696D655F75733E20533C6D39
:1011C000696E5F66656564726174653E20543C6D4E
:1011D000696E5F74726176656C5F66656564726185
:1011E00074653E0020540020520020204D323034DF
:1011F000205000416363656C65726174696F6E2095
:1012000028756E6974732F7332293A20503C7072BE
:10121000696E745F616363656C3E20523C726574F5
:10122000726163745F616363656C3E20543C7472E9
:101230006176656C5F616363656C3E0A0020450002
:10124000205A0020590020204D3230312058004DC6
:101250006178696D756D20416363656C6572617459
:10126000696F6E2028756E6974732F7332293A0A7C
:1012700000204500205A0020590020204D323033F4
:101280002058004D6178696D756D206665656472E2
:10129000617465732028756E6974732F73293A0A17
:1012A0000053746570732070657220756E69743AAE
:1012B0000A002020473231202020203B20556E6933
:1012C000747320696E206D6D0048617264636F6491
:1012D00065642044656661756C7420536574746937
:1012E0006E6773204C6F616465640A0028230000F8
:1012F0002823000064000000E8030000000096437B
:101300000000964300000041000020420000C94256
:101310000000C9420000C84400405044290A00208F
:1013200062797465733B2063726320002073746F6D
:101330007265642073657474696E67732072657476
:10134000726965766564202800202863616C637586
:101350006C6174656429210A0020213D2000454507
:1013600050524F4D20435243206D69736D61746339
:1013700068202D202873746F726564292000205323
:10138000697A653A2000496E6465783A2000204DFC
:1013900061726C696E3D563634290A002845455005
:1013A000524F4D3D00454550524F4D20766572736A
:1013B000696F6E206D69736D617463682000290A1E
:1013C000002062797465733B20637263200053656B
:1013D0007474696E67732053746F7265642028009B
:1013E000454550524F4D206461746173697A6520A0
:1013F0006572726F722E0A0050726F62696E67209A
:101400006661696C65640A005761726E696E673A5D
:1014100020486F6D696E672042756D702044697653
:1014200069736F72203C20310A0002020420666951
:101430007273740A005A0059005800486F6D652095
:101440000020746F6F206C6F6E6720657874727502
:1014500073696F6E2070726576656E7465640A00DC
:1014600020636F6C6420657874727573696F6E2089
:1014700070726576656E7465640A0020453A0020D6
:101480005A3A0020593A00583A000000F041000052
:10149000F04100000041FF01010000A0400000A059
:1014A00040000000400000254300004543000021AB
:1014B00043000040C000003E4300001F43000022E4
:1014C0004300003E4300001F43000040C00000E016
:1014D000C0000000C020746F6F206C6F6E672065C5
:1014E0007874727573696F6E2070726576656E744C
:1014F00065640A0020636F6C64206578747275738C
:10150000696F6E2070726576656E7465640A00623C
:101510007573793A2070617573656420666F722007
:10152000696E7075740A00627573793A207061751E
:1015300073656420666F7220757365720A00627548
:1015400073793A2070726F63657373696E670A000E
:101550004D3131372050726F62652073756363655A
:10156000737366756C0A0020496E76616C6964203D
:1015700065787472756465722000205A3A200020E4
:10158000593A200042656420583A200050726F6238
:1015900065205A204F66667365743A20003F5A20D2
:1015A0006F7574206F662072616E676520282D321A
:1015B00020746F2035290A00556E6B6E6F776E2090
:1015C000636F6D6D616E643A202200454550524F45
:1015D0004D204F4B0A004543484F00494E464F00AF
:1015E0004552524F52530044525952554E00434FA8
:1015F0004D4D554E49434154494F4E006F6666006C
:10160000D615DB15E015E715EE1544454255473A6A
:1016100000205A00205900580020204D61783A20BF
:1016200000205A00205900580020204D696E3A20B1
:1016300000536F667420656E6473746F70733A2024
:10164000002569730025696D202569730025696887
:101650002025696D20256973002569642025696846
:101660002025696D20256973002569792025696425
:10167000202569682025696D2025697300507269ED
:101680006E742074696D653A20004D3131332053FA
:10169000002F2F20004361703A004D4F54494F4EA8
:1016A0005F4D4F44455300544845524D414C5F50A7
:1016B000524F54454354494F4E004155544F5245A3
:1016C000504F52545F53445F53544154555300504C
:1016D000524F4D50545F535550504F525400454D4A
:1016E000455247454E43595F50415253455200437E
:1016F0004153455F4C494748545F4252494748541B
:101700004E45535300544F47474C455F4C4947485B
:10171000545300534F4654574152455F504F57451D
:1017200052004255494C445F50455243454E540087
:101730004C4556454C494E475F44415441005A5F21
:1017400050524F4245004155544F4C4556454C0070
:101750005052494E545F4A4F420050524F475245F3
:101760005353004155544F5245504F52545F5445C6
:101770004D5000564F4C554D455452494300454538
:1017800050524F4D0053455249414C5F584F4E5FA8
:10179000584F4646004649524D574152455F4E41CB
:1017A0004D453A4D61726C696E20204649524D5745
:1017B0004152455F56455253494F4E3A322E302ED4
:1017C000302E39352045585452554445525F5459AE
:1017D00050453A53696E676C6545787472756465F7
:1017E0007220534F555243455F434F44455F555216
:1017F0004C3A68747470733A2F2F636F64652E616E
:101800006C6570686F626A656374732E636F6D2FA9
:10181000646966667573696F6E2F4D41524C494E0F
:101820002050524F544F434F4C5F56455253494FEF
:101830004E3A312E30204D414348494E455F545970
:1018400050453A4C756C7A426F74204D696E692030
:1018500045585452554445525F434F554E543A31C2
:1018600020555549443A33353134383762362D6383
:101870006139612D346331612D383736352D643649
:10188000363862316461363538350A0020284E6FAB
:101890007420796574206D656173757265642900C3
:1018A000202041766572616765206D656173757290
:1018B0006564206261636B6C61736820286D6D29BB
:1018C0003A002020536D6F6F7468696E6720286D31
:1018D0006D293A2020202020202020202020202098
:1018E00020202020530020204261636B6C617368CC
:1018F0002044697374616E636520286D6D293A20F8
:1019000020202020202020002020202020284631B8
:101910002E30203D2066756C6C2C2046302E3020F9
:101920003D206E6F6E65290A002020436F7272653C
:101930006374696F6E20416D6F756E742F466164BC
:10194000652D6F75743A2020202020460061637455
:101950006976653A0A00696E004261636B6C617377
:101960006820636F7272656374696F6E206973209B
:1019700000205A0020506F736974696F6E616C208B
:101980004572726F723A0A004E6F7A7A6C65205413
:101990006970204F757465722044696D656E736956
:1019A0006F6E733A0A002020546F703A2000202096
:1019B00046726F6E743A200020204C6566743A209F
:1019C000004261636B6C6173683A0A00205A0043FD
:1019D000656E7465723A0A00202046726F6E743A22
:1019E000200020204C6566743A20002020546F703F
:1019F0003A200053696465733A0A00426564204CDA
:101A00006576656C696E6720004661696C65642067
:101A1000746F20656E61626C6520426564204C6560
:101A200076656C696E670A00426564204C65766570
:101A30006C20436F7272656374696F6E204D6174C0
:101A40007269783A000A0A426564204C6576656CD2
:101A500020436F7272656374696F6E204D6174729A
:101A600069783A00202B000A436F727265637465CF
:101A70006420426564204865696768742076732E27
:101A80002042656420546F706F6C6F67793A0A006A
:101A9000202B000A426564204865696768742054F9
:101AA0006F706F6772617068793A0A2020202B2D61
:101AB0002D2D204241434B202D2D2B0A2020207C10
:101AC00020202020202020202020207C0A204C20A4
:101AD0007C20202020282B29202020207C20520A16
:101AE0002045207C20202020202020202020207C19
:101AF00020490A2046207C20282D29204E20282BF2
:101B000029207C20470A2054207C202020202020CF
:101B100020202020207C20480A2020207C202020FB
:101B200020282D29202020207C20540A2020207CC1
:101B300020202020202020202020207C0A2020205F
:101B40004F2D2D2046524F4E54202D2D2B0A20284C
:101B5000302C30290A003474682070726F6265205E
:101B6000706F696E742C2064697374616E63652094
:101B700066726F6D20706C616E653A20002028449B
:101B8000525952554E2900473239204175746F2001
:101B9000426564204C6576656C696E67003F20285D
:101BA0004C2C522C462C4229206F7574206F6620D5
:101BB000626F756E64732E0A003F50726F6265200B
:101BC000706F696E74732028592920697320696DBC
:101BD000706C61757369626C652028322D32292E14
:101BE0000A003F50726F626520706F696E747320D7
:101BF00028582920697320696D706C61757369625A
:101C00006C652028322D32292E0A003F285629657E
:101C100072626F7365206C6576656C2069732069EC
:101C20006D706C61757369626C652028302D342984
:101C30002E0A00416476616E6365204B3D003F4B88
:101C40002076616C7565206F7574206F66207261F7
:101C50006E67652028302D3130292E0A004D313134
:101C60003720486F7420456E642048656174696E42
:101C7000672E2E2E0A4D3130342053313730205408
:101C8000300A473238204F310A4731205932352047
:101C90005A31302046353030300A4D3130392052FB
:101CA0003137302054300A4D313137205265776951
:101CB00070696E67206E6F7A7A6C650A54300A47D5
:101CC00031205834352059313732204635303030C4
:101CD0000A4731205A310A4D3130392052313730DC
:101CE0000A473120583435205931373220463430B4
:101CF00030300A47312058343520593137322046A8
:101D0000343030300A473120583435205931373299
:101D10002046343030300A4731205834352059318C
:101D200037322046343030300A473120583435209D
:101D3000593137322046343030300A473120583458
:101D40003520593137322046343030300A4731207F
:101D500058343520593137322046343030300A4734
:101D60003120583435205931373220463430303024
:101D70000A47312058343520593137322046343023
:101D800030300A4731205834352059313732204617
:101D9000343030300A473120583435205931373209
:101DA0002046343030300A473120583435205931FC
:101DB00037322046343030300A4731205A31350A24
:101DC0004D3130362053323535200A4730205830D7
:101DD0002059300A4D3130392052313630205430BC
:101DE0000A4D3130370A0020466C6F773A200020C8
:101DF000643A0020693A0020703A00204500205AD9
:101E000000205900204D393220580043290A006132
:101E1000626C656420286D696E2074656D702000A9
:101E200064697300656E00436F6C6420657874723A
:101E30007564657320617265200020540020520093
:101E4000416363656C65726174696F6E3A2050001E
:101E5000496E76616C696420657874727564657228
:101E60000A0020643A0020693A0020703A004732A4
:101E70002F47332062616420706172616D65746503
:101E800072730A005072696E7465722073746F7099
:101E90007065642064756520746F206572726F725E
:101EA000732E2046697820746865206572726F729F
:101EB00020616E6420757365204D39393920746F47
:101EC00020726573746172742E202854656D70657C
:101ED0007261747572652069732072657365742E02
:101EE0002053657420697420616674657220726580
:101EF0007374617274696E67290A004E6F204368BB
:101F000065636B73756D2077697468206C696E65A5
:101F1000206E756D6265722C204C617374204C6963
:101F20006E653A2000636865636B73756D206D693B
:101F3000736D617463682C204C617374204C696EFE
:101F4000653A20004C696E65204E756D62657220A1
:101F50006973206E6F74204C617374204C696E65D8
:101F6000204E756D6265722B312C204C617374208C
:101F70004C696E653A20004D313130005265736511
:101F80006E643A20002042002050006F6B00656EA6
:101F90007175657565696E6720220050494420415E
:101FA00075746F74756E65206661696C6564212057
:101FB000426164206578747275646572206E756D17
:101FC0006265720A006F6B002020506C616E6E6556
:101FD0007242756666657242797465733A200020B4
:101FE00046726565204D656D6F72793A2000436FCA
:101FF0006D70696C65643A204D6172202034203226
:102000003031390A00207C20417574686F723A20A3
:1020100028416C657068204F626A6563747320495B
:102020006E632E2C204C756C7A426F742047697455
:10203000205265706F7369746F7279290A000020ED
:102040004C61737420557064617465643A20003289
:102050002E302E302E39350A004D61726C696E00BB
:1020600020536F6674776172652052657365740AD8
:1020700000205761746368646F67205265736574EC
:102080000A002042726F776E206F7574205265735C
:1020900065740A002045787465726E616C20526523
:1020A0007365740A00506F77657255700A00737417
:1020B0006172740A005072696E7465722068616C96
:1020C0007465642E206B696C6C28292063616C6CCC
:1020D0006564210A004B494C4C206361757365644B
:1020E00020627920746F6F206D75636820696E615E
:1020F00063746976652074696D65202D206375723F
:1021000072656E7420636F6D6D616E643A20004D70
:102110003132310A4730205A31300A47323820589C
:10212000302059300A4731320A4D3130392052318E
:1021300036300A4D3131372050726F62696E672038
:102140006265640070726F62655F72657769706561
:102150000050726F62696E67206661696C65640029
:102160004D31313720426564206C6576656C696E4F
:1021700067206661696C65642E0A4730205A3130E9
:102180000A47302045300A4D333030205032352058
:10219000533838300A4D33303020503530205330EA
:1021A0000A4D3330302050323520533838300A4D04
:1021B000333030205035302053300A4D333030200A
:1021C00050323520533838300A47342053310070AC
:1021D000726F62655F6661696C65640050726F74EE
:1021E00065637465642050696E0A0025301D0C1EFD
:1021F000282924311C0B184527232F1B0A17444379
:10220000222B1A4142043803FF3604080606000157
:10221000841A2F69668F11241FBECFEFD1E2DEBF73
:10222000CDBF00E00CBF13E0A0E0B2E0E8ECF9E6BF
:1022300001E00BBF02C007900D92AC37B107D9F790
:102240002EE0ACE7B3E001C01D92A63EB207E1F775
:1022500011E1CBE0D1E100E006C021970109802F18
:10226000FE010E9479ADC830D10780E00807A9F7C8
:1022700066D40C94E2B40C9400001F920F920FB637
:102280000F9211242F933F938F939F93AF93BF93FC
:1022900080917D0390917E03A0917F03B091800394
:1022A00030917C0323E0230F2D3720F40196A11DEC
:1022B000B11D05C026E8230F0296A11DB11D209374
:1022C0007C0380937D0390937E03A0937F03B09360
:1022D00080038091810390918203A0918303B09148
:1022E00084030196A11DB11D809381039093820305
:1022F000A0938303B0938403BF91AF919F918F917B
:102300003F912F910F900FBE0F901F9018952FB7F0
:10231000F89460917D0370917E0380917F0390918A
:1023200080032FBF08953FB7F89480918103909167
:102330008203A0918303B091840326B5A89B05C0B6
:102340002F3F19F00196A11DB11D3FBFBA2FA92F34
:10235000982F8827820F911DA11DB11DBC01CD01B1
:1023600042E0660F771F881F991F4A95D1F708959D
:102370008F929F92AF92BF92CF92DF92EF92FF9295
:102380006B017C01D0DF4B015C01C114D104E1047D
:10239000F104F1F091D3C7DFDC01CB018819990971
:1023A000AA09BB09883E9340A105B10570F321E05D
:1023B000C21AD108E108F10888EE880E83E0981E61
:1023C000A11CB11CC114D104E104F10421F7DDCF3B
:1023D000FF90EF90DF90CF90BF90AF909F908F9045
:1023E0000895789484B5826084BD84B5816084BD8D
:1023F00085B5826085BD85B5816085BDEEE6F0E07E
:10240000808181608083E1E8F0E0108280818260D9
:102410008083808181608083E0E8F0E0808181605A
:102420008083E1EBF0E0808184608083E0EBF0E08A
:10243000808181608083E1E9F0E080818260808337
:10244000808181608083E0E9F0E080818160808329
:10245000E1EAF0E080818260808380818160808316
:10246000E0EAF0E0808181608083E1E2F1E0808158
:1024700082608083808181608083E0E2F1E08081FE
:1024800081608083EAE7F0E08081846080838081DE
:102490008260808380818160808380818068808386
:1024A0001092C10008951F93CF93DF93182FEB0173
:1024B00061E016D1209711F460E004C0CF3FD10550
:1024C00031F461E0812FDF91CF911F9145C1E12F60
:1024D000F0E0ED51FE4FE4914E2F50E0FA013197BC
:1024E000E231F10508F09DC08827EE58FF4F8F4F6D
:1024F0000C9479AD84B5806884BDC7BD97C084B5A0
:10250000806284BDC8BD92C0809180008068809345
:102510008000D0938900C093880088C0809180009B
:10252000806280938000D0938B00C0938A007EC02D
:1025300080918000886080938000D0938D00C0934C
:102540008C0074C08091B00080688093B000C0930C
:10255000B3006CC08091B00080628093B000C093E3
:10256000B40064C080919000806880939000D09304
:102570009900C09398005AC0809190008062809327
:102580009000D0939B00C0939A0050C0809190001F
:10259000886080939000D0939D00C0939C0046C0BB
:1025A0008091A00080688093A0008091A0008F7B24
:1025B0008093A000D093A900C093A80037C0809159
:1025C000A00080628093A000D093AB00C093AA00CB
:1025D0002DC08091A00088608093A000D093AD00B2
:1025E000C093AC0023C080912001806880932001BB
:1025F000D0932901C093280119C0809120018062E5
:1026000080932001D0932B01C0932A010FC08091A9
:102610002001886080932001D0932D01C0932C016C
:1026200005C0C038D1050CF04CCF46CFDF91CF911B
:102630001F91089590E0FC013197E231F10508F017
:102640004EC08827EC57FF4F8F4F0C9479AD809187
:1026500080008F7703C0809180008F7D8093800001
:10266000089580918000877FF9CF84B58F7702C06D
:1026700084B58F7D84BD08958091B0008F7703C0AD
:102680008091B0008F7D8093B0000895809190007C
:102690008F7707C0809190008F7D03C0809190005C
:1026A000877F8093900008958091A0008F7707C066
:1026B0008091A0008F7D03C08091A000877F8093D0
:1026C000A0000895809120018F7707C0809120019C
:1026D0008F7D03C080912001877F80932001089522
:1026E000CF93DF9390E0FC01E75DFD4F2491FC0167
:1026F000E159FD4F8491882361F190E0880F991F83
:10270000FC01E751FD4FC591D491FC01E153FD4F10
:10271000A591B491611109C09FB7F8948881209563
:1027200082238883EC912E230BC0623061F49FB723
:10273000F8943881822F809583238883EC912E2B07
:102740002C939FBF06C08FB7F894E8812E2B288367
:102750008FBFDF91CF9108951F93CF93DF93282FE1
:1027600030E0F901ED51FE4F8491F901E75DFD4F35
:10277000D491F901E159FD4FC491CC23C1F0162F3A
:10278000811158DFEC2FF0E0EE0FFF1FE153FD4FFA
:10279000A591B4918FB7F894111105C09C91ED2FBC
:1027A000E095E92302C0EC91ED2BEC938FBFDF9114
:1027B000CF911F910895CF93DF93282F30E0F90137
:1027C000ED51FE4F8491F901E75DFD4FD491F90180
:1027D000E159FD4FC491CC2389F081112BDFEC2FFF
:1027E000F0E0EE0FFF1FEB54FD4FA591B491EC917B
:1027F000ED2381E090E021F480E002C080E090E0F1
:10280000DF91CF91089508951F920F920FB60F9206
:1028100011240BB60F922F933F934F935F936F93B7
:102820007F938F939F93AF93BF93EF93FF93E09129
:102830000402F09105021995FF91EF91BF91AF91BC
:102840009F918F917F916F915F914F913F912F91C8
:102850000F900BBE0F900FBE0F901F9018951F92F8
:102860000F920FB60F9211240BB60F922F933F9336
:102870004F935F936F937F938F939F93AF93BF9388
:10288000EF93FF93E0910602F09107021995FF91F3
:10289000EF91BF91AF919F918F917F916F915F91D8
:1028A0004F913F912F910F900BBE0F900FBE0F9045
:1028B0001F9018951F920F920FB60F9211240BB60E
:1028C0000F922F933F934F935F936F937F938F93C9
:1028D0009F93AF93BF93EF93FF93E0910802F09122
:1028E00009021995FF91EF91BF91AF919F918F913F
:1028F0007F916F915F914F913F912F910F900BBE00
:102900000F900FBE0F901F9018951F920F920FB649
:102910000F9211240BB60F922F933F934F935F9317
:102920006F937F938F939F93AF93BF93EF93FF9397
:10293000E0910A02F0910B021995FF91EF91BF917E
:10294000AF919F918F917F916F915F914F913F9147
:102950002F910F900BBE0F900FBE0F901F901895E8
:102960001F920F920FB60F9211240BB60F922F9356
:102970003F934F935F936F937F938F939F93AF9307
:10298000BF93EF93FF93E0910002F091010219953C
:10299000FF91EF91BF91AF919F918F917F916F9137
:1029A0005F914F913F912F910F900BBE0F900FBEF3
:1029B0000F901F9018951F920F920FB60F9211242F
:1029C0000BB60F922F933F934F935F936F937F9329
:1029D0008F939F93AF93BF93EF93FF93E091020286
:1029E000F09103021995FF91EF91BF91AF919F91E3
:1029F0008F917F916F915F914F913F912F910F90A8
:102A00000BBE0F900FBE0F901F9018951F920F9244
:102A10000FB60F9211240BB60F922F933F934F9343
:102A20005F936F937F938F939F93AF93BF93EF9336
:102A3000FF93E0910C02F0910D021995FF91EF9137
:102A4000BF91AF919F918F917F916F915F914F91C6
:102A50003F912F910F900BBE0F900FBE0F901F90C4
:102A600018951F920F920FB60F9211240BB60F926A
:102A70002F933F934F935F936F937F938F939F9386
:102A8000AF93BF93EF93FF93E0910E02F0910F028B
:102A90001995FF91EF91BF91AF919F918F917F9188
:102AA0006F915F914F913F912F910F900BBE0F90BF
:102AB0000FBE0F901F90189508954F925F926F92DE
:102AC0007F92AF92BF92CF92DF92EF92FF920F93DD
:102AD0001F93CF93DF93CDB7DEB729013A019B0156
:102AE000AC0124193509460957098A899B89AC89A3
:102AF000BD89BC01CD016A197B098C099D090E9421
:102B000018ADA801970124193509460957090E94F3
:102B10005DADCA01B9016A0D7B1D8C1D9D1DDF9144
:102B2000CF911F910F91FF90EF90DF90CF90BF90CA
:102B3000AF907F906F905F904F900895089551DC13
:102B4000FDDF0E94A4A8C0E0D0E00E942AA920973F
:102B5000E1F30E940000F9CFCF93C82F0E94D92D36
:102B6000CC2349F024982C9A65E070E080E090E056
:102B7000FFDB149A03C0249A2C981498CF910895DF
:102B800080E0EACFCF92DF92EF92FF926B017C015F
:102B900083E3C816D104E104F10468F082E3C81AA3
:102BA000D108E108F10862E370E080E090E0E0DB4A
:102BB0000E941522EDCFC701B601DADBFF90EF903E
:102BC000DF90CF900C941522DC01FB01460F571FBC
:102BD000E417F507C1F081912D913C9111973827A9
:102BE00098E0B901660F771F37FF06C09B0181E2AD
:102BF000282780E1382701C09B01915091F7119659
:102C00003C932E93E5CF0895CF93DF93FC018491FD
:102C1000EF012196882319F087D2FE01F8CFDF91CA
:102C2000CF9108958AE093E0EFCF80E193E0ECCF7D
:102C30000F931F93CF93DF931F921F92CDB7DEB7F1
:102C400069837A83E1DF6981062F7A81172FF80182
:102C500081918F01882311F067D2F9CF0F900F90E7
:102C6000DF91CF911F910F910895CF93DF93EB01E7
:102C7000CBDF6AE070E0CE01DF91CF9148C3CF9205
:102C8000DF92EF92FF926A017B01BEDF4AE050E0E3
:102C9000C701B601FF90EF90DF90CF9027C3CF928E
:102CA000DF92EF92FF926A017B01AEDF42E050E0DB
:102CB000C701B601FF90EF90DF90CF90B3C3CF92E2
:102CC000DF92EF92FF926A017B019EDF42E050E0CB
:102CD000C701B601FF90EF90DF90CF90A3C3CF93D1
:102CE000DF93EB0191DF6AE070E0CE01DF91CF91DD
:102CF00023C3CF92DF92EF92FF926A017B0184DFC0
:102D00004AE050E0C701B601FF90EF90DF90CF900E
:102D10000DC3811103C083E093E002C087E093E01C
:102D200073CFF7DF8AE000C2CF93DF931F921F9229
:102D3000CDB7DEB72091E00E3091E10ECE010196C5
:102D40002115310519F4865E9E4002C0821B930B4B
:102D50009A83898389819A810F900F90DF91CF9117
:102D6000089581E0089581E008958F929F92AF9237
:102D7000BF92CF92DF92EF92FF920F931F93CF9368
:102D8000DF931F921F92CDB7DEB76C0159018B0103
:102D90007B01E40EF51E0E151F0561F1F601808022
:102DA0009180F80161918F016983C4016A830E9457
:102DB000CCB46A81681779F0C4010E94D4B4C4010C
:102DC0000E94CCB49981891731F02CDF87E193E020
:102DD0001BDF81E010C041E050E0BE016F5F7F4F1C
:102DE000C501F2DEF601408151814F5F5F4F518393
:102DF0004083D1CF80E00F900F90DF91CF911F9152
:102E00000F91FF90EF90DF90CF90BF90AF909F9089
:102E10008F9008958F929F92AF92BF92CF92DF9240
:102E2000EF92FF920F93CF93DF931F92CDB7DEB750
:102E30005C016B017A014901F501808191810E9459
:102E4000CCB48983002311F0F601808341E050E087
:102E5000BE016F5F7F4FC401B7DEF5014081518134
:102E60004F5F5F4F51834083FFEFCF1ADF0A81E04E
:102E7000E81AF10809F780E00F90DF91CF910F91E8
:102E8000FF90EF90DF90CF90BF90AF909F908F908A
:102E9000089598E288E10FB6F894A89580936000B1
:102EA0000FBE9093600008951F920F920FB60F927D
:102EB00011240BB60F920F931F932F933F934F93B1
:102EC0005F936F937F938F939F93AF93BF93CF93B2
:102ED000DF93EF93FF930091AB03D091AA0311E02E
:102EE0001D0F1F77C091C60090918603492F092EB0
:102EF000000C550B660B770B4C30510508F046C0A3
:102F0000FA018827EA56FF4F8F4F0C9479ADCD34E4
:102F100041F0CE34B9F481E005C0CA3330F0CD348D
:102F200071F582E0809386034AC0C03308F047C041
:102F3000C03209F444C0CD3211F541C0C13329F08B
:102F4000C43329F0C032D9F43AC083E0EBCF88E033
:102F5000E9CFC03321F0C13391F486E0E3CF84E0C0
:102F6000E1CFC83361F485E0DDCFC23341F487E0BF
:102F7000D9CFC13321F489E0D5CFC03311F08BE034
:102F8000D1CF8AE0CFCFCA30D1F417C0CA30B9F45C
:102F900080913504882389F0973049F09A3059F0B0
:102FA000953059F410925B021092DF0E06C081E05A
:102FB0008093360402C00E945EA710928603101709
:102FC00031F0ED2FF0E0E655FC4FC283D12FD093C6
:102FD000AA03FF91EF91DF91CF91BF91AF919F91A4
:102FE0008F917F916F915F914F913F912F911F91A1
:102FF0000F910F900BBE0F900FBE0F901F90189562
:103000001F920F920FB60F9211240BB60F922F93AF
:103010008F939F93EF93FF9380918903209188036F
:10302000281791F0E82FF0E0E857FC4F92818F5F6E
:103030008F719093C600809389039091C000906433
:103040009093C000281305C08091C1008F7D8093AC
:10305000C100FF91EF919F918F912F910F900BBE27
:103060000F900FBE0F901F9018959B01AC0110920E
:10307000C000211581EE380741055105C1F080914E
:10308000C00082608093C00060E079E08DE390E052
:103090000E945DADCA01B9016150710981099109B0
:1030A00022E030E040E050E00E945DAD02C020E14F
:1030B00030E03093C5002093C4008091C10080614E
:1030C0008093C1008091C10088608093C10080918D
:1030D000C10080688093C1008091C1008F7D809382
:1030E000C1001092870308958091AA039091AB03C9
:1030F000891759F0E92FF0E0E655FC4F82819F5F78
:103100009F779093AB0390E008958FEF9FEF089522
:10311000EAEAF3E0808181830895EAEAF3E08081BE
:103120009181891B8F77089591E090938703909107
:10313000C10095FD04C09091C00095FD40C0209154
:1031400088032F5F2F710FB607FC34C0909189035D
:10315000291322C09091C00095FF1DC09091890352
:1031600040918803491791F0E92FF0E0E857FC4FB0
:1031700032819F5F9F713093C60090938903309195
:10318000C00030643093C000491305C09091C10065
:103190009F7D9093C100DACFE0918803F0E0E8577B
:1031A000FC4F8283209388038091C10080628093CA
:1031B000C1000895909189032913EECFFBCF80932E
:1031C000C6008091C00080648093C00008958DE0A7
:1031D000ABDF8AE0A9CFCF93DF93EC0189918823FD
:1031E00011F0A2DFFBCFDF91CF91F1CF8F929F92B1
:1031F000AF92BF92EF92FF921F93CF93DF93CDB721
:10320000DEB7A0970FB6F894DEBF0FBECDBF611535
:1032100071058105910579F110E0842E912CA12C86
:10322000B12CEE24E394F12CEC0EFD1EE10EF11C0A
:1032300017FDFA94A50194010E943BADF70160834C
:10324000B901CA011F5F611571058105910549F733
:10325000115010F1E1E0F0E0EC0FFD1FE10FF11D66
:1032600017FDFA9580818A3010F097E301C090E352
:10327000890F5ADFEDCF80E3A0960FB6F894DEBF3A
:103280000FBECDBFDF91CF911F91FF90EF90BF9008
:10329000AF909F908F9048CFA0960FB6F894DEBF66
:1032A0000FBECDBFDF91CF911F91FF90EF90BF90E8
:1032B000AF909F908F900895CF92DF92EF92FF9200
:1032C0006B017C0197FF0AC08DE22EDFF094E09441
:1032D000D094C094C11CD11CE11CF11C4AE0C70170
:1032E000B601FF90EF90DF90CF9080CF4115510550
:1032F00011F4862F19CF4A30510509F4DDCF76CF6E
:10330000AB01682F880F770B880B990BEFCFAB01C0
:10331000BC01990F880B990BE9CFAB01BC01990F48
:10332000880B990BE3DF53CFE1DF51CF41155105F6
:1033300011F4862FF9CE5ACFAB01BC0180E090E0AA
:10334000F5CF8F929F92AF92BF92CF92DF92EF9282
:10335000FF92CF936B017C01B42E20E030E0A901F5
:103360000E9410AA87FF06C08DE2DEDEF7FAF09415
:10337000F7F8F094C0E060E070E080E09FE3CB15E8
:1033800041F02DEC3CEC4CEC5DE30E944EACCF5F89
:10339000F6CF9B01AC01C701B6010E9437A96B01B2
:1033A0007C010E9484AA4B015C014AE01FDFCC2310
:1033B00079F1C501B4010E94B0AA9B01AC01C7011B
:1033C000B6010E9436A96B017C018EE2ADDE20E0E1
:1033D00030E040E251E4C701B6010E944EAC4B011F
:1033E0005C010E947FAA6B01770FEE08FF08C701FE
:1033F000B60162DFC701B6010E94B2AA9B01AC010F
:10340000C501B4010E9436A96B017C01C150F9F6D7
:10341000CF91FF90EF90DF90CF90BF90AF909F90B3
:103420008F9008958ECFCF92DF92EF92FF920F93FD
:103430001F930E9487110091300410913104209154
:103440003204309133046B017C01C01AD10AE20AC4
:10345000F30AF7FC52C08B019C010C53164F2F4FFF
:103460003F4F009330041093310420933204309383
:103470003304079B39C0069B37C0059B35C020919C
:10348000B704211131C0049B2FC000912C0410916E
:103490002D0420912E0430912F04011511052105D2
:1034A000310571F0DC01CB01801B910BA20BB30B3A
:1034B00080569A4EA109B109B7FF02C068E701C062
:1034C00060E06093340480910201611180958870FE
:1034D0008093000170E086E01F910F91FF90EF90C4
:1034E000DF90CF900C94531260932C0470932D04B2
:1034F00080932E0490932F04C8CF1F910F91FF90BB
:10350000EF90DF90CF90089581E080933504089587
:1035100090910E068917D1F00E94475880910E06AF
:10352000882359F041E855E06DE775E089E795E0BB
:103530000E940A5710920E0607C081E080930E0683
:1035400089E795E00E9478570C941D4C089580E01F
:10355000DFDF8AEE95E00C94CBA20F931F93CF93FD
:10356000DF931F92CDB7DEB78C0181E493E06983CE
:103570004BDBC80149DB6981662339F08AE00F9093
:10358000DF91CF911F910F91CFCD0F90DF91CF9110
:103590001F910F91089561E088E393E0DECF61E031
:1035A00081E393E0DACFEF92FF920F931F93CF93D3
:1035B000DF931F92CDB7DEB78C017B0180E2498398
:1035C000B3DD49814F3F11F084E501C082E4ACDDF9
:1035D0008AE3AADDF801608171818281938142E0F2
:1035E00050E020DFF701408151816281738183E5E2
:1035F00093E055DB62E070E080E090E00F90DF91B7
:10360000CF911F910F91FF90EF900C94B811811101
:1036100009C0CB016F3F710519F010F08FEF90E0FA
:103620008093C004089597FF03C08091B70404C03D
:10363000FC01E458FB4F808190E008952F923F9267
:103640004F925F926F927F928F929F92AF92BF92B2
:10365000CF92DF92EF92FF92CF93DF9300D01F9231
:10366000CDB7DEB76090C1047090C2048090C504ED
:103670009090C604A090C704B090C804B301072C72
:10368000000C880B990B0E94B2AAA50194010E941C
:1036900036A96B017C0120ED3CEC4CE45DE36091CC
:1036A0009D0470919E0480919F049091A0040E94BB
:1036B0004EAC1B012C0120916804309169044091AB
:1036C0006A0450916B04C501B4010E9436A99B01A4
:1036D000AC01C201B1010E944EAC1B012C0123E3DD
:1036E00033E343E75FE36091640470916504809184
:1036F0006604909167040E944EAC9B01AC01C2012C
:10370000B1010E9437A969837A838B839C8360937C
:1037100064047093650480936604909367048092B8
:10372000680490926904A0926A04B0926B0420E04D
:1037300030E040E251E4C701B6010E9413AC181614
:1037400054F481E080935B04412C512C2FE7622ECE
:1037500023E4722EC0C020E030E040E251ECC7010B
:10376000B6010E9410AA87FD02C0672839F481E0E3
:1037700080935B04412C512C3201ADC080915B04DD
:10378000882351F010925704109258041092590453
:1037900010925A0410925B042091570430915804FF
:1037A0004091590450915A04C701B6010E9437A9AB
:1037B0004B015C0160935704709358048093590443
:1037C00090935A0420919504309196044091970467
:1037D00050919804C701B6010E944EAC2B013C01E8
:1037E00060935C0470935D0480935E0490935F0427
:1037F0002091990430919A0440919B0450919C042B
:10380000C501B4010E944EAC9B01AC016093600401
:10381000709361048093620490936304C301B201C6
:103820000E9437A929813A814B815C810E9436A987
:103830002B013C0120E030E04FE753E40E9413AC41
:1038400020E030E0A9011816DCF4C701B6010E949F
:1038500013AC1816B4F5A7019601C501B4010E9476
:1038600036A9609357047093580480935904909339
:103870005A04412C512C9FE7692E93E4792E2BC0DA
:10388000C301B2010E9410AA87FF25C020E030E0EA
:10389000A901C701B6010E9410AA87FF19C0A7019C
:1038A0009601C501B4010E9436A960935704709334
:1038B00058048093590490935A04412C512C32019E
:1038C0000AC0412C512C8FE7682E83E4782E03C068
:1038D000412C512C3201C301B2010F900F900F9077
:1038E0000F90DF91CF91FF90EF90DF90CF90BF903E
:1038F000AF909F908F907F906F905F904F903F9090
:103900002F9008954F925F926F927F928F929F9225
:10391000AF92BF92CF92DF92EF92FF92CF93DF935D
:10392000CDB7DEB72C970FB6F894DEBF0FBECDBF74
:103930008091BC049091BD04A091BE04B091BF04DD
:1039400089839A83AB83BC836091B8047091B90476
:10395000072E000C880B990B0E94B2AA29813A818C
:103960004B815C810E9436A96B017C01209153043C
:103970003091540440915504509156040E9437A947
:103980004B015C016093530470935404809355047D
:10399000909356042091A3043091A4044091A5046F
:1039A0005091A604C701B6010E944EAC6D837E8380
:1039B0008F839887609347047093480480934904E9
:1039C00090934A042091A7043091A8044091A9043F
:1039D0005091AA04C501B4010E944EAC69877A8750
:1039E0008B879C8760934B0470934C0480934D04A9
:1039F00090934E0420ED3CEC4CE45DE36091AB040D
:103A00007091AC048091AD049091AE040E944EACD4
:103A10002B013C0120914304309144044091450422
:103A20005091460469817A818B819C810E9436A9DC
:103A30009B01AC01C301B2010E944EAC2B013C01C1
:103A400023E333E343E75FE360914F047091500455
:103A500080915104909152040E944EAC9B01AC01A4
:103A6000C301B2010E9437A92B013C0160934F04AE
:103A700070935004809351049093520489819A81E9
:103A8000AB81BC818093430490934404A09345048C
:103A9000B093460429853A854B855C856D817E818E
:103AA0008F8198850E9437A9A30192010E9436A9AF
:103AB0002B013C0120E030E04FE753E40E9413ACBF
:103AC00020E030E0A9011816DCF4C701B6010E941D
:103AD00013AC1816B4F5A7019601C501B4010E94F4
:103AE00036A96093530470935404809355049093C3
:103AF0005604412C512C9FE7692E93E4792E2BC05C
:103B0000C301B2010E9410AA87FF25C020E030E067
:103B1000A901C701B6010E9410AA87FF19C0A70119
:103B20009601C501B4010E9436A9609353047093B5
:103B300054048093550490935604412C512C320127
:103B40000AC0412C512C8FE7682E83E4782E03C0E5
:103B5000412C512C3201C301B2012C960FB6F894BE
:103B6000DEBF0FBECDBFDF91CF91FF90EF90DF9012
:103B7000CF90BF90AF909F908F907F906F905F900D
:103B80004F9008954F925F926F927F928F929F9283
:103B9000AF92BF92CF92DF92EF92FF920F931F935B
:103BA000CF93DF933C01C62F662389F03ED86AE0AD
:103BB00070E08C2F90E0ABDB86E993E025D880E0C5
:103BC00090E00E94A3A760E070E0CB017AC0B0E271
:103BD000A0E06A2F70E0AB014B0F511D5595479542
:103BE0004A1711F04B130BC0E1EAF7E065917491AD
:103BF000072E000C880B990B0E94B2AA62C0CA0162
:103C00000197880F991F880F991FFC01ED5DF84FF0
:103C1000059114919A01220F331F220F331FF901CE
:103C2000ED5DF84FC591D4916016710614F4B42F70
:103C3000D2CFA42FC615D7050CF4CBCF8B5D984FF0
:103C4000FC01E590F490F901EB5DF84FC590D4903C
:103C5000B7010F2C000C880B990B0E94B2AA4B01E4
:103C60005C01B301601B710B072E000C880B990BD4
:103C70000E94B2AA2B013C01B6016E197F09072EE2
:103C8000000C880B990B0E94B2AA9B01AC01C301E6
:103C9000B2010E944EAC6B017C01C01BD10BBE0176
:103CA000DD0F880B990B0E94B2AA9B01AC01C701E2
:103CB000B6010E9417AA9B01AC01C501B4010E9484
:103CC00037A9DF91CF911F910F91FF90EF90DF9077
:103CD000CF90BF90AF909F908F907F906F905F90AC
:103CE0004F9008954F925F926F927F928F929F9222
:103CF000AF92BF92CF92DF92EF92FF920F931F93FA
:103D0000CF93DF933C01BAE3A0E06A2F70E0AB01F0
:103D10004B0F511D559547954A1711F04B130BC08A
:103D2000E1E2F7E065917491072E000C880B990B86
:103D30000E94B2AA62C0CA010197880F991F880F1A
:103D4000991FFC01E55CF94F059114919A01220F2E
:103D5000331F220F331FF901E55CF94FC591D49150
:103D60006016710614F4B42FD2CFA42FC615D70550
:103D70000CF4CBCF835C994FFC01E590F490F901F2
:103D8000E35CF94FC590D490B7010F2C000C880B61
:103D9000990B0E94B2AA4B015C01B301601B710B2D
:103DA000072E000C880B990B0E94B2AA2B013C0134
:103DB000B6016E197F09072E000C880B990B0E9423
:103DC000B2AA9B01AC01C301B2010E944EAC6B01CF
:103DD0007C01C01BD10BBE01DD0F880B990B0E942B
:103DE000B2AA9B01AC01C701B6010E9417AA9B01B0
:103DF000AC01C501B4010E9437A9DF91CF911F9199
:103E00000F91FF90EF90DF90CF90BF90AF909F9079
:103E10008F907F906F905F904F90089560E08091B9
:103E2000C3049091C404AEDE6093C5047093C604CD
:103E30008093C7049093C8048091BA049091BB0406
:103E400051DF6093BC047093BD048093BE049093D3
:103E5000BF04A89510928D04089567707727E82F06
:103E6000880FFF0BED51FE4FE4918E2F90E0FC0187
:103E70003797EC30F10508F58827EE55FF4F8F4F47
:103E80000C9479AD8091B100887F682B6093B1006C
:103E9000089580919100887F682B60939100089528
:103EA0008091A100887F682B6093A1000895809184
:103EB0002101887F682B6093210108956D9A759880
:103EC00080910101806180930101809102018071E4
:103ED00080930001809101018860809301018091AD
:103EE00002018870809300019D9AA598809101013C
:103EF00080628093010164E070E088E0AEDF809131
:103F0000010188608093010164E070E086E0A5DF34
:103F100087ED80937A0010927E0010927D00809150
:103F20007E00816080937E0080917E00846080931B
:103F30007E0080E888BD80916E00846080936E0072
:103F40006AEF70E080E090E00E94B81185E090E0B8
:103F500090937E0480937D0460E08091170290919D
:103F6000180210DE20E030E040EA50E40E9410AA7F
:103F700087FF0AC080911702909118024097909392
:103F8000180280931702E8CF81E391E09093160224
:103F90008093150260E080917F0490918004F2DDAF
:103FA00020E030E848E953E40E9413AC181654F4BA
:103FB00080917F0490918004409690938004809338
:103FC0007F04E8CF80911B0290911C028BDE20E0E1
:103FD00030E040EA50E40E9410AA87FF0AC08091B6
:103FE0001B0290911C02409790931C0280931B022D
:103FF000E9CF8091B5049091B60474DE20E030E002
:1040000046E153E40E9413AC181654F48091B504B1
:104010009091B60440969093B6048093B504E9CF8E
:104020000895CF92DF92EF92FF928091C104909118
:10403000C2040097B9F0C090C504D090C604E090C7
:10404000C704F090C8040D97BC01990F880B990B19
:104050000E94B2AA9B01AC01C701B6010E9410AA3E
:1040600087FD09C010928F04109290041092910461
:10407000109292041EC020E030E040E050E4C701FE
:10408000B6010E9437A90E9484AA70939404609399
:1040900093040E948711DC01CB01805E914BAF4FEE
:1040A000BF4F80938F0490939004A0939104B0939A
:1040B0009204FF90EF90DF90CF900895CF92DF921F
:1040C000EF92FF928091B8049091B9040097B9F0F3
:1040D000C090BC04D090BD04E090BE04F090BF043A
:1040E0000897BC01990F880B990B0E94B2AA9B01FB
:1040F000AC01C701B6010E9410AA87FD09C0109249
:10410000AF041092B0041092B1041092B2041EC019
:1041100020E030E040E050E4C701B6010E9437A93A
:104120000E9484AA7093B4046093B3040E94871120
:10413000DC01CB01805A9541AF4FBF4F8093AF0454
:104140009093B004A093B104B093B204FF90EF90A9
:10415000DF90CF90089580911502909116020F97ED
:104160001816190614F480E090E09093C20480932E
:10417000C10480E056DF1092B9041092B8049EDFAB
:1041800080911502909116020F971816190614F4D3
:1041900080E090E09093C2048093C10480E041DF0E
:1041A00010927C0475981092B9041092B804109281
:1041B000B704A5980895EF92FF920F931F93CF93A2
:1041C000C82F7B018A0180915C028823B1F00E9494
:1041D0001516C7010E94041682E694E00E94041698
:1041E000C7FD07C06AE070E08C2FCC0F990B95D803
:1041F00004C08DE594E00E94041680916C04811146
:104200000DC010925C0281E080936C04C801CF91D4
:104210001F910F91FF90EF900C94A3A7CF911F9146
:104220000F91FF90EF9097CF8F3F19F04CE354E040
:1042300002C04CE454E06AE274E0BDCF8F3F19F055
:1042400049E054E002C049E154E067EF73E0B3CFC6
:104250002F923F924F925F926F927F928F929F9296
:10426000AF92BF92CF92DF92EF92FF920F931F9384
:10427000CF93DF9300D01F92CDB7DEB75C017A8376
:1042800069834A01170107FD05C0802F002E000C2D
:10429000990B02C081E090E0F9014080518062807A
:1042A00073809C01220F331F220F331F3C832B830B
:1042B000255C3B4F7901A3019201F7016081718177
:1042C000828193810E9410AA882391F0F701408295
:1042D00051826282738211E020E030E0A901C301C3
:1042E000B2010E9413AC18160CF010E0F501108317
:1042F000F50180818230D1F0833009F45EC08130D5
:1043000009F07CC0EB81FC81E55CFB4F20813181B1
:1043100042815381F40160817181828193810E9485
:1043200010AA87FD6BC082E0F50180832B813C8160
:10433000255C3B4F7901B60180E090E00E94B0AA75
:104340009B01AC01F70160817181828193810E94A0
:1043500036A99B01AC01F401608171818281938156
:104360000E9413AC87FD16C00E9487116B017C016F
:104370009101A8EEB3E00E9481ADDC01CB018C0D70
:104380009D1DAE1DBF1DE981FA8180839183A283AB
:10439000B38334C00E948711E981FA81C080D18043
:1043A000E280F380DC01CB018C199D09AE09BF09C5
:1043B000B7FD24C083E0F50180830F3F19F04FE67D
:1043C00053E002C042E853E06FE573E0802F0F90A6
:1043D0000F900F900F90DF91CF911F910F91FF9051
:1043E000EF90DF90CF90BF90AF909F908F907F9095
:1043F0006F905F904F903F902F90DDCE0F900F9079
:104400000F900F90DF91CF911F910F91FF90EF9040
:10441000DF90CF90BF90AF909F908F907F906F90E4
:104420005F904F903F902F9008958F929F92AF9200
:10443000BF92CF92DF92EF92FF920F93CF93DF93D1
:1044400000D01F92CDB7DEB78091360481111DC117
:1044500080918D04811110C00F900F900F900F90DC
:10446000DF91CF910F91FF90EF90DF90CF90BF90B1
:10447000AF909F908F900895D1DC0E9487114B01DF
:104480005C018091130290911402181619060CF029
:1044900001C1019790931402809313026091C104AB
:1044A0007091C204072E000C880B990B0E94B2AACF
:1044B00069837A838B839C834EE1C42ED12C5FE089
:1044C000E52EF12C00E09E012F5F3F4F45EC54E0BC
:1044D00067E774E08BE794E0BBDEC090C504D09042
:1044E000C604E090C704F090C80480917D049091C8
:1044F0007E04BC01990F880B990B0E94B2AA9B0104
:10450000AC01C701B6010E9413AC1816CCF460913F
:10451000150270911602072E000C880B990B0E9451
:10452000B2AA9B01AC01C701B6010E9410AA87FF85
:1045300007C080E083D80E947FAA7595679501C067
:1045400060E060937C0480918F0490919004A0912E
:104550009104B09192040097A105B10521F1A50144
:104560009401281B390B4A0B5B0B57FD1CC0609153
:1045700093047091940480E090E00E94B0AA9B01A3
:10458000AC016091C5047091C6048091C7049091FC
:10459000C8040E9410AA87FF9EC045EE53E066ED56
:1045A00073E080E008DE8091AF049091B004A091A8
:1045B000B104B091B2040097A105B10509F1881AC0
:1045C000990AAA0ABB0AB7FC1BC06091B304709198
:1045D000B40480E090E00E94B0AA2091BC04309125
:1045E000BD044091BE045091BF040E9413AC181644
:1045F0000CF06FC043EC53E064EB73E08FEFDBDD56
:104600006091B8047091B904072E000C880B990BC7
:104610000E94B2AA69837A838B839C839AE0C92E15
:10462000D12C2FE0E22EF12C0FEF9E012F5F3F4F98
:104630004CEB54E062E774E086E794E009DE80909A
:10464000BC049090BD04A090BE04B090BF0420E0D4
:1046500030E040EA50E4C501B4010E9413AC87FD8C
:1046600010C020E030E046E153E4C501B4010E94EF
:1046700010AA181634F046D90E947FAA759567953E
:1046800001C060E06093B704E7CE80E090E00E9454
:10469000A3A7DECEC090C504D090C604E090C704A6
:1046A000F090C80420E030E848E953E4C701B601BF
:1046B0000E9413AC181694F020E030E040EA50E479
:1046C000C701B6010E9410AA87FFE8CE80E0B6DDE0
:1046D000E5CEF4DC95CF80E0A4DC65CF80E0A4DDFE
:1046E000C090C504D090C604E090C704F090C80400
:1046F000E3CF80918104909182049093C4048093CD
:10470000C3048091A1049091A2049093BB04809370
:10471000BA0481E080938D0408951F93CF93DF93B3
:1047200080918D04811101C0E4DF8CE0E1E8F4E0C8
:10473000DF011D928A95E9F71092A2041092A1045C
:10474000C091C304D091C404D195C195D109809181
:10475000C1049091C20411E0181619062CF0809142
:104760007C04811101C010E080917F04909180044D
:104770009195819591098C179D0714F480E054DD83
:104780008091170290911802919581959109C8170F
:10479000D90724F4112311F080E050DD8091B80492
:1047A0009091B904C1E0181619062CF08091B70455
:1047B000811101C0C0E02091BA043091BB04809106
:1047C000B5049091B6048217930714F08FEF2CDD97
:1047D00020911B0230911C028091BA049091BB047D
:1047E000821793073CF0CC2329F08FEFDF91CF9114
:1047F0001F9124CDDF91CF911F9108950F930FB793
:104800000F9300916E000B7F00936E0078940F93CE
:104810000BB70F930CB70F921F922F933F934F93A9
:104820005F936F937F938F939F93AF93BF93EF9318
:10483000FF931124C7D0FF91EF91BF91AF919F914A
:104840008F917F916F915F914F913F912F911F9029
:104850000F900CBF0F910BBF0F910460F894009361
:104860006E000F910FBF0F911895CF938091120298
:104870008F3790F08F5790917C0490933A0499234E
:1048800011F0759A01C075989091B704909339040E
:10489000992359F0A59A0AC090913A04891708F013
:1048A000759890913904891708F0A598805F8093D6
:1048B00012029091380481E0892780933804809116
:1048C000110285301CF4C1E0C80F01C0C0E0823085
:1048D000A1F184F4882329F1813009F062C010929B
:1048E0007B0080E480937C0080917A0080648093D8
:1048F0007A0057C0843009F43EC094F1853009F045
:1049000050C090913704911102C080933704809178
:104910003704815080933704882309F442C0C5E0EE
:1049200040C0809110028F5F80311CF48093100290
:1049300038C010921002F1DE34C080917A0086FDFA
:104940002DC0809178009091790020918104309160
:104950008204820F931F909382048093810421C06C
:1049600010927B0082E480937C0080917A008064C6
:1049700080937A0016C080917A0086FD11C08091E4
:104980007800909179002091A1043091A204820FC7
:10499000931F9093A2048093A10403C0C2E001C0BE
:1049A000C4E0C09311020E94252F80918806909147
:1049B0008906009729F001979093890680938806CD
:1049C000CF91089552CF1F93CF93DF93CDB7DEB72A
:1049D00028970FB6F894DEBF0FBECDBF182F609199
:1049E000C1047091C204072E000C880B990B0E9421
:1049F000B2AA69837A838B839C838091C50490914A
:104A0000C604A091C704B091C8048D839E83AF8370
:104A1000B8874DEFBE016F5F7F4FCE0105960E94B4
:104A2000D31A6091B8047091B904072E000C880B5A
:104A3000990B0E94B2AA69837A838B839C838091AD
:104A4000BC049091BD04A091BE04B091BF048D83BD
:104A50009E83AF83B8874FEFBE016F5F7F4FCE015C
:104A600005960E94D31A8BE593E00E940416812FCD
:104A700090E00E94131B6AE070E00E94871986E5AF
:104A800093E00E9404168091B7046AE070E090E021
:104A90000E94871928960FB6F894DEBF0FBECDBFCF
:104AA000DF91CF911F9108952F923F924F925F9285
:104AB0006F927F928F929F92AF92BF92CF92DF922E
:104AC000EF92FF920F931F93CF93DF93CDB7DEB793
:104AD000C155D1090FB6F894DEBF0FBECDBF6296A7
:104AE0009FAF8EAF6297162F4BAB2C962FAF2C97A4
:104AF0000E948711688B798B8A8B9B8B17FD04C072
:104B0000B4E1CB2ED12C03C0ACE3CA2ED12C6296DB
:104B1000AEADBFAD62972D913D914D915C912FA7A8
:104B200038AB49AB5AAB17FDB3C4E12E012E000CD4
:104B3000FF08F701EE0FFF1FEB5EFD4F60817181F3
:104B40006F507109072E000C880B990B0E94B2AAB6
:104B50009B01AC016FA578A989A99AA90E9413AC01
:104B60001816ECF480E196E0CF5ADF4F0FB6F894B8
:104B7000DEBF0FBECDBFDF91CF911F910F91FF9090
:104B8000EF90DF90CF90BF90AF909F908F907F90ED
:104B90006F905F904F903F902F900C9404168CEF85
:104BA00095E00E940416D7DAF701E458FB4F8FE72F
:104BB000808380E090E0A0E5B1E425968CAF9DAFC6
:104BC000AEAFBFAF25979601A8EEB3E00E9481ADCE
:104BD00021966CAF7DAF8EAF9FAF21979B01AC014B
:104BE00088899989AA89BB89280F391F4A1F5B1FA9
:104BF0002DAB3EAB4FAB58AF81E080935B02288971
:104C000039894A895B892EA33FA348A759A72AA3BC
:104C10003BA34CA35DA3812C912C54018C8A9D8ACB
:104C2000AE8ABF8A75016401188E30E4398F4CE179
:104C30004A8F56E45B8F1C8E1D8E1E8E1F8E1EA605
:104C400089AE9AAEABAEBCAE8FE790E0A0E0B0E02C
:104C50008E839F83A887B987EFE74E2E512C612C56
:104C6000712C1AA61BA61CA61DA691E09A871F866A
:104C70001E861982212C312C00E0812F012E000C80
:104C8000990BDC01A458BB4F2796BFAFAEAF279757
:104C9000880F991F880F991FFC01EB53FB4FF9A355
:104CA000E8A32BA9022E000C330B3CAB2BAB80915D
:104CB0005B02882309F4C1C20E9487116A837B8347
:104CC0008C839D8380918D04882309F424C1A6D808
:104CD00017FF0AC03091BC0439832090BD04309086
:104CE000BE040091BF0409C0A8A1B9A1BC91B983B9
:104CF000E8A1F9A12180328003812981322D432D41
:104D0000502F6C8D7D8D8E8D9F8D0E9410AA87FFF8
:104D100005C0F981FC8F2D8E3E8E0F8F2981322D9B
:104D2000432D502F688D798D8A8D9B8D0E9413ACF9
:104D300018162CF42981288F298E3A8E0B8F3A85EC
:104D4000332309F486C06296AEADBFAD6297BC91C5
:104D50002896BFAF28976296EEADFFAD6297F181BE
:104D60002996FFAF29976296AEADBFAD62971296B6
:104D7000BC912A96BFAF2A976296EEADFFAD6297BF
:104D8000F3812B96FFAF2B9728962FAD2897299666
:104D90003FAD29974B2F5F2F6981722D832D902F67
:104DA0000E9413AC18160CF0B6C02A813B814C81CE
:104DB0005D818EA19FA1A8A5B9A5281B390B4A0B1F
:104DC0005B0B60962CAF3DAF4EAF5FAF6097DA01E3
:104DD000C90188589341A109B109B7FD9CC0D3010D
:104DE000C2012E813F8148855985821B930BA40BFC
:104DF000B50BB595A7959795879517FF03C0809339
:104E0000B70405C02796EEADFFAD27978083609667
:104E10002CAD3DAD4EAD5FAD60972AA73BA74CA72B
:104E20005DA728963FAD28973C8F29964FAD2997CF
:104E30004D8F2A965FAD2A975E8F2B968FAD2B975D
:104E40008F8F2A813B814C815D812AA33BA34CA398
:104E50005DA36296AEADBFAD62972D913D914D9130
:104E60005C916981722D832D902F0E9410AA87FF7B
:104E70000DC38A819B81AC81BD812AA13BA14CA13C
:104E80005DA1821B930BA40BB50BAC01BD0148586F
:104E900053416109710977FDF9C24E855F85452B44
:104EA00009F0E6C18E819F81A885B985840D951D85
:104EB000A61DB71DB595A7959795879517FFE0C2D5
:104EC0008093B7042E853F852F5F3F4F3F872E8706
:104ED0006296AEADBFAD6297BC91B88F6296EEADF3
:104EE000FFAD6297F181F98F6296AEADBFAD62976B
:104EF0001296BC91BA8F6296EEADFFAD6297F381C8
:104F0000FB8F2A813B814C815D812EA33FA348A763
:104F100059A731E03A8720E030E040EA51E4629658
:104F2000AEADBFAD62976D917D918D919C910E94C8
:104F300037A99B01AC016981722D832D902F0E94AE
:104F400013AC18162CF488E895E00E94041675C17D
:104F50008A819B81AC81BD81288939894A895B8995
:104F6000821B930BA40BB50BB7FD9AC0812F17FDC5
:104F700080E029DD8AE00E9494188A819B81AC81BF
:104F8000BD818053984FAF4FBF4F888B998BAA8BB1
:104F9000BB8B9EA5911161C029AD3AAD4BAD5CAD07
:104FA0006981722D832D902F0E9413AC1816DCF5A9
:104FB00020E030E040E050E46981722D832D902F95
:104FC0000E9437A969AF7AAF8BAF9CAF2A813B8132
:104FD0004C815D8121968CAD9DADAEADBFAD21976D
:104FE000280F391F4A1F5B1F2DAB3EAB4FAB58AF8D
:104FF00025962CAD3DAD4EAD5FAD25976FA578A93B
:1050000089A99AA90E9436A99B01AC0191E09EA7AB
:105010006981722D832D902F0E9413AC18160CF409
:105020003FC01EA63DC08A819B81AC81BD812DA958
:105030003EA94FA958AD821B930BA40BB50BB7FD2E
:105040002FC01F3F19F043E655E002C045E755E089
:1050500064E575E0812FAFD823C020E030E040EA5E
:1050600051E46296AEADBFAD62976D917D918D9129
:105070009C910E9436A99B01AC016981722D832D00
:10508000902F0E9410AA87FF0BC01F3F19F04DE21E
:1050900055E002C040E455E06DE175E0812F8BD80A
:1050A0008A819B81AC81BD81880F991FAA1FBB1F7C
:1050B0002AA13BA14CA15DA1821B930BA40BB50BB4
:1050C0002EA13FA148A559A5821B930BA40BB50B9C
:1050D00081389F44A241B10528F08FEF94E00E94EF
:1050E0000416ABC04E855F858BA99CA984179507D4
:1050F0000CF0DDCD433051050CF4D9CD82EA94E0BB
:105100000E94041617FD05C02DE9622E24E0722EC0
:1051100004C09EE9692E94E0792E80E894E00E9414
:105120000416C3010E940416B701A60189E994E0A0
:105130000E944F168AE00E94941880E894E00E9432
:105140000416C3010E9404164C895D896E897F890B
:1051500085E994E00E944F168AE00E94941880E846
:1051600094E00E940416C3010E940416B501A40134
:1051700081E994E00E944F168AE00E9494182C96D0
:105180009FAD2C97992309F4A4C117FF2BC0C0929F
:10519000A304D092A404E092A504F092A6042CEA01
:1051A00035EC47E25EE36C897D898E899F890E9498
:1051B0004EAC6093A7047093A8048093A9049093C5
:1051C000AA042CEA35EC47E25EE3C501B4010E9473
:1051D00017AA6093AB047093AC048093AD049093D2
:1051E000AE0477C1ACE01A029001112489010B567C
:1051F0001B4FF801C082D182E282F3822CEA35ECA7
:1052000047E25EE36C897D898E899F890E944EAC5E
:10521000D80114966D937D938D939C9317972CEAE8
:1052200035EC47E25EE3C501B4010E9417AAF8011C
:1052300060877187828793874CC1CF5ADF4F0FB643
:10524000F894DEBF0FBECDBFDF91CF911F910F91BC
:10525000FF90EF90DF90CF90BF90AF909F908F9096
:105260007F906F905F904F903F902F900C94AB2069
:105270002AA53BA54CA55DA5280F391F4A1F5B1F1A
:105280002A873B874C875D872AA53BA54CA55DA552
:10529000281B390B4A0B5B0BCA01B9012E813F81D8
:1052A000488559850E9418AD2A853B854C855D85CA
:1052B0000E945DADD301C201820F931FA41FB51FD1
:1052C00084319105A105B105FCF02C013D018C3E16
:1052D0009105A105B1052CF06BEE462E512C612CE9
:1052E000712C40E84416510461047104DCF08EEF27
:1052F00090E0A0E0B0E084199509A609B7098E8373
:105300009F83A887B98712C054E1452E512C612C88
:10531000712C24E130E040E050E02E833F83488749
:10532000598704C04E825F8268867986B301A201E4
:1053300084EF95E00E943F164E815F8168857985F4
:105340008FEE95E00E943F16488D598D6A8D7B8DBA
:1053500088EE95E00E944F164C8D5D8D6E8D7F8D91
:1053600081EE95E00E944F164E855F8543305105D2
:105370000CF498CD6E817F81888599850E94B2AAB0
:1053800020E030E040E850E40E944EAC6B017C012C
:10539000288D398D4A8D5B8D6C8D7D8D8E8D9F8D89
:1053A0000E9436A92BED3FE049E450E40E944EAC48
:1053B00020E030E040E05FE30E944EAC9B01AC0196
:1053C000C701B6010E9417AA6B017C016A857B8523
:1053D0008C859D850E94B2AA2FE632E143E85AE30C
:1053E0000E944EAC4B015C01B701A6018BED95E02C
:1053F0000E944F16B501A40185ED95E00E944F165D
:105400002AE939E949E15FE3C701B6010E944EACE0
:105410006B017C019B01AC010E9437A9A50194019D
:105420000E9417AA6C8B7D8B8E8B9F8BA50194019C
:10543000C701B6010E944EAC20E030E040E05EE3E0
:105440000E944EAC4B015C0185EC95E00E94041675
:10545000B701A6018FEB95E00E944F164C895D893C
:105460006E897F8989EB95E00E944F16B501A401F2
:1054700083EB95E00E944F168AE00E94941812CDAB
:105480002796EEADFFAD279780831CCD1A8643CDBE
:1054900020E030E047E053E46FA578A989A99AA9F4
:1054A0000E9413AC18160CF45DCB8CEF95E00E94B3
:1054B00004160E94AB208FE78093B70420E030E011
:1054C00040E051E425962CAF3DAF4EAF5FAF25973E
:1054D0007ACBCF5ADF4F0FB6F894DEBF0FBECDBFE9
:1054E000DF91CF911F910F91FF90EF90DF90CF90C0
:1054F000BF90AF909F908F907F906F905F904F90F4
:105500003F902F900895CF92DF92EF92FF9280917B
:1055100071048823A1F10E948711C0906D04D0907E
:105520006E04E0906F04F0907004DC01CB018C19E4
:105530009D09AE09BF09B7FD22C00E9487116B010A
:105540007C012091710430E0A8EEB3E00E9481ADAF
:10555000DC01CB018C0D9D1DAE1DBF1D80936D0424
:1055600090936E04A0936F04B093700480E02BDAE4
:105570008AE0FF90EF90DF90CF900C949418FF900A
:10558000EF90DF90CF9008952F923F924F925F92CD
:105590006F927F928F929F92AF92BF92CF92DF9243
:1055A000EF92FF920F931F93CF93DF93CDB7DEB7A8
:1055B00063970FB6F894DEBF0FBECDBF888B698BA3
:1055C00081E080935B021A821B821C821D821886F6
:1055D00019861A861B8619821C862CE32D873CE1CE
:1055E0003E8746E44F87C12CD12C80E8E82E9FEB04
:1055F000F92E812C912C54016091C1047091C20448
:10560000072E000C880B990B0E94B2AA6A8B7B8B29
:10561000182F092F9B01482F592FB601C7010E944F
:1056200010AA8823A1F12091C5043091C6044091AD
:10563000C7045091C8046A897B89812F902F0E94EA
:1056400010AA881F8827881F89835989552319F133
:10565000882309F180915B0280915B0263960FB60B
:10566000F894DEBF0FBECDBFDF91CF911F910F9198
:10567000FF90EF90DF90CF90BF90AF909F908F9072
:105680007F906F905F904F903F902F900895CA8ABF
:10569000DB8A1E2D0F2D0E9487116B017C01DC011E
:1056A000CB01288539854A855B85821B930BA40B2A
:1056B000B50BB7FD34C0D701C60188519C4FAF4F21
:1056C000BF4F88879987AA87BB8788897CD98FE451
:1056D00093E00E94041681149104A104B104C9F05E
:1056E000D501C40188519C4FAF4FBF4FBC01CD01C4
:1056F0006C197D098E099F0928EE33E040E050E0E7
:105700000E943BADCA01B9014AE050E00E947619FF
:1057100003C08FE30E9494188AE00E9494180E94AC
:1057200097A80E9487116093F80B7093F90B8093F0
:10573000FA0B9093FB0B2090C5043090C604909117
:10574000C7049E83A091C804AF839101492F5A2FAB
:105750006A897B89812F902F0E9436A92B013C01F9
:1057600020E030E0A9010E9413AC87FF04C0C30110
:10577000B201905802C0C301B20120E030E040E223
:1057800051E481149104A104B10429F40E9410AAE7
:1057900087FF07C004C00E9413AC181614F446011A
:1057A0005701B981BB2391F12A813B814C815D81F5
:1057B000211531054105510541F0D701C601821B74
:1057C000930BA40BB50BB7FD21C091014E815F81F6
:1057D0006C857D858E859F850E9436A920E030E00E
:1057E00040EC5FE30E9410AA87FD34CFD701C601C9
:1057F000805A9541AF4FBF4F8A839B83AC83BD8353
:105800002C863D869E819E87AF81AF8780915B020B
:10581000882309F41FCF81149104A104B10429F451
:10582000CA88DB88E12EF02EE7CEB8EECB1AB3E0C3
:10583000DB0AE108F108C818D908EA08FB08F7FEF6
:1058400009CFEECF2F923F924F925F926F927F924D
:105850008F929F92AF92BF92CF92DF92EF92FF9280
:105860000F931F93CF93DF93CDB7DEB762970FB639
:10587000F894DEBF0FBECDBF888B81E080935B02C2
:105880001A821B821C821D82188619861A861B8624
:1058900019821C862CE32D873CE13E8746E44F8726
:1058A000C12CD12C80E8E82E9FEBF92E812C912C75
:1058B00054016091B8047091B904072E000C880B54
:1058C000990B0E94B2AA698B7A8B182F092F9B0122
:1058D000482F592FB601C7010E9410AA8823A1F1B1
:1058E0002091BC043091BD044091BE045091BF048E
:1058F00069897A89812F902F0E9410AA881F882792
:10590000881F89835889552319F1882309F18091CB
:105910005B0280915B0262960FB6F894DEBF0FBE09
:10592000CDBFDF91CF911F910F91FF90EF90DF904E
:10593000CF90BF90AF909F908F907F906F905F902F
:105940004F903F902F900895C98ADA8A1E2D0F2D0F
:105950000E9487116B017C01DC01CB012885398510
:105960004A855B85821B930BA40BB50BB7FD34C036
:10597000D701C60188519C4FAF4FBF4F8887998789
:10598000AA87BB8780E01FD88BE493E00E940416AF
:1059900081149104A104B104C9F0D501C401885156
:1059A0009C4FAF4FBF4FBC01CD016C197D098E09D3
:1059B0009F0928EE33E040E050E00E943BADCA0171
:1059C000B9014AE050E00E94761903C08FE30E94BB
:1059D00094188AE00E9494180E9497A80E94871148
:1059E0006093F80B7093F90B8093FA0B9093FB0B79
:1059F0009091BC049E83A091BD04AF832090BE040F
:105A00003090BF04292F3A2FA10169897A89812F0B
:105A1000902F0E9436A92B013C0120E030E0A90123
:105A20000E9413AC87FF04C0C301B201905802C0AA
:105A3000C301B20120E030E040EA50E48114910457
:105A4000A104B10429F40E9410AA87FF07C004C072
:105A50000E9413AC181614F446015701B981BB23F8
:105A600091F12A813B814C815D81211531054105F0
:105A7000510541F0D701C601821B930BA40BB50B56
:105A8000B7FD21C02E813F81A1016C857D858E856A
:105A90009F850E9436A920E030E040EC5FE30E9441
:105AA00010AA87FD34CFD701C601805A9541AF4F68
:105AB000BF4F8A839B83AC83BD839E819C87AF81CC
:105AC000AD872E863F8680915B02882309F41FCF25
:105AD00081149104A104B10429F4C988DA88E12E63
:105AE000F02EE7CEB8EECB1AB3E0DB0AE108F108FE
:105AF000C818D908EA08FB08F7FE09CFEECFCF9304
:105B0000C82F6115710519F0CB010E94041682EBB4
:105B100097E00E940416C11103C083EA97E002C017
:105B200088EA97E00E9404168AE0CF910C949418BA
:105B30008091D1048093D20408958091D004882369
:105B400019F01092D00408958EE098E00C94A3A769
:105B50008091D204811105C08091CC04811101C0D3
:105B6000089562E070E080E090E00E94C2158091AC
:105B7000CD04882339F061E070E080E090E00E947D
:105B8000C215F5CF08958093D2048093D104E0CF5D
:105B900026982E9A25982D9A24982C9A3F98479AC1
:105BA0000A98129A0998119A81E0EDCF8093D20455
:105BB000CFCF8093CC04CCCF8091D004882339F10F
:105BC0009091D0048091CB04981709F10E9412168D
:105BD0008FEF97E00E9404168091D00480FD1CC0D6
:105BE0008091D00484FD18C08091D00481FD1EC036
:105BF0008091D00485FD1AC08091D00482FD20C020
:105C00008091D00486FD1CC08AE00E949418809187
:105C1000D0048093CB04089580E00E940E58AB011D
:105C2000BC018BEF97E00E944F16DECF81E00E940F
:105C30000E58AB01BC0187EF97E00E944F16DCCFF6
:105C400082E00E940E58AB01BC0183EF97E00E94F6
:105C50004F16DACFCF9389ED97E00E94041683B1F7
:105C6000C1E086FB882780F963ED77E08C2747DF6A
:105C700086B180956DEC77E0881F8827881F3FDF0D
:105C800083B185FB882780F967EC77E08C2737DFC5
:105C900080B182FB882780F961EC77E08C272FDFC9
:105CA00083B1829581706BEB77E08C2728DF80B120
:105CB0008695817065EB77E08C27CF9120CF80911E
:105CC000CF041E9904C081608093CF0403C08E7FEF
:105CD0008093CF048091CF04379904C08061809372
:105CE000CF0403C08F7E8093CF048091CF041D9991
:105CF00004C082608093CF0403C08D7F8093CF0463
:105D00008091CF04029904C080628093CF0403C0C5
:105D10008F7D8093CF048091CF041C9904C0846050
:105D20008093CF0403C08B7F8093CF048091CF04F6
:105D3000019904C080648093CF0403C08F7B80935B
:105D4000CF049091CA048091CF04981731F092E06B
:105D50009093CD048093CA0409C08091CD04882318
:105D600029F081508093CD04882349F08091D2049A
:105D7000811108C08091CC04811104C008959093D2
:105D8000CE04F4CF8091410580FF1BC09091420565
:105D90008091CE0490FF0BC080FF13C08091D0048F
:105DA00081608093D00480E00E940C580AC084FF78
:105DB00008C08091D00480618093D00480E00E946C
:105DC0000C588091410581FF1BC090914205809144
:105DD000CE0491FF0BC081FF13C08091D00482607C
:105DE0008093D00481E00E940C580AC085FF08C04F
:105DF0008091D00480628093D00481E00E940C588E
:105E00008091410582FF20C08091420582FF10C031
:105E10008091CC048823C1F08091CE0482FF14C00D
:105E20008091D00484608093D00482E00C940C585C
:105E30008091CE0486FF08C08091D0048064809356
:105E4000D00482E00C940C58089539CFCF93882366
:105E5000A1F0C82F0E94121684E50E9494186AE0EF
:105E600070E08C2F90E00E94871980E20E949418C5
:105E70008CE198E0CF910C940416CF910895089589
:105E800080918D0690918A06891B8F7019F480E0AD
:105E900090E0089590918706992351F0833030F473
:105EA0008FEF890F19F080938706F1CF1092870644
:105EB000E0918A0686E5E89FF0011124E257F94F48
:105EC000808180FDE4CF80918A068F5F8F70809300
:105ED0008C0690918A0680918B06981306C080915B
:105EE0008C0680938B06CF010895CF010895EFE6CD
:105EF000F0E080818260808308958091420580FF78
:105F000009C080910B018270809309018FEF80930B
:105F1000D30409C080910B018095827080930901A0
:105F200081E08093D3048091420581FF0AC0809173
:105F30000B0180958170809309018FEF8093D404C9
:105F400008C080910B0181708093090181E08093EA
:105F5000D4048091420582FF09C080910B018470B6
:105F6000809309018FEF8093D50409C080910B01C4
:105F7000809584708093090181E08093D5040000AE
:105F80000000000008950F930FB70F9300916E006B
:105F90000F930B7F00936E0000916F000D7F0093B5
:105FA0006F000F930BB70F930CB70F921F922F93A5
:105FB0003F934F935F936F937F938F939F93AF9391
:105FC000BF93EF93FF9311240E94A338FF91EF91A9
:105FD000BF91AF919F918F917F916F915F914F9101
:105FE0003F912F911F900F900CBF0F910BBF0F91FE
:105FF0000260F89400936F000F9100936E000F9170
:106000000FBF0F911895CF92DF92EF92FF920F93EF
:106010001F93809140058823D1F010924005809114
:10602000430590914405892B91F0109241051092FF
:1060300044051092430590918D0680918A06981729
:1060400031F080918A068F5F8F7080938A068091ED
:10605000430590914405892B09F4AAC140910F058D
:1060600050911005609111057091120590913705BE
:106070000091030510910405209105053091060556
:10608000041B150B260B370B892F90E0A0E0B0E026
:10609000081719072A073B0710F4D901C801E82F90
:1060A000840F951FA61FB71F80930F0590931005AF
:1060B000A0931105B09312052091840030918500C2
:1060C000225E3F4F40912705509128056091290598
:1060D00070912A058091170590911805A0911905D6
:1060E000B0911A05840F951FA61FB71F809327052F
:1060F00090932805A0932905B0932A05B7FD1CC0ED
:10610000409A4091D7045091D8046091D90470917D
:10611000DA048091D304082E000C990BAA0BBB0B58
:10612000840F951FA61FB71F8093D7049093D804A0
:10613000A093D904B093DA0440912B0550912C051B
:1061400060912D0570912E0580911B0590911C0585
:10615000A0911D05B0911E05840F951FA61FB71FA6
:1061600080932B0590932C05A0932D05B0932E05BD
:10617000B7FD1CC0419A4091DB045091DC04609152
:10618000DD047091DE048091D404082E000C990B7C
:10619000AA0BBB0B840F951FA61FB71F8093DB04B0
:1061A0009093DC04A093DD04B093DE0440912F05AE
:1061B00050913005609131057091320580911F0535
:1061C00090912005A0912105B0912205840F951F83
:1061D000A61FB71F80932F0590933005A09331051C
:1061E000B0933205B7FD1CC0429A4091DF04509134
:1061F000E0046091E1047091E2048091D504082EDE
:10620000000C990BAA0BBB0B840F951FA61FB71F81
:106210008093DF049093E004A093E104B093E20440
:1062200040913305509134056091350570913605E4
:106230008091230590912405A0912505B091260514
:10624000840F951FA61FB71F8093330590933405C5
:10625000A0933505B0933605B7FD3CC0C090E3046C
:10626000D090E404E090E504F090E6044091D60478
:10627000042E000C550B660B770B4C0D5D1D6E1D2F
:106280007F1D4093E3045093E4046093E50470930E
:10629000E604409113055091140560911505709125
:1062A0001605841B950BA60BB70B809333059093B3
:1062B0003405A0933505B093360590914205809141
:1062C000F80493FF04C081508093F80403C08F5FEB
:1062D0008093F80480918400909185008217930741
:1062E000C8F38091270590912805A0912905B091C8
:1062F0002A05B7FD15C04091130550911405609112
:10630000150570911605841B950BA60BB70B809392
:10631000270590932805A0932905B0932A05409856
:1063200080912B0590912C05A0912D05B0912E0503
:10633000B7FD15C0409113055091140560911505E6
:1063400070911605841B950BA60BB70B80932B053C
:1063500090932C05A0932D05B0932E054198809124
:106360002F0590913005A0913105B0913205B7FD10
:1063700015C0409113055091140560911505709159
:106380001605841B950BA60BB70B80932F059093D6
:106390003005A0933105B09332054298E15041F0A9
:1063A000809184009091850082179307C8F388CE6E
:1063B0001F910F91FF90EF90DF90CF900895CF92B3
:1063C000DF92EF92FF928091F704882309F465C071
:1063D000C0900F05D0901005E0901105F0901205C7
:1063E00040910705509108056091090570910A05D3
:1063F0008091F8044C155D056E057F05E8F4209149
:10640000FD043091FE04E091FB04F091FC04E217DE
:10641000F30790F481508093F804215031093093B0
:10642000FE042093FD0440912102509122026091CC
:1064300023027091240234C0C416D506E606F7067E
:10644000E8F42091FD043091FE044091F90450914C
:10645000FA042417350790F48F5F8093F8042F5FB8
:106460003F4F3093FE042093FD0440912102509150
:106470002202609123027091240212C08FEF9FEFDD
:10648000DC018093210290932202A0932302B09317
:1064900024024FEF5FEFBA0103C04FEF5FEFBA0185
:1064A0008091F80487FD06C080910B018074809371
:1064B000090106C080910B018095807480930901C9
:1064C0002091840030918500225E3F4F8091F80436
:1064D000882311F1439A809184009091850082175E
:1064E0009307C8F38091F80487FF04C08F5F8093FF
:1064F000F80403C081508093F80443988091F80415
:10650000882321F38091840090918500821793075E
:10651000C8F3225E3F4FDACFCB01BA01FF90EF9074
:10652000DF90CF900895BC01209143053091440540
:1065300040914305509144052417350711F09A0105
:10654000F7CF81E06217730709F080E00895CF93D9
:10655000DF93EC0188819981AA81BB81E7EDF4E0AA
:1065600080839183A283B383EB0188819981AA817F
:10657000BB8184839583A683B783EA01888199814F
:10658000AA81BB8180879187A287B387E90188812F
:106590009981AA81BB8184879587A687B787DF9178
:1065A000CF9108953F924F925F926F927F928F9218
:1065B0009F92AF92BF92CF92DF92EF92FF920F9392
:1065C0001F93CF93DF93CDB7DEB728970FB6F8941C
:1065D000DEBF0FBECDBFA0914305B091440510971B
:1065E00039F180900F0590901005A0901105B090A2
:1065F00012054091030550910405609105057091C5
:10660000060584169506A606B706C8F01092410541
:10661000109244051092430590918D0680918A0650
:10662000981731F080918A068F5F8F7080938A0669
:1066300070EDC72E77E0D72EE12CF12C97C1409159
:106640000B0550910C0560910D0570910E054815D4
:1066500059056A057B0508F46EC000913C05109150
:106660003D0520913E0530913F05D1964D915D91BC
:106670006D917C91D497EE27059FF12D169FC00157
:10668000269F900D259F800D911D069FF00D811D69
:106690009E1F159FF00D811D9E1F249FF00D811DD3
:1066A0009E1F149FF10D8E1F9E1FF6958E1F9E1F1D
:1066B000709F800D911D719F900D1124FD01EB5B6A
:1066C000FF4F4081518162817381480F591F611DC5
:1066D000711D4093F3045093F4046093F504709398
:1066E000F6043497C080D180E280F380C416D506CA
:1066F000E606F70640F4C092F304D092F404E09268
:10670000F504F092F6044091F3045091F404609182
:10671000F5047091F6048AE798E0BB24B394FC0179
:10672000C590D590E590F490C416D506E606F70618
:1067300008F475C27FC2409007055090080560902C
:10674000090570900A05481459046A047B0408F08E
:1067500080C0209138053091390540913A0550911B
:106760003B052D833E834F835887D1960D911D9114
:106770002D913C91D4974D815E816F817885EE2774
:10678000419FF12D529FC001629F900D619F800D2E
:10679000911D429FF00D811D9E1F519FF00D811D87
:1067A0009E1F609FF00D811D9E1F509FF10D8E1F3B
:1067B0009E1FF6958E1F9E1F349F800D911D359F45
:1067C000900D11248C0120E030E0C090F304D090B3
:1067D000F404E090F504F090F604CD01875B9F4F40
:1067E000FC010C151D052E053F05C0F440815181AB
:1067F0006281738149835A836B837C83C01AD10A77
:10680000E20AF30AC416D506E606F70610F46A0192
:106810007B018AE798E03324339410C0C080D18094
:10682000E280F380F6CFF694E794D794C794330CC4
:10683000049628E08639920709F480C2FC0105918C
:106840001591259134910C151D052E053F0558F322
:1068500075C28091F8048823D9F0D7964D915C9148
:10686000D89760E070E000912102109122022091FF
:10687000230230912402041715072607370741F039
:1068800010922502109226021092270210922802DE
:1068900040911D0250911E0260911F0270912002D2
:1068A00077FF5CC0AF5BBF4F8D919D910D90BC9108
:1068B000A02D2AE738E041E0F901C590D590E59098
:1068C000F490C816D906EA06FB0658F4B695A795C3
:1068D00097958795440F2C5F3F4F58E02639350731
:1068E00059F74093370580329105A105B10520F491
:1068F00080E290E0A0E0B0E08097A109B1098115A5
:1069000078E09707A105B10508F4CEC224E0929F74
:10691000F00111249F012656334FF90132966591FB
:106920007491EE27879FA001869F410D5E1F0694FC
:106930004E1F5E1F112460E070E0F9018591949173
:10694000A0E0B0E0841B950BA60BB70B80931D0253
:1069500090931E02A0931F02B0932002C0901D02CC
:10696000D0901E02E0901F02F0902002809143051B
:1069700090914405892B09F01DC382DA9093440558
:1069800080934305892B09F415C3E0914305F091E9
:106990004405808183FF19C09F012F5D3F4FAF01E8
:1069A000435E5F4FBF01675E7F4FCF014596CFDDEE
:1069B00090918D0680918A069817F9F280918A0647
:1069C0008F5F8F7080938A06D8CFC588D688E78876
:1069D000F08C81E0C114D104E104F10409F480E0F9
:1069E000018D128D238D348D011511052105310581
:1069F00009F08260458D568D678D70A14115510556
:106A00006105710509F08460809341051092380595
:106A10001092390510923A0510923B0510923C05F0
:106A200010923D0510923E0510923F0585A196A15A
:106A3000A7A1B0A58093030590930405A093050535
:106A4000B0930605882499245401881A990AAA0A41
:106A5000BB0A8092330590923405A0923505B0921E
:106A6000360580922F0590923005A0923105B092A4
:106A7000320580922B0590922C05A0922D05B092A4
:106A80002E058092270590922805A0922905B092A4
:106A90002A05CC0CDD1CEE1CFF1CC0921705D09201
:106AA0001805E0921905F0921A05000F111F221F18
:106AB000331F00931B0510931C0520931D05309375
:106AC0001E05440F551F661F771F40931F055093E7
:106AD0002005609321057093220541A152A163A175
:106AE00074A1440F551F661F771F409323055093D1
:106AF00024056093250570932605880F991FAA1F0A
:106B0000BB1F8093130590931405A0931505B093B4
:106B1000160510920F051092100510921105109293
:106B2000120581A592A5A3A5B4A580930B0590930A
:106B30000C05A0930D05B0930E0585A596A5A7A5F8
:106B4000B0A98093070590930805A0930905B09319
:106B50000A0586A98093F704882309F183AD94ADD3
:106B60009093FC048093FB0481AD92AD9093FA0462
:106B70008093F904109225021092260210922702A7
:106B80001092280287A990ADA0E0B0E08093210286
:106B900090932202A0932302B09324020BC08FEFA4
:106BA0009FEFDC018093210290932202A0932302A5
:106BB000B093240285A990914205891719F080931A
:106BC00042059BD97CD88FEF9FEFDC0180931D029B
:106BD00090931E02A0931F02B0932002E091430500
:106BE000F0914405EB5BFF4F80819181A281B381DD
:106BF0008093F3049093F404A093F504B093F60407
:106C00002AE738E041E0F901C590D590E590F4908D
:106C1000C816D906EA06FB0608F46BC176C176955C
:106C2000679557954795BB0C0496E8E086399E0713
:106C300009F075CDB09237054032510561057105F7
:106C400020F440E250E060E070E0405251096109F8
:106C50007109411588E058076105710500F194E05C
:106C6000599FF0011124CF018656934FFC013296B3
:106C7000E590F490F701DD244F9F50014E9FA10C49
:106C8000BD1C0694AD1CBD1C1124FC01C590D49004
:106C9000E12CF12CCA18DB08E108F10824C06A01D4
:106CA0007B01F694E794D794C794F601EC7FCF016B
:106CB0008656974F7C01FC0185919491F70132969D
:106CC000E590F49047704E9DB0014F9D700D1124DA
:106CD000AB0163E0569547956A95E1F76C01C41ADC
:106CE000D50AE12CF12C0C0D1D1D2E1D3F1D00930E
:106CF0003C0510933D0520933E0530933F05909150
:106D0000F7048091F804992309F465C0882309F4F5
:106D10002DCED7968D919C91D897A0E0B0E0409170
:106D2000210250912202609123027091240248179F
:106D300059076A077B0709F051C018CE3092370512
:106D4000F0E2CF16D104E104F10428F430E2C32EBE
:106D5000D12CE12CF12CF0E2CF1AD108E108F10896
:106D6000C11428E0D206E104F10408F440C034E084
:106D7000D39EC00111248656934FFC013296059193
:106D800014916C2D3327619FA001609F410D531F0B
:106D90000694431F531F1124FC01C590D490E12C8D
:106DA000F12CC41AD50AE108F1084D815E816F818A
:106DB00078854C0D5D1D6E1D7F1D409338055093E9
:106DC000390560933A0570933B058091F704811172
:106DD00032C08091F804882309F4C8CD10922502AE
:106DE000109226021092270210922802BFCD97011E
:106DF00086013695279517950795F801EC7FCF0109
:106E00008656974FFC0105911491FC0132964591ED
:106E100054913C2D3770349FC001359F900D112443
:106E200023E0969587952A95E1F76801C81AD90A53
:106E3000E12CF12CBACF430C511C611C711C48147D
:106E400059046A047B04C8F48091F804882309F487
:106E50008DCDD7964D915C91D89760E070E0009110
:106E60002102109122022091230230912402041762
:106E700015072607370709F479CD109225021092DD
:106E800026021092270210922802D7968D919C918B
:106E9000D897A0E0B0E08093210290932202A093C3
:106EA0002302B093240262CDAC01BD0176956795B3
:106EB00057954795FA01EC7FAF014656574FFA01B7
:106EC00025913491FA013296659174918770869F6D
:106ED000A001879F500D1124CA01F3E09695879574
:106EE000FA95E1F7A901481B590BCA01A0E0B0E0EF
:106EF0002DCDB695A79597958795440F2C5F3F4F5D
:106F000068E02639360709F07ECE40933705803297
:106F10009105A105B10520F480E290E0A0E0B0E089
:106F20008097A109B109811558E09507A105B10520
:106F3000F8F064E0969FF00111249F012656334F2C
:106F4000F901329665917491EE27879FA001869F83
:106F5000410D5E1F06944E1F5E1F1124F901C5905E
:106F6000D490E12CF12CC41AD50AE108F10822C012
:106F7000AC01BD017695679557954795FA01EC7F71
:106F8000AF014656574FFA01C590D490FA01329698
:106F9000459154918770849F9001859F300D1124F5
:106FA000C901A3E096958795AA95E1F7C81AD90A71
:106FB000E12CF12CC701B60128960FB6F894DEBF7C
:106FC0000FBECDBFDF91CF911F910F91FF90EF903A
:106FD000DF90CF90BF90AF909F908F907F906F90F9
:106FE0005F904F903F900895CF92DF92EF92FF9283
:106FF0001F93CF93DF938FEF9FEF90938900809340
:1070000088001AE0C0E0D0E078948091FF0490916D
:107010000005A0910105B0910205892B8A2B8B2BCD
:1070200011F40E9403308091250290912602A091D4
:107030002702B0912802892B8A2B8B2B49F4BFD9C8
:107040006093250270932602809327029093280272
:107050008091FF0490910005A0910105B091020577
:10706000892B8A2B8B2B49F49DDA6093FF04709354
:1070700000058093010590930205C090FF04D09015
:107080000005E0900105F090020540912502509125
:1070900026026091270270912802FC2DED2D3E2DD5
:1070A0002F2D4C155D056E057F0520F4F42FE52F7F
:1070B000362F272F8F2F9E2FA32FB22F009721E03F
:1070C000A207B10520F08FEF9FEFA0E0B0E0C81A53
:1070D000D90AEA0AFB0AC092FF04D0920005E092A6
:1070E0000105F09202054F3F2FEF5207620772072A
:1070F00061F0481B590B6A0B7B0B409325025093A0
:1071000026026093270270932802F894209184004D
:1071100030918500205F3F4F115039F0C80FD91FC3
:10712000C217D30708F470CF01C0E901D0938900DA
:10713000C09388007894DF91CF911F91FF90EF90DA
:10714000DF90CF90089550CF90916F0091FB222750
:1071500020F991FF05C090916F009D7F90936F0083
:1071600094E0899FF0011124E952FB4F6081718105
:1071700082819381222329F020916F002260209345
:107180006F00089590916F0091FB222720F991FFE5
:1071900005C090916F009D7F90936F0034E0839FB6
:1071A000C0011124FC01E952FB4F408151816281F1
:1071B0007381FC01E951FB4F4083518362837383E8
:1071C00081E080934005222329F080916F00826046
:1071D00080936F00089590916F0091FB222720F912
:1071E00091FF05C090916F009D7F90936F0094E098
:1071F000899FF0011124E951FB4F608171818281E7
:107200009381222329F020916F00226020936F0048
:1072100008954F925F926F927F928F929F92AF925A
:10722000BF92CF92DF92EF92FF9280916F0081FB2D
:10723000992790F981FF05C080916F008D7F809321
:107240006F004090D7045090D8046090D90470909B
:10725000DA048090DB049090DC04A090DD04B09010
:10726000DE04C090DF04D090E004E090E104F090F0
:10727000E204992329F080916F00826080936F006F
:1072800080E798E00E9404164AE050E0C301B20192
:107290000E9476198CE698E00E9404164AE050E0BD
:1072A000C501B4010E94761988E698E00E94041690
:1072B0004AE050E0C701B6010E9476198AE0FF90CB
:1072C000EF90DF90CF90BF90AF909F908F907F9086
:1072D0006F905F904F900C949418DB01833070F4A2
:1072E00094E0899FF0011124EB5BFA4FAB01770F1B
:1072F000660B770B4083518362837383813091F0F7
:1073000018F08230E9F008952FEF30E00E9490AD40
:1073100020ED37E040E050E00E945DADB9018EE223
:107320000C9453122FEF30E00E9490AD20ED37E027
:1073300040E050E00E945DADB9018DE20C94531223
:107340002FEF30E00E9490AD20ED37E040E050E0BC
:107350000E945DADB9018CE20C945312CF93DF9380
:10736000C5E4D5E06881798180E0B7DF6C817D81FB
:1073700081E0B3DF6885798582E0DF91CF91ADCF81
:10738000EAE0F1E080818860808380818061808391
:10739000808180628083E2DFE1E2F1E08081887FAA
:1073A00081608083089567FD2CC0813061F028F0F2
:1073B000823099F08330D9F024C0662311F0A19A6D
:1073C0002AC0A19828C08091080161118095807819
:1073D0008093060147FF27C008958091080161113D
:1073E000809580748093060147FF23C008958091A3
:1073F00008016111809588708093060147FF21C0C4
:10740000089547FD26C0813071F038F0823089F050
:107410008330B9F0089547FD1CC0442311F0A09AB1
:107420000895A0980895442311F0A29A0895A2986F
:107430000895809108014111809580728093060122
:107440000895809108014111809580718093060113
:1074500008950895643091F040F4613059F062303D
:10746000A9F420E040E061E09ECF683059F060313F
:1074700049F00CC020E040E060E095CF20E041E022
:1074800060E091CF20E041E061E08DCF0E941516D1
:1074900080E598E00C9404160F931F93CF93999A6C
:1074A000989A809107018068809307019A9A809149
:1074B00007018064809307018091070180628093B7
:1074C000070180910701886080930701809107017F
:1074D0008061809307010DE013E0C0E0F801619145
:1074E0008F018C2FB7DFCF5FC630C1F7CF911F91CF
:1074F0000F91089545DFD0DFEAE0F1E080818260FE
:1075000080838081816080838081846080838081AA
:10751000806480830F9A179A0E9A169A0D9A159A7C
:107520000C9A149A389A4098179A80918A058E7FFF
:1075300080938A05399A4198169A80918A058D7FA1
:1075400080938A053A9A4298159A80918A058B7F92
:1075500080938A053B9A4398149AA0E8B0E08C91F6
:107560008C7F8C93E1E8F0E08081877E8860808367
:107570008C918F738C938081887F8260808380E080
:1075800090E4909389008093880010928500109277
:107590008400EFE6F0E0808182608083789482E06E
:1075A000809342050C947D2F8BE398E00E94041693
:1075B000919902C080E301C081E30E9494189099E0
:1075C00002C080E301C081E30E94941887E398E041
:1075D0000E94041680910601881F8827881F805DFD
:1075E0000E949418929902C080E301C081E30E9436
:1075F000941883E398E00E9404168091060186FDAA
:1076000002C080E301C081E30E94941880910601CA
:1076100085FD02C080E301C081E30E9494188EE2E0
:1076200098E00E9404168091060183FD02C080E369
:1076300001C081E30E9494188091060184FD02C07C
:1076400080E301C081E30C949418CF93DF93CDB70E
:10765000DEB760970FB6F894DEBF0FBECDBF809146
:10766000790590917A05A0917B05B0917C0589837D
:107670009A83AB83BC8380917D0590917E05A09118
:107680007F05B09180058D839E83AF83B8878091FD
:10769000810590918205A0918305B0918405898729
:1076A0009A87AB87BC878091850590918605A091CC
:1076B0008705B09188058D879E87AF87B88B0E941C
:1076C000BE686091500270915102072E000C880B29
:1076D000990B0E94B2AA2AE037ED43E25CE30E94D4
:1076E0004EAC60934C0270934D0280934E02909387
:1076F0004F0280E00E94CE4E81E00E94CE4E82E09A
:107700000E94CE4E2BDE0E94056940E150E069E701
:1077100075E0CE0101960E94C8B1892B51F06096A8
:107720000FB6F894DEBF0FBECDBFDF91CF910C94A2
:10773000F54B60960FB6F894DEBF0FBECDBFDF915C
:10774000CF9108958734924041F00E94151680EE43
:1077500093E10E94041681E0089580E00895EF927D
:10776000FF920F931F93CF93DF93CDB7DEB7C4582B
:10777000D1090FB6F894DEBF0FBECDBFED961CAE9B
:107780001DAE1EAE1FAEED9785E492E5A2E5B0E01A
:10779000E9968CAF9DAFAEAFBFAFE997CF57DF4F44
:1077A00019821882C158D04084E690E0C158DF4F5A
:1077B00099838883CF57D0400E94B116109252050A
:1077C0009E012F573F4F44E050E0BE016B587F4F62
:1077D000CE0181589F4F0E94B516C158DF4F888156
:1077E0009981CF57D0400296C158DF4F9983888343
:1077F000CF57D040CF57DF4F19821882C158D040A1
:1078000081E0CC57DF4F8883C458D0409E012F576A
:107810003F4F41E050E0BE016C577F4FCE01815891
:107820009F4F0E94B5169E012F573F4F48E450E0EE
:107830006FE376E0CE0181589F4F0E94B5169E01FE
:107840002F573F4F40E150E06FE076E0CE01815886
:107850009F4F0E94B5168AE097EDA3EABCE3ED9630
:107860008CAF9DAFAEAFBFAFED979E012F573F4F8F
:1078700044E050E0BE0167587F4FCE0181589F4FD2
:107880000E94B5168E010F5F1F4F8CE0F801119218
:107890008A95E9F79E012F573F4F4CE050E0B80121
:1078A000CE0181589F4F0E94B51680E090E0A0E283
:1078B000B1E489839A83AB83BC839E012F573F4FEA
:1078C00044E050E0B801CE0181589F4F0E94B516A8
:1078D000ED961CAE1DAE1EAE1FAEED9783E0AE96CC
:1078E0008FAFAE9789839E012F573F4F44E050E002
:1078F000BE0167587F4FCE0181589F4F0E94B51639
:107900009E012F573F4F41E050E0BE0163597F4F2A
:10791000CE0181589F4F0E94B5169E012F573F4FB1
:1079200041E050E0B801CE0181589F4F0E94B5164A
:107930002AE0F22EFA949E012F573F4F44E050E088
:10794000FF2049F0BE0167587F4FCE0181589F4FFD
:107950000E94B516EFCF63E575E0CE0181589F4FC9
:107960000E94B5169E012F573F4F44E250E06AEE49
:1079700075E0CE0181589F4F0E94B51683E0CD5728
:10798000DF4F8883C358D040EE968FAFEE97E196D5
:107990001CAE1DAE1EAE1FAEE19719821A821B826D
:1079A0001C82ED961CAE1DAE1EAE1FAEED979E0165
:1079B0002F573F4F41E050E0BE016D577F4FCE0142
:1079C00081589F4F0E94B5169E012F573F4F41E0AF
:1079D00050E0BE0163587F4FCE0181589F4F0E94F7
:1079E000B5169E012F573F4F44E050E0B801CE013D
:1079F00081589F4F0E94B5169E012F573F4F44E07C
:107A000050E0BE0163597F4FCE0181589F4F0E94C5
:107A1000B5169AE0E92EF12CF1E0EF1AF10871F0B9
:107A20009E012F573F4F44E050E0BE0167587F4F03
:107A3000CE0181589F4F0E94B516EECFAE961FAE75
:107A4000AE978FEF89839E012F573F4F41E050E063
:107A5000BE0163597F4FCE0181589F4F0E94B516DA
:107A60009E012F573F4F41E050E0B801CE018158B1
:107A70009F4F0E94B51680E1F82EF8018F2D1192CC
:107A80008A95E9F79E012F573F4F40E150E0B8013A
:107A9000CE0181589F4F0E94B51688EC90E0AF96BA
:107AA0009FAF8EAFAF9780EF90E0E1969FAF8EAF24
:107AB000E19786E490E09A8389838EE690E09C8348
:107AC0008B83EE961FAEEE97EF961FAEEF979E015B
:107AD0002F573F4F44E050E0BE0163597F4FCE0126
:107AE00081589F4F0E94B5169E012F573F4F44E08B
:107AF00050E0B801CE0181589F4F0E94B5169E01FB
:107B00002F573F4F42E050E0BE0163587F4FCE01F8
:107B100081589F4F0E94B516F8011192FA94E9F727
:107B200080E090E0A0E8BFE38D879E87AF87B88BA9
:107B30008091950490919604A0919704B091980437
:107B400089839A83AB83BC838091990490919A0432
:107B5000A0919B04B0919C048D839E83AF83B887D2
:107B600080919D0490919E04A0919F04B091A004E7
:107B700089879A87AB87BC879E012F573F4F40E18B
:107B800050E0B801CE0181589F4F0E94B51684E1A4
:107B900090E09A8389839E012F573F4F42E050E047
:107BA000B801CE0181589F4F0E94B5169E012F57F4
:107BB0003F4F4CE050E063EA74E0CE0181589F4FA4
:107BC0000E94B51680E290E09A8389839E012F5728
:107BD0003F4F42E050E0B801CE0181589F4F0E94D4
:107BE000B51681E089839E012F573F4F41E050E059
:107BF000B801CE0181589F4F0E94B51680E2EDE595
:107C0000F2E0D80101900D928A95E1F79E012F577D
:107C10003F4F40E250E0B801CE0181589F4F0E9493
:107C2000B516AE961FAEAE979E012F573F4F41E05F
:107C300050E0BE0163597F4FCE0181589F4F0E9493
:107C4000B516198280E090E0A0E4B0E4ED968CAF28
:107C50009DAFAEAFBFAFED979E012F573F4F41E0B5
:107C600050E0B801CE0181589F4F0E94B5169E0189
:107C70002F573F4F44E050E0BE0167587F4FCE0181
:107C800081589F4F0E94B5168AE1F80111928A959A
:107C9000E9F79E012F573F4F4AE150E0B801CE016E
:107CA00081589F4F0E94B51684E3EDE7F2E0D801BA
:107CB00001900D928A95E1F79E012F573F4F44E3C3
:107CC00050E0B801CE0181589F4F0E94B5161A822C
:107CD00019821C821B821E821D829E012F573F4FDC
:107CE00046E050E0B801CE0181589F4F0E94B51682
:107CF0008DE0F80111928A95E9F79E012F573F4FC9
:107D00004DE050E0B801CE0181589F4F0E94B5165A
:107D10009E012F573F4F44E050E061EB75E0CE01EC
:107D200081589F4F0E94B5169E012F573F4F4CE040
:107D300050E065E475E0CE0181589F4F0E94B51672
:107D40008CE6F80111928A95E9F79E012F573F4F73
:107D50004CE650E0B801CE0181589F4F0E94B51605
:107D60009E012F573F4F4CE050E06EED75E0CE0185
:107D700081589F4F0E94B516E1961CAE1DAE1EAEF7
:107D80001FAEE197E5961CAE1DAE1EAE1FAEE59789
:107D90009E012F573F4F48E050E0BE0163597F4F8F
:107DA000CE0181589F4F0E94B516809152058111D6
:107DB0004FC0C158DF4F08811981CF57D0400456BA
:107DC0001109CF57DF4F88819981C158D040AF96B4
:107DD0009FAF8EAFAF9784E690E0C158DF4F998395
:107DE0008883CF57D0409E012F573F4F44E050E04B
:107DF00063E173E0CE0181589F4F0E94B5169E014A
:107E00002F573F4F42E050E0BE0163597F4FCE01F4
:107E100081589F4F0E94B5160E941216B8018EEC31
:107E200093E10E946F16AF964EAD5FADAF9760E0E5
:107E300070E081EC93E10E9479168EEB93E10E9451
:107E40000416C8017FDC90915205892B809352055E
:107E50000E94B3169091520581E08927CC57DF4FDD
:107E60000FB6F894DEBF0FBECDBFDF91CF911F914B
:107E70000F91FF90EF9008951F93CF93DF93CDB7AD
:107E8000DEB72C970FB6F894DEBF0FBECDBFAFE3C1
:107E9000B6E020E030E0C9012430310510F083E085
:107EA00090E0880F991F880F991FFC01E45FFC4E3A
:107EB000459155916591749154964D935D936D9351
:107EC0007C935797FC01E450FD4E45915591659187
:107ED000749194964D935D936D937C939797FC0169
:107EE000E451FD4E45915591659174914D935D938B
:107EF0006D937D932F5F3F4F2430310509F0CBCF39
:107F000080E29EE4A0E0B0E080934F06909350069C
:107F1000A0935106B093520680E090E0AAEFB4E43B
:107F20008093730690937406A0937506B0937606BB
:107F300040E050E86BE375E4409377065093780691
:107F40006093790670937A0680937B0690937C0603
:107F5000A0937D06B0937E0610927F061092800655
:107F60001092810610928206109283061092840667
:107F7000109285061092860680E090E0A0E4B1E4BD
:107F800080930F0690931006A0931106B0931206EB
:107F90008093130690931406A0931506B0931606CB
:107FA0008DEC9CECACECBEE3809317069093180626
:107FB000A0931906B0931A0680E090E0A0E2B1E425
:107FC00080931B0690931C06A0931D06B0931E067B
:107FD0000E94A71A80E090E0A0EBBFEB80935305CE
:107FE00090935405A0935505B09356058CEE91E5FA
:107FF000A6EEB1E48093950490939604A093970421
:10800000B093980480EF98E3A0EABEE380939904CC
:1080100090939A04A0939B04B0939C0488EB92E9FC
:10802000A5E2B4E480939D0490939E04A0939F04E2
:10803000B093A00480E090E0A3E9B3E48093A304AC
:108040009093A404A093A504B093A60483EC94E6B3
:10805000AAE2B1E48093A7049093A804A093A90492
:10806000B093AA0480EB98EBA1E1B5E48093AB0454
:108070009093AC04A093AD04B093AE0481E00E9451
:10808000C32D0E943F2F1092B1051092B20510929D
:10809000B3051092B4058CE0E1EBF2E0DE0111963D
:1080A00001900D928A95E1F713E01150C0F084E041
:1080B000189F90011124E1E0F0E0EC0FFD1FE20FAA
:1080C000F31F6081718182819381F901EB5BFA4F2B
:1080D0006083718382839383812FFFD8E6CFB5DAE3
:1080E0000E94121689EC92E12C960FB6F894DEBF2E
:1080F0000FBECDBFDF91CF911F910C940416CF938B
:10810000C82F811102C00E94121682EB92E10E94D8
:1081100004168DE990E10E9404168AE00E949418EA
:108120008AE00E949418C11106C00E94121681EACA
:1081300092E10E9404166FEF81E08C270E94489123
:10814000C11108C00E94121683E892E10E94041631
:108150000E94121640916306509164066091650674
:10816000709166068AE792E10E944F164091670679
:10817000509168066091690670916A0687E792E1FE
:108180000E944F1640916B0650916C0660916D06EF
:1081900070916E0684E792E10E944F1640916F063F
:1081A00050917006609171067091720681E792E1BC
:1081B0000E944F168AE00E949418C11108C00E94C4
:1081C00012168FE492E10E9404160E94121660912A
:1081D0003F067091400680914106909142060E94B0
:1081E000B0AAAB01BC0186E492E10E944F166091F7
:1081F00043067091440680914506909146060E9480
:10820000B0AAAB01BC0183E492E10E944F166091D9
:108210004706709148068091490690914A060E944F
:10822000B0AAAB01BC0180E492E10E944F166091BC
:108230004B0670914C0680914D0690914E060E941F
:10824000B0AAAB01BC018DE392E10E944F168AE017
:108250000E949418C11108C00E94121683EF91E188
:108260000E9404160E9412164091730650917406E3
:1082700060917506709176068AEE91E10E944F1624
:1082800040917706509178066091790670917A0650
:1082900087EE91E10E944F1640917B0650917C063B
:1082A00060917D0670917E0684EE91E10E944F16EA
:1082B0008AE00E949418C11113C00E9412168CE922
:1082C00091E10E94041681E791E10E94041682E682
:1082D00091E10E9404168AE00E9494180E941216EE
:1082E00060914F0670915006809151069091520610
:1082F0000E94B0AAAB01BC0189E591E10E944F1632
:1083000040917F06509180066091810670918206AF
:1083100086E591E10E944F164091830650918406B4
:10832000609185067091860683E591E10E944F1663
:1083300040910F065091100660911106709112063F
:1083400080E591E10E944F1640911306509114066A
:1083500060911506709116068DE491E10E944F160A
:1083600040911706509118066091190670911A06EF
:108370008AE491E10E944F1640911B0650911C0621
:1083800060911D0670911E0687E491E10E944F16D0
:108390008AE00E949418C11108C00E94121683E35B
:1083A00091E10E9404160E94121660910E0670E080
:1083B0008AE291E10E9435168AE00E949418C11168
:1083C00008C00E9412168BE191E10E9404160E94DF
:1083D0001216409195045091960460919704709103
:1083E000980482E191E10E944F162CEA35EC47E2B5
:1083F0005EE36091990470919A0480919B0490913E
:108400009C040E9417AAAB01BC018FE091E10E947D
:108410005F162CEA35EC47E25EE360919D047091B3
:108420009E0480919F049091A0040E944EACAB01E9
:10843000BC018CE091E10E945F168AE00E949418D2
:10844000C11102C00E9412164091A3045091A404CD
:108450006091A5047091A60483E091E10E944F16FB
:108460002CEA35EC47E25EE36091A7047091A80422
:108470008091A9049091AA040E9417AAAB01BC01A3
:1084800080E091E10E945F162CEA35EC47E25EE362
:108490006091AB047091AC048091AD049091AE04F6
:1084A0000E944EACAB01BC018DEF90E10E945F16C3
:1084B0008AE00E949418C11110C00E9412168EEE1C
:1084C00090E10E9404168DE990E10E9404168AE969
:1084D00090E10E9404160E9412164091530550919B
:1084E0005405609155057091560585EE90E10E9406
:1084F0004F168AE00E949418C11108C00E941216FB
:1085000084ED90E10E9404160E9412164091B1057C
:108510005091B2056091B3057091B4058BEC90E178
:108520000E944F168AE00E949418C11108C00E9450
:10853000121682EB90E10E9404160E9412164091DE
:10854000450550914605609147057091480589EAB7
:1085500090E10E9479164091490550914A05609139
:108560004B0570914C0586EA90E10E947916409186
:108570004D0550914E0560914F057091500583EA6D
:1085800090E10E9479168AE0CF910C9494182F9272
:108590003F924F925F926F927F928F929F92AF9293
:1085A000BF92CF92DF92EF92FF920F931F93CF93E0
:1085B000DF93CDB7DEB7C45AD1090FB6F894DEBF4A
:1085C0000FBECDBF2DB73EB7CD55DF4F39832883C2
:1085D000C35AD040C756DF4F19821882C959D040BC
:1085E00084E690E0C956DF4F99838883C759D0400D
:1085F0000E94B11601E09E0127563F4F44E050E033
:10860000BE016F567F4FCE0189569F4F0E940A17B9
:108610009E0127563F4F42E050E0BE016B567F4F10
:10862000CE0189569F4F0E940A1743E050E0BE01D9
:108630006F567F4F83E193E00E94E7B1892B39F1B8
:10864000CC56DF4F8881C459D040882359F08FE33E
:10865000CF56DF4F8883C159D040CE56DF4F1882A6
:10866000C259D0400E94121685EA93E10E94041676
:10867000BE016F567F4F8CE993E10E9418168EE879
:1086800093E10E94041681E0809352052CC5C357E4
:10869000DF4F188219821A821B82CD58D040C756EC
:1086A000DF4F19821882C959D04001E09E01275638
:1086B0003F4F41E050E0BE0164567F4FCE018956E6
:1086C0009F4F0E940A178DB79EB7C156DF4F9983FF
:1086D0008883CF59D0406E019DE7C90ED11C80E13F
:1086E000EDEBF2E0D60101900D928A95E1F77E0163
:1086F000EDE6EE0EF11C80E1EDECF2E0D701019029
:108700000D928A95E1F780E1EDEDF2E09E012F5F99
:108710003F4F5901D90101900D928A95E1F7C45656
:10872000DF4F4881CC59D04050E04D5F5F4F440F40
:10873000551F440F551F8DB79EB7841B950B0FB661
:10874000F8949EBF0FBE8DBFEDB7FEB731961F01E7
:108750000091510511E0012728563F4FBF01CE017E
:1087600089569F4F0E940A170091510501279E01CB
:1087700027563F4F44E050E06FE476E0CE01895643
:108780009F4F0E940A17C456DF4F8880CC59D040B3
:10879000912CF3E08F0E911C880C991C880C991C6D
:1087A0002DB73EB7281939090FB6F8943EBF0FBE52
:1087B0002DBF8DB79EB701962C01EDB7FEB7E81916
:1087C000F9090FB6F894FEBF0FBEEDBF2DB73EB747
:1087D0002F5F3F4F39010091510501279E01275618
:1087E0003F4FA401BC01CE0189569F4F0E940A173A
:1087F0000091510501279E0127563F4FA401B30167
:10880000CE0189569F4F0E940A1730915105C256DA
:10881000DF4F3883CE59D040332309F4CBC011E069
:10882000C256DF4F0881CE59D04001279E012756FE
:108830003F4F44E050E063E776E0CE0189569F4F1A
:108840000E940A170091510501279E0127563F4FAC
:1088500044E050E067E776E0CE0189569F4F0E94E2
:108860000A170091510501279E0127563F4F44E00A
:1088700050E06BE776E0CE0189569F4F0E940A17C1
:108880000091510501279E0127563F4F44E050E0DB
:108890006FE776E0CE0189569F4F0E940A1700913C
:1088A000510501279E0127563F4F44E050E063E801
:1088B00076E0CE0189569F4F0E940A17009151051C
:1088C00001279E0127563F4F40E150E06FE076E0E0
:1088D000CE0189569F4F0E940A170091510501272A
:1088E0009E0127563F4F44E050E0BE0163577F4F43
:1088F000CE0189569F4F0E940A17C156DF4F8881CB
:108900009981CF59D0400FB6F8949EBF0FBE8DBF4E
:108910000091510501279E0127563F4F4CE050E042
:10892000BE016F5F7F4FCE0189569F4F0E940A178D
:108930000091510501279E0127563F4F44E050E02A
:10894000BE0163577F4FCE0189569F4F0E940A1781
:108950000091510501279E0127563F4F44E050E00A
:10896000BE0163577F4FCE0189569F4F0E940A1761
:1089700001E09E0127563F4F41E050E0B701CE0194
:1089800089569F4F0E940A179E0127563F4F41E08C
:1089900050E0BE016F5F7F4FCE0189569F4F0E940E
:1089A0000A17F701A0808981A89E50011124812C0B
:1089B000912C9DC0C456DF4F8881CC59D04090E0A7
:1089C0009C012E5F3F4FCF55DF4F39832883C15A1B
:1089D000D040AFE3B6E040E050E080E090E04601F8
:1089E000B70131E0C356DF4F3883CD59D040CF5562
:1089F000DF4FE881F981C15AD040E817F90764F4E4
:108A0000C356DF4F1882CD59D0409C018430910568
:108A100058F023E030E008C0F101E40FF51F0081B9
:108A20001181228133810BC0220F331F220F331F8C
:108A3000F401E20FF31F00811181228133810D9334
:108A40001D932D933D93C356DF4FF881CD59D040F0
:108A5000FF2341F0F201E40FF51F00811181228113
:108A6000338111C09C018430910510F023E030E087
:108A7000220F331F220F331FFB01E20FF31F008170
:108A800011812281338150960D931D932D933C9338
:108A90005397C356DF4F2881CD59D040222341F050
:108AA000F301E40FF51F008111812281338111C090
:108AB0009C018430910510F023E030E0220F331F39
:108AC000220F331FF501E20FF31F00811181228174
:108AD000338190960D931D932D933C93939701961C
:108AE0004C5F5F4F8430910509F07BCF98CE0091A9
:108AF00051058A149B0491F001279E0127563F4F90
:108B000044E050E0BE0163577F4FCE0189569F4F2E
:108B10000E940A173FEF831A930AE9CF11E0012759
:108B20009E0127563F4F44E050E063E575E0CE01DB
:108B300089569F4F0E940A170091510501279E01F7
:108B400027563F4F44E250E06AEE75E0CE01895669
:108B50009F4F0E940A1701E09E0127563F4F41E0B8
:108B600050E0BE0165567F4FCE0189569F4F0E944F
:108B70000A179E0127563F4F41E050E0B601CE0153
:108B800089569F4F0E940A170091510501279E01A7
:108B900027563F4F44E050E0B701CE0189569F4F22
:108BA0000E940A170091510501279E0127563F4F49
:108BB00044E050E0BE016F5F7F4FCE0189569F4F6A
:108BC0000E940A17C556DF4FA880CB59D040F60146
:108BD0008081A89E50011124812C912C0091510577
:108BE0008A149B0491F001279E0127563F4F44E0D1
:108BF00050E0BE0163577F4FCE0189569F4F0E94C0
:108C00000A17FFEF8F1A9F0AE9CF11E001279E0193
:108C100027563F4F41E050E0B701CE0189569F4FA4
:108C20000E940A170091510501279E0127563F4FC8
:108C300041E050E0BE016F5F7F4FCE0189569F4FEC
:108C40000E940A170091510501279E0127563F4FA8
:108C500040E150E0BE016F5F7F4FCE0189569F4FCC
:108C60000E940A170091510501279E0127563F4F88
:108C700044E050E0B701CE0189569F4F0E940A1789
:108C80000091510501279E0127563F4F44E050E0D7
:108C9000BE016F5F7F4FCE0189569F4F0E940A171A
:108CA0000091510501279E0127563F4F42E050E0B9
:108CB000B601CE0189569F4F0E940A1700915105B7
:108CC00001279E0127563F4F40E150E0BE016F5FF4
:108CD0007F4FCE0189569F4F0E940A170091510580
:108CE00001112EC089809A80AB80BC8020E030E8E2
:108CF0004BE355E4C501B4010E9410AA882301F199
:108D00008092950490929604A0929704B092980451
:108D10008D819E81AF81B8858093990490939A0448
:108D2000A0939B04B0939C0489859A85AB85BC85F0
:108D300080939D0490939E04A0939F04B093A004FD
:108D400011E001279E0127563F4F42E050E0BE014F
:108D50006F5F7F4FCE0189569F4F0E940A17009187
:108D6000510501279E0127563F4F4CE050E0BE01C0
:108D70006F5F7F4FCE0189569F4F0E940A17009167
:108D80005105011115C020E030E84BE355E469813D
:108D90007A818B819C810E9410AA882349F08CE003
:108DA000FE013196A3EAB4E001900D928A95E1F7B5
:108DB00011E001279E0127563F4F42E050E0BE01DF
:108DC0006F5F7F4FCE0189569F4F0E940A17009117
:108DD000510501279E0127563F4F41E050E0BE015B
:108DE0006F5F7F4FCE0189569F4F0E940A170091F7
:108DF000510501279E0127563F4F40E250E0BE013A
:108E00006F5F7F4FCE0189569F4F0E940A170091D6
:108E1000510501279E0127563F4F41E050E0B70121
:108E2000CE0189569F4F0E940A17009151050127D4
:108E30009E0127563F4F45E050E0BE016F5F7F4FD8
:108E4000CE0189569F4F0E940A17809151058111CA
:108E500002C00E943F2F0091510511E001279E01A1
:108E600027563F4F4AE150E0BE016F5F7F4FCE0172
:108E700089569F4F0E940A170091510501279E01B4
:108E800027563F4F44E350E0BE016F5F7F4FCE0156
:108E900089569F4F0E940A170091510501279E0194
:108EA00027563F4F46E050E0BE016F5F7F4FCE0137
:108EB00089569F4F0E940A170091510501279E0174
:108EC00027563F4F4DE050E0BE016F5F7F4FCE0110
:108ED00089569F4F0E940A170091510501279E0154
:108EE00027563F4F44E050E0BE016F5F7F4FCE01F9
:108EF00089569F4F0E940A170091510501110CC01D
:108F000089819A81AB81BC818093B1059093B20530
:108F1000A093B305B093B40581E008279E012756BE
:108F20003F4F4CE050E0BE016F5F7F4FCE0189564E
:108F30009F4F0E940A1700915105011109C08CE052
:108F4000FE013196A5E4B5E001900D928A95E1F716
:108F500011E001279E0127563F4F4CE650E0BE012D
:108F60006F5F7F4FCE0189569F4F0E940A1719826B
:108F70001A821B821C821D821E821F8218861986FD
:108F80001A861B861C860091510501279E012756D3
:108F90003F4F4CE050E0BE016F5F7F4FCE018956DE
:108FA0009F4F0E940A170091510501279E012756E5
:108FB0003F4F48E050E0BE016F5F7F4FCE018956C2
:108FC0009F4F0E940A17C956DF4F88819981C75960
:108FD000D040845691090E94A23B80935205882379
:108FE000C1F00E941216C956DF4F68817981C759B6
:108FF000D0406456710986E893E10E94351667E413
:1090000072E08EE793E10E946F168AE00E94941846
:1090100060C0C756DF4F28813981C959D040CB562F
:10902000DF4F88819981C559D0402817390729F128
:10903000109352050E9415168EE593E10E940416C6
:109040006AE070E0CB56DF4F88819981C559D040E6
:109050000E949C1989E593E10E9404166AE070E081
:10906000C756DF4F88819981C959D0400E949C1909
:1090700089E493E10E9404162CC08091510581116E
:1090800028C00E94121603E113E0F80181918F01BC
:10909000882319F00E949418F8CFC956DF4F6881D1
:1090A0007981C759D040645671098CE293E10E94DE
:1090B0003516C756DF4F48815981C959D04060E005
:1090C00070E08FE193E10E9479168CE193E10E94B8
:1090D000041680915105811106C0809152058111BD
:1090E00002C00E94253B80915105811101C007D823
:1090F0000E94B3169091520581E08927CD55DF4F2C
:1091000028813981C35AD0400FB6F8943EBF0FBEB4
:109110002DBFCC55DF4F0FB6F894DEBF0FBECDBFCD
:10912000DF91CF911F910F91FF90EF90DF90CF9043
:10913000BF90AF909F908F907F906F905F904F9077
:109140003F902F90089581E08093510520DA10928E
:1091500051050895F8DF81111ACA0E943C3F81E051
:109160000895BF92CF92DF92EF92FF920F931F93D9
:10917000CF93DF93CDB7DEB728970FB6F894DEBF55
:109180000FBECDBF9091CC04981709F47AC0B82EC9
:10919000882309F453C080E090E0A0EAB0E48D8316
:1091A0009E83AF83B887C0905305D0905405E0905C
:1091B0005505F090560520E030E0A901C701B60141
:1091C0000E9410AA87FF0CC0A701960160E070E022
:1091D00080EA90E40E9436A96D837E838F8398870E
:1091E00020E030E04FE153E46D817E818F819885EE
:1091F0000E9413AC181644F480E090E0AFE1B3E4B1
:109200008D839E83AF83B88720918105309182053D
:1092100040918305509184056D817E818F81988571
:109220000E9413AC181654F419821A821B821C82F5
:10923000BE016F5F7F4FCE010596C1D46091790565
:1092400070917A0580917B0590917C0520917D0538
:1092500030917E0540917F055091800519821A82D8
:109260001B821C82E0908105F090820500918305AD
:1092700010918405FE0131966F01C5D38B2D0E949C
:10928000D92D80E028960FB6F894DEBF0FBECDBF73
:10929000DF91CF911F910F91FF90EF90DF90CF90D2
:1092A000BF9008952F923F924F925F926F927F925C
:1092B0008F929F92AF92BF92CF92DF92EF92FF92E6
:1092C0000F931F93CF93DF93CDB7DEB7A0970FB661
:1092D000F894DEBF0FBECDBF1C017F8F6E8F498F0C
:1092E00028A3DC018D909D90AD90BC90FB01408047
:1092F00051806280738022ED30E040EE50ECC3017B
:10930000B201002309F43BC00E9413AC87FD35C2B3
:1093100027E030E04EE353E4C301B2010E9410AAFB
:1093200018160CF42AC223EA31E040E450ECC501DF
:10933000B4010E9413AC87FD20C227E030E042E276
:1093400053E4C501B4010E9410AA18160CF415C20A
:1093500027E030E041E253E4C501B4010E9410AAC5
:1093600018160CF40AC227E030E041E253E4C301CE
:10937000B2010E9410AA18160CF4FFC124C00E946A
:1093800013AC87FDFAC127E030E04EE353E4C3019C
:10939000B2010E9410AA18160CF4EFC123EA31E0C2
:1093A00040E450ECC501B4010E9413AC87FDE5C157
:1093B00027E030E042E253E4C501B4010E9410AA64
:1093C00018160CF4DAC1E0908105F0908205009146
:1093D0008305109184058091480290914902A091E3
:1093E0004A02B0914B028A8F9B8FAC8FBD8F8091C8
:1093F000420290914302A0914402B09145028093B1
:10940000480290934902A0934A02B0934B021982FA
:109410001A821B821C82DE0111966D01A30192014A
:10942000C501B401F0D281E09CDE81113EC1809182
:109430008A0582FF11C02091530530915405409157
:1094400055055091560560E070E080E890EC0E9470
:1094500036A96B017C0106C0C12CD12C40E2E42E60
:1094600041ECF42ECD8ADE8AEF8AF88E812C912C85
:10947000A12C31E4B32E898A9A8AAB8ABC8ABE01B8
:109480006F5E7F4FCE0145969AD31091D004109213
:10949000D00482E0FCD1D1D112FD05C060E070E0C3
:1094A00080EC9FE7BDC040908105509082056090A0
:1094B00083057090840589829A82AB82BC8220E009
:1094C00030E040EA50E4C301B2010E9437A96D8345
:1094D0007E838F8398878E010B5F1F4FBE016F5F66
:1094E0007F4FC8016CD3CD86DE86EF86F88A80E098
:1094F00090E0A0E8BFE389879A87AB87BC87BE016D
:10950000675F7F4FCE010D965AD3F090D004109232
:10951000D00482E0BCD191D1F2FEC0CF8091260C64
:109520008F3F09F45BC0C0908105D0908205E09028
:109530008305F09084058090810590908205A0902D
:109540008305B090840520E030E040E05FE3C70190
:10955000B6010E9437A99B01AC01C501B4010E946C
:1095600010AA87FF1CC01C991AC080E090E0A0E8F8
:10957000BFE389839A83AB83BC832AE037ED43EA58
:109580005BE3C501B4010E9437A96D837E838F839D
:109590009887BE016F5F7F4FC80111D3CCCFA70161
:1095A0009601C501B4010E9436A99B01AC016091EE
:1095B0002F0C7091300C8091310C9091320C0E94E4
:1095C00037A960932F0C7093300C8093310C9093DB
:1095D000320C8091260C8F5F8093260C20E030E0C7
:1095E00040E450E46091810570918205809183058B
:1095F000909184050E944EAC6B017C01A301920105
:10960000C301B2010E9437A99B01AC01C701B60199
:109610000E9437A92DEC3CEC4CE45EE30E944EAC7A
:1096200020915305309154054091550550915605B0
:109630000E9437A97B018C01898D8250823048F5C8
:1096400080E090E0A0E0B1E489839A83AB83BC839F
:1096500060918105709182058091830590918405C8
:10966000A98DA33029F020E030E040EA50E404C0A6
:1096700020E030E048EC51E40E9437A96D837E83FE
:109680008F839887BE016F5F7F4FCE01059697D27B
:1096900007C0B98DB13021F480E063DD811105C0D0
:1096A000E8A1E33008F449C008C098A1933008F459
:1096B0006DC0E12CF12C00EC1FE727E1C22E23E066
:1096C000D22ED6018D916D01882319F00E94941835
:1096D000F8CFF101608171818281938143E050E094
:1096E0000E94121A9FE1C92E93E0D92ED6018D91C6
:1096F0006D01882319F00E949418F8CFEE8DFF8D2C
:10970000608171818281938143E050E00E94121A4E
:1097100084E2C82E83E0D82ED6018D916D01882376
:1097200019F00E949418F8CF43E050E0B701C80147
:109730000E94121A8AE00E9494188A8D9B8DAC8D2B
:10974000BD8D8093480290934902A0934A02B09342
:109750004B029701A801B701C8010E94FCAC882305
:1097600089F080E0FEDC0E94151688EF93E10E94EC
:1097700004162E2D7F2DC8011AC020E070E080EC69
:109780009FE715C02E2D7F2DC80111C08A8D9B8D9E
:10979000AC8DBD8D8093480290934902A0934A02FC
:1097A000B0934B02E12CF12C00EC1FE7DACFC22E74
:1097B000D72E7C01C701B601A0960FB6F894DEBF84
:1097C0000FBECDBFDF91CF911F910F91FF90EF9012
:1097D000DF90CF90BF90AF909F908F907F906F90D1
:1097E0005F904F903F902F900895CF93DF93C9E7FC
:1097F000D5E0488159816A817B8187E894E10E94A4
:109800004F164C815D816E817F8183E894E10E94D7
:109810004F16488559856A857B858FE794E10E94BC
:109820004F164C855D856E857F858BE794E10E94A0
:109830004F16DF91CF910C94093925E835E041E8C6
:1098400055E06DE775E089E795E00C94156885E8CB
:1098500095E00C946268CF93DF9380E00E943358C8
:10986000CDE5D5E0688379838A839B8381E00E947C
:1098700033586C837D838E839F8382E00E943358AC
:10988000688779878A879B87DF91CF9108951F9397
:10989000CF93DF93CDB7DEB760970FB6F894DEBFF6
:1098A0000FBECDBF182FD7DF80915D0590915E056B
:1098B000A0915F05B091600589839A83AB83BC83D7
:1098C0008091610590916205A0916305B091640556
:1098D0008D839E83AF83B8878091650590916605DF
:1098E000A0916705B091680589879A87AB87BC8787
:1098F0008091850590918605A0918705B091880596
:109900008D879E87AF87B88BCE0101960E947857CE
:109910001E3F51F480E1FE013196A9E7B5E00190C8
:109920000D928A95E1F716C024E0129FC001112420
:10993000FC01E758FA4FA1E0B0E0AC0FBD1FA80F43
:10994000B91F8D919D910D90BC91A02D8083918325
:10995000A283B38360960FB6F894DEBF0FBECDBF6F
:10996000DF91CF911F910895AF92BF92CF92DF9276
:10997000EF920F931F93A12CB12C6501E12C08E409
:1099800012E025E835E041E855E06DE775E089E74C
:1099900095E00E94D9661F910F91EF90DF90CF90D4
:1099A000BF90AF900895AF92BF92CF92DF92EF92A7
:1099B0000F931F93CF93DF9300D01F92CDB7DEB7E5
:1099C00069837A838B839C83A12CB12C6501E12C64
:1099D0008E010F5F1F4F25E735E041E755E06DE64B
:1099E00075E089E695E00E94D9660F900F900F9080
:1099F0000F90DF91CF911F910F91EF90DF90CF905B
:109A0000BF90AF9008954F925F926F927F928F9226
:109A10009F92AF92BF92CF92DF92EF92FF920F93FD
:109A20001F93CF93DF93CDB7DEB72C970FB6F89483
:109A3000DEBF0FBECDBF6D837E838F83988729875E
:109A40003A874B875C87470158013601809148026D
:109A500090914902A0914A02B0914B0289839A8366
:109A6000AB83BC83D601CD90DD90ED90FC9020E0DF
:109A700030E0A901C701B6010E9410AA811106C0F9
:109A8000E2E9F4E1C590D590E590F490A501940148
:109A90006091810570918205809183059091840584
:109AA0000E9410AA87FF11C0C0924802D0924902BA
:109AB000E0924A02F0924B028092810590928205D8
:109AC000A0928305B09284054FDFF301408051805E
:109AD0006280738020E030E0A901C301B2010E94DE
:109AE00010AA811108C04090420250904302609039
:109AF000440270904502409248025092490260929E
:109B00004A0270924B028D819E81AF81B88580930D
:109B1000790590937A05A0937B05B0937C058985A0
:109B20009A85AB85BC8580937D0590937E05A09337
:109B30007F05B093800518DFA50194016091810530
:109B40007091820580918305909184050E9413ACE9
:109B500018168CF4C0924802D0924902E0924A0250
:109B6000F0924B028092810590928205A09283052B
:109B7000B0928405F9DE89819A81AB81BC818093A2
:109B8000480290934902A0934A02B0934B022C964C
:109B90000FB6F894DEBF0FBECDBFDF91CF911F91FE
:109BA0000F91FF90EF90DF90CF90BF90AF909F907C
:109BB0008F907F906F905F904F900C944758CF920A
:109BC000DF92EF92FF920F931F936B01FC01E080F5
:109BD000F18002811381E9E7F5E024813581468136
:109BE000578160817181828193810DDF1F910F9177
:109BF000FF90EF90DF90CF900895CF92DF92EF9299
:109C0000FF920F931F936A01E0908105F090820507
:109C10000091830510918405FB01208131814281EF
:109C20005381FC016081718182819381ECDE1F91FF
:109C30000F91FF90EF90DF90CF9008958823F9F077
:109C40008091480290914902A0914A02B0914B0242
:109C50008093590590935A05A0935B05B0935C05DA
:109C60008091460290914702909358058093570542
:109C700084E690E090934702809346020895809195
:109C8000590590915A05A0915B05B0915C058093B0
:109C9000480290934902A0934A02B0934B028091EC
:109CA0005705909158059093470280934602089576
:109CB0008091480290914902A0914A02B0914B02D2
:109CC0008093590590935A05A0935B05B0935C056A
:109CD00080914602909147029093580580935705D2
:109CE00084E690E09093470280934602089580E0D6
:109CF000A5CFCF92DF92EF92FF92CF93DF93209187
:109D00004102222309F443C0EC01C0902902D09003
:109D10002A02E0902B02F0902C02A70196016881A4
:109D200079818A819B810E9413AC181624F4C88221
:109D3000D982EA82FB82C0902D02D0902E02E09060
:109D40002F02F0903002A70196016C817D818E81F7
:109D50009F810E9413AC181624F4CC82DD82EE821F
:109D6000FF82C0903102D0903202E0903302F09036
:109D70003402A7019601688579858A859B850E94B2
:109D800013AC181624F4C886D986EA86FB86DF91C0
:109D9000CF91FF90EF90DF90CF90089524E0829FC5
:109DA000C0011124FC01E753FB4E4591559165918B
:109DB0007491FC01EB5CFD4F40835183628373839C
:109DC000FC01E354FB4E4591559165917491FC0162
:109DD000E75DFD4F408351836283738308958F92C3
:109DE0009F92AF92BF92CF92DF92EF92FF9289E65D
:109DF00095E07FDF8091850383FD7DC0C090750570
:109E0000D0907605E0907705F09078052091850553
:109E1000309186054091870550918805C701B601AC
:109E20000E9410AA882309F466C06091C50470914D
:109E3000C6048091C7049091C80420918E0421111A
:109E400017C00E947FAA2091190230911A0262174E
:109E5000730774F4C0928505D0928605E092870559
:109E6000F09288050E94121680E694E10E94041682
:109E70008090750590907605A0907705B090780554
:109E80002091850530918605409187055091880580
:109E9000C501B4010E9436A96B017C0120E030E0CD
:109EA000A9010E9413AC87FF04C0C701B6019058F6
:109EB00002C0C701B60120914C0230914D02409181
:109EC0004E0250914F020E944EAC20E030E048E438
:109ED00053E40E9413AC181674F480928505909296
:109EE0008605A0928705B09288050E94121681E42B
:109EF00094E10E9404166091460270914702072E79
:109F0000000C880B990B0E94B2AA20914802309154
:109F1000490240914A0250914B020E944EAC2AE005
:109F200037ED43E25CE30E944EAC3DDD80E1E9E6C3
:109F3000F5E0A9E7B5E001900D928A95E1F7FF9071
:109F4000EF90DF90CF90BF90AF909F908F9008954B
:109F50001F93CF93DF93882329F0D0918B05D09561
:109F6000D17001C0D0E0662339F010918B051695B1
:109F7000117081E0182701C010E0442341F0C09126
:109F80008B05C2FBCC27C0F981E0C82701C0C0E027
:109F9000D11104C0111102C0CC23E9F00E941216A5
:109FA0008BE394E10E940416DD2321F089E394E120
:109FB0000E940416112321F087E394E10E94041605
:109FC000CC2321F085E394E10E9404168DE294E114
:109FD0000E940416C1E08C2FDF91CF911F9108954C
:109FE000CF92DF92EF92FF92CF93DF93C82FD0E012
:109FF000FE01E65DFB4E8491811107C00E9412169E
:10A0000088E094E10E9404168AE0FE01EE0FFF1F33
:10A01000EE0FFF1FE657FB4EC590D590E590F490EC
:10A02000682F70E080E090E00E94B2AA9B01AC0132
:10A03000C701B6010E9417AADF91CF91FF90EF9060
:10A04000DF90CF9008954F925F926F927F928F92A0
:10A050009F92AF92BF92CF92DF92EF92FF920F93B7
:10A060001F93CF93DF93CDB7DEB768970FB6F89401
:10A07000DEBF0FBECDBF2A013B016901E82EF12CE6
:10A08000F701EA56FB4EE491AA24A3941E160CF4A1
:10A09000A12CBB24B39420E030E0A901C301B2019C
:10A0A0000E9413AC18160CF0B12C80E0DCD7698349
:10A0B0007A838B839C8381E0D6D76D837E838F8365
:10A0C000988782E0D0D769877A878B879C8783E0DF
:10A0D000CAD76D877E878F87988BEE0CFF1CEE0C9E
:10A0E000FF1C88248394912C8C0E9D1E8E0C9F1C2B
:10A0F000F40110821182128213829E01235F3F4F6E
:10A10000AE01475F5F4FBE016B5F7F4FCE0101968F
:10A110000E943A67F4014082518262827382198AF6
:10A120001A8A1B8A1C8A20E030E0A901B801C60106
:10A130000E9410AA811108C0F701E657FB4E8591D5
:10A140009591A591B49102C0C801D6018D8B9E8BCB
:10A15000AF8BB88FCE0141966C01E12C8E010B5E66
:10A160001F4F9E01235F3F4FAE01475F5F4FBE0110
:10A170006B5F7F4F40970E94F66589D7AB100E94B6
:10A180009D2D68960FB6F894DEBF0FBECDBFDF9150
:10A19000CF911F910F91FF90EF90DF90CF90BF90E4
:10A1A000AF909F908F907F906F905F904F900895A9
:10A1B00021E030E0082E01C0220F0A94EAF79091C6
:10A1C0008A05922B90938A0590918B05292B2093D9
:10A1D0008B0524E0829FC0011124FC01EF54FB4E4B
:10A1E0004591559165917491FC01E758FA4F408370
:10A1F00051836283738308954F925F926F927F922F
:10A200008F929F92AF92BF92FF920F931F93CF9323
:10A21000DF93833008F06AC0F82EC82FD0E0FE012B
:10A22000EA56FB4E8491CC0FDD1FCC0FDD1FFE01E3
:10A23000EB55FB4E4590559065907490682F880FB4
:10A24000770B880B990B0E94B2AA4B015C0120E0AE
:10A2500030E040EC5FE3C301B2010E944EACA501C7
:10A2600094010E944EACAB01BC0100E010E09801EB
:10A270008F2DE9DEFE01E756FB4E25913591459184
:10A280005491C501B4010E944EAC4B015C0120E029
:10A2900030E0A9010E9410AA8823C1F0B501A401F1
:10A2A000705800E010E098018F2DCDDE8F2D98DEE4
:10A2B0002B013C01A5019401C501B4010E9437A9FD
:10A2C000AB01BC01930182018F2DBDDE8F2D70DFAC
:10A2D000B4DAFE01E759FA4FC758DA4F88819981FD
:10A2E000AA81BB8180839183A283B383DF91CF91C5
:10A2F0001F910F91FF90BF90AF909F908F907F9094
:10A300006F905F904F90089580E1EEECF5E0DF01F3
:10A31000982F1D929A95E9F7E1EAF5E0DF01982F71
:10A320001D929A95E9F7EAEBF5E0DF011D928A9517
:10A33000E9F71092B6051092B7051092B805109281
:10A34000B9058AEE95E00E94CBA210928A0610927F
:10A350008D0610928B0610928C0610928706089537
:10A360004F925F926F927F928F929F92AF92BF9225
:10A37000CF92DF92EF92FF920F931F93CF93DF93D1
:10A38000CDB7DEB768970FB6F894DEBF0FBECDBF6E
:10A390008C015B014A01FC01EF5BFF4F6081718121
:10A3A000828193810E94B0AA6B017C01D5012D911D
:10A3B0003D914D915C910E944EAC0E94FDA90E947E
:10A3C00084AA69877A878B879C87F40120813181F1
:10A3D00042815381C701B6010E944EAC0E94FDA983
:10A3E0000E9484AA6D877E878F87988B29853A85FE
:10A3F0004B855C85283731054105510540F488E7D8
:10A4000090E0A0E0B0E089879A87AB87BC872D8574
:10A410003E854F855889283731054105510540F45F
:10A4200088E790E0A0E0B0E08D879E87AF87B88B8B
:10A430009801235B3F4FD9018D919D910D90BC9167
:10A44000A02D89839A83AB83BC83BC01CD010E947C
:10A45000B2AA2B013C0169857A858B859C850E9477
:10A46000B0AA698B7A8B8B8B9C8B20E030E0A901A2
:10A47000C301B2010E9410AA882329F1A701960105
:10A48000C701B6010E944EAC4B015C0129893A8993
:10A490004B895C89CA01B9010E944EAC9B01AC0199
:10A4A000C501B4010E9436A94B015C01A3019201D0
:10A4B000C301B2010E9437A99B01AC01C501B401DF
:10A4C0000E9417AA03C060E070E0CB010E94FDA9C2
:10A4D0000E9484AA6D837E838F83988769817A81A5
:10A4E0008B819C8190958095709561957F4F8F4F62
:10A4F0009F4F0E94B2AA4B015C016D857E858F85BE
:10A5000098890E94B0AA69837A838B839C8320E018
:10A5100030E0A901C501B4010E9410AA882349F1C5
:10A5200029813A814B815C81CA01B9010E944EACFC
:10A530006D8B7E8B8F8B988FA7019601C701B6011B
:10A540000E944EAC9B01AC016D897E898F89988DEC
:10A550000E9436A96B017C01A5019401C501B401DB
:10A560000E9437A99B01AC01C701B6010E9417AA3E
:10A5700003C060E070E0CB010E94EDAAF80185A065
:10A5800096A0A7A0B0A4750164012D813E814F81E2
:10A590005885C21AD30AE40AF50A0E9484AAC61A88
:10A5A000D70AE80AF90AF7FE73C020E030E0A901F3
:10A5B000C301B2010E9410AA882309F443C0A30179
:10A5C0009201C301B2010E9437A96B017C01C50150
:10A5D000B4010E94B0AA9B01AC01C701B6010E9460
:10A5E0004EAC6B017C0129893A894B895C89CA018F
:10A5F000B9010E944EAC9B01AC01C701B6010E949B
:10A6000036A96B017C0129813A814B815C81CA01A9
:10A61000B9010E944EAC9B01AC01C701B6010E947A
:10A6200037A96B017C0120E030E040E850E4C30131
:10A63000B2010E944EAC9B01AC01C701B6010E9461
:10A6400017AA03C060E070E0CB010E94FDA97B0166
:10A650006C0120E030E0A9010E9413AC181624F030
:10A66000E12CF12CC12CD12CB701C6010E9484AA87
:10A670006D837E838F83988786169706A806B90612
:10A6800020F48D829E82AF82B886C12CD12C7601B7
:10A690008D819E81AF81B885F80181A792A7A3A77C
:10A6A000B4A7C80ED91EEA1EFB1EC5A6D6A6E7A6ED
:10A6B000F0AAEB5BFF4F29853A854B855C852083AB
:10A6C00031834283538334968D859E85AF85B889C7
:10A6D00080839183A283B38368960FB6F894DEBF1C
:10A6E0000FBECDBFDF91CF911F910F91FF90EF90E3
:10A6F000DF90CF90BF90AF909F908F907F906F90A2
:10A700005F904F9008952F923F924F925F926F9279
:10A710007F928F929F92AF92BF92CF92DF92EF92F1
:10A72000FF920F931F93CF93DF93009709F471C0AB
:10A730008B01EC01D984CA847B846C848D809E80DB
:10A74000AF80B8842D2D3C2D472D562DC501B40169
:10A750000E9410AA811108C00115110509F459C001
:10A76000F801808180FF55C0888181FD34C00115CA
:10A77000110531F0F801258036804780508408C0EB
:10A780008BE0282E87ED382E83E2482E8BE3582E5F
:10A7900089899A89AB89BC89BC01CD0190589B01FC
:10A7A000AC010E9437A92D853E854F8558890E94AE
:10A7B0004EAC9B01AC01C201B1010E9436A97B01E4
:10A7C0008C019B01AC016D2D7C2D872D962D0E9457
:10A7D00010AA87FF04C0ED2CFC2C072D162D970125
:10A7E000A801C501B4010E9410AA882391F08881B4
:10A7F00081608883CE010E949332882321F0888172
:10A800008E7F888306C0A701B8014D835E836F8366
:10A810007887DF91CF911F910F91FF90EF90DF909C
:10A82000CF90BF90AF909F908F907F906F905F90F0
:10A830004F903F902F900895FF920F931F93CF93C7
:10A84000DF93C0918D06C150CF70D0918B0680915F
:10A850008D06D817E9F060E070E086E5F82ECD1798
:10A86000B9F0FC9E800111240257194FF801808134
:10A8700083FD03C0C80147DFB801C150CF7080918C
:10A880008B06D81761F3CD1719F0DF5FDF70F7CFB4
:10A89000DF91CF911F910F91FF9008954F925F929A
:10A8A0006F927F928F929F92AF92BF92FF920F937F
:10A8B0001F93CF93DF93009709F459C0F42EEB0157
:10A8C0008C01FC01808181FD3CC045805680678001
:10A8D00070848D809E80AF80B884A5019401C301EF
:10A8E000B2010E9410AA87FF2CC0F80181899289C9
:10A8F000A389B489BC01CD0190589B01AC010E9491
:10A9000037A9F80125853685478550890E944EACC8
:10A910009B01AC01C301B2010E9436A92B013C018D
:10A92000A50194010E9410AA87FF0BC08881816055
:10A930008883CE010E949332882391F088818E7F94
:10A94000888329853A854B855C856D817E818F81E1
:10A9500098850E9410AA81110AC0F0928B0607C048
:10A960004D825E826F827886F0928B06EACFDF910D
:10A97000CF911F910F91FF90BF90AF909F908F90BC
:10A980007F906F905F904F900895CF92DF92EF92FB
:10A99000FF920F931F93CF93DF9310918B06C0E02C
:10A9A000D0E086E5C82E80918D06181709F1C19E6A
:10A9B000B0011124CB018257994F7C01FC018081A9
:10A9C00083FD0AC00E2DDF2C209769F0CE010E9476
:10A9D0009332882341F002C00C2FDD2E1F5F1F70C1
:10A9E000C02FDD2DE0CF412FB701CE0157DFF6CFCD
:10A9F000DF91CF911F910F91FF90EF90DF90CF905B
:10AA000008952F923F924F925F926F927F928F9212
:10AA10009F92AF92BF92CF92DF92EF92FF920F93ED
:10AA20001F93CF93DF93CDB7DEB72E970FB6F89471
:10AA3000DEBF0FBECDBF20918A06298730918D06DB
:10AA40003B8796E58B85E9858E1759F08B8581507C
:10AA50008F70989FF0011124E257F94F208123FD58
:10AA60000DC0812C912CA12CB12C1A861C861D8620
:10AA70001E86212C312C00E010E01AC08B87E2CF1B
:10AA8000F6E52985F29FC0011124FC01E257F94F38
:10AA90001F01808183FF11C0FA84EC84DD84CE84A1
:10AAA00089858F5F8F708987FA86EC86DD86CE86F2
:10AAB000F9852B85F213E4CF93C065817681878178
:10AAC00090850E94BBACF62EE72ED82EC92E01151C
:10AAD000110509F47FC0F801808180FD04C0F101F7
:10AAE000808180FF77C0F801808181608083C80108
:10AAF0000E94933281116AC0F80161817281838161
:10AB000094810E94BBAC2B013C019B01AC0160E035
:10AB100070E080E89FE30E9417AA4B015C019B0153
:10AB2000AC016F2D7E2D8D2D9C2D0E944EAC698326
:10AB30007A838B839C83A50194016A857C858D85AE
:10AB40009E850E944EAC6D837E838F839887AE0175
:10AB50004F5F5F4FBE016B5F7F4FC80101DCF801A3
:10AB600086A9882399F12091B1053091B2054091D1
:10AB7000B3055091B405FD96608171818281938106
:10AB80000E944EAC20915F063091600640916106B4
:10AB9000509162060E944EAC4B015C019B01AC01DE
:10ABA000C301B2010E944EAC0E9484AAF80172AFA8
:10ABB00061AFA50194016F2D7E2D8D2D9C2D0E94DE
:10ABC0004EAC0E9484AAF80174AF63AFF801808193
:10ABD0008E7F80838F2C9E2CAD2CBC2C810160CF6E
:10ABE0002114310409F473C0F101808181608083F4
:10ABF000C8010E949332811166C0F10161817281A6
:10AC0000838194810E94BBAC6B017C019B01AC01F0
:10AC100060E070E080E89FE30E9417AA2B013C01EE
:10AC20002DEC3CEC4CE45DE30E944EAC69837A83EE
:10AC30008B839C83A3019201B401C5010E944EAC99
:10AC40006D837E838F839887AE014F5F5F4FBE0118
:10AC50006B5F7F4FC10184DBF10186A9882399F1E5
:10AC60002091B1053091B2054091B3055091B405E2
:10AC7000FD9660817181828193810E944EAC20910A
:10AC80005F063091600640916106509162060E9415
:10AC90004EAC4B015C019B01AC01C701B6010E94A7
:10ACA0004EAC0E9484AAF10172AF61AF2DEC3CEC76
:10ACB0004CE45DE3C501B4010E944EAC0E9484AA3D
:10ACC000F10174AF63AFF10180818E7F80832E9696
:10ACD0000FB6F894DEBF0FBECDBFDF91CF911F91AD
:10ACE0000F91FF90EF90DF90CF90BF90AF909F902B
:10ACF0008F907F906F905F904F903F902F9008952E
:10AD000080918D0690918B0681508F70891711F07C
:10AD100093DD3BDE76CEAF92BF92CF92DF92EF9281
:10AD2000FF920F931F93CF9390918D0680918A0687
:10AD3000981791F0E0918A0686E5E89FF0011124CA
:10AD4000E152F94FC08180918A0690918D06891752
:10AD500029F08F5F8F70F9CFC091C004CC2339F1F7
:10AD60000E94871100919D0510919E0520919F05DD
:10AD70003091A005DC01CB0101151105210531053C
:10AD800071F48C599F4FAF4FBF4F80939D059093A7
:10AD90009E05A0939F05B093A005CFEF1EC0801B1A
:10ADA000910BA20BB30BB7FF18C0CFEF16C01092D8
:10ADB0009D0510929E0510929F051092A00560E0DF
:10ADC00070E088E0CF911F910F91FF90EF90DF909E
:10ADD000CF90BF90AF900C9453126C2F70E080E036
:10ADE00090E01F921F921F922FEF2F9326E4A22E26
:10ADF000B12CC12CD12CE12CF12C8701EA9421E05B
:10AE000030E040E050E00E945D150F900F900F90F1
:10AE10000F90D7CFCF92DF92EF92FF920F931F93B5
:10AE2000CF93DF93CDB7DEB728970FB6F894DEBF88
:10AE30000FBECDBF20910E06222309F44AC06A013D
:10AE40008B017C0120E030E040E450E4FC016081B3
:10AE50007181828193810E9437A96D837E838F8364
:10AE6000988720E030E04EE353E4F801608171817F
:10AE7000828193810E9436A969837A838B839C8324
:10AE80009601AE014F5F5F4FBE016B5F7F4F8AEE51
:10AE900095E00E9403A220E030E040E450E46D81A0
:10AEA0007E818F8198850E9436A9F7016083718326
:10AEB0008283938320E030E04EE353E469817A811A
:10AEC0008B819C810E9437A9F80160837183828302
:10AED000938328960FB6F894DEBF0FBECDBFDF91E7
:10AEE000CF911F910F91FF90EF90DF90CF90089539
:10AEF0000F931F93CF93DF93CDB7DEB7AC970FB609
:10AF0000F894DEBF0FBECDBF20910E06222309F4B8
:10AF100050C08C016AEE75E0CE0101960E9486A3B6
:10AF200020E030E040E450E4F801608171818281EA
:10AF300093810E9437A969A77AA78BA79CA720E0D5
:10AF400030E04EE353E4F801648175818681978196
:10AF50000E9436A96DA37EA38FA398A79801285FAE
:10AF60003F4FAE014B5D5F4FBE01675D7F4FCE012E
:10AF700001960E9403A220E030E040E450E469A57D
:10AF80007AA58BA59CA50E9436A9F80160837183E0
:10AF90008283938320E030E04EE353E46DA17EA1F1
:10AFA0008FA198A50E9437A9F801648375838683D1
:10AFB0009783AC960FB6F894DEBF0FBECDBFDF917E
:10AFC000CF911F910F91089580916F0081FB992778
:10AFD00090F981FF05C080916F008D7F80936F0095
:10AFE00080918A0680938D0680938B0680938C06D1
:10AFF00084E68093870628EE33E030938906209319
:10B000008806992329F080916F00826080936F00F9
:10B0100081E08093400508950C94C238CF93C82FE7
:10B020000E94EB380E94B2AA24E0C29FF0011124D2
:10B03000E15EF94F20813181428153810E944EAC03
:10B04000CF91089590918D0680918A06981719F0F6
:10B050000E9497A8F7CF8091880690918906892B46
:10B06000B9F70C946EA7CF93C82F0E94A4380E9402
:10B07000B2AA24E0C29FF0011124E15EF94F2081C1
:10B080003181428153810E944EACCF9108959091BD
:10B090008D0680918A06981719F00E9497A8F7CF1D
:10B0A0008091880690918906892BB9F708952F928F
:10B0B0003F924F925F926F927F928F929F92AF9248
:10B0C000BF92CF92DF92EF92FF920F931F93CF9395
:10B0D000DF93CDB7DEB766970FB6F894DEBF0FBE2D
:10B0E000CDBFB88AAF86E0919C05DC2CDE26672BAD
:10B0F000682B692B19F48D2D8E7FD82E232B242BB2
:10B10000252B19F49D2D9D7FD92EEF28E02AE12AC9
:10B1100019F4AD2DAB7FDA2E8D2D8E2780939C05F3
:10B120008091330C9091340CA091350CB091360C79
:10B130008D839E83AF83B88720E030E0A901BC01F6
:10B14000CD010E9410AA882309F420C180915302E6
:10B1500090915402A0915502B091560289879A8726
:10B16000AB87BC87A7E3BCE0BE87AD87EF85F889D6
:10B17000FA83E98380E995E09E8B8D8BAFE3B6E09F
:10B18000BC83AB83212C312C812C912C5401EC2DD0
:10B19000F0E0FA8BE98B8D2D90E09C8B8B8BAD854D
:10B1A000BE85CD90DD90ED90FD90BE87AD8720E00F
:10B1B00030E0A901C701B6010E9410AA882309F452
:10B1C000CEC009891A89022C02C0159507950A94E8
:10B1D000E2F7017011278B899C89022C02C095959A
:10B1E00087950A94E2F780FF38C0ED89FE89608177
:10B1F0007181828193810E94B2AA2B013C010115C9
:10B20000110529F420E030E040E85FE304C020E0CD
:10B2100030E040E85FEB6D817E818F8198850E94F0
:10B220004EACA70196010E944EACAB81BC815496F6
:10B230002D913D914D915C9157970E944EAC9B0191
:10B24000AC01C301B2010E9437A90E947FAAED8917
:10B25000FE896083718382839383AD89BE89CD909B
:10B26000DD90ED90FC90C114D104E104F10409F4E7
:10B2700076C020E030E0A90169857A858B859C85C0
:10B280000E9410AA882309F441C0D701C60188276B
:10B29000B7FD83959927AA27BB270817190709F037
:10B2A0005EC020E030E0A901C501B4010E9410AAEF
:10B2B00081111CC029853A854B855C85EF85F8890D
:10B2C00065857685878590890E9417AA4B015C0168
:10B2D00020E030E040E85FE30E9413AC181634F43D
:10B2E000812C912C80E8A82E8FE3B82EC701B601DF
:10B2F0000E94B2AAA50194010E944EAC0E947FAAAE
:10B30000611571058105910519F429C0C701B601C0
:10B310008B019C0197FF07C0002711279801061B8E
:10B32000170B280B390BA981BA8155964D905D906A
:10B330006D907C905897040D151D261D371DFD013D
:10B34000058B168B278B308FC61AD70AE80AF90AA5
:10B35000AD89BE89CD92DD92ED92FC921397BFEF3D
:10B360002B1A3B0AE981FA813496FA83E9838D89A5
:10B370009E8904969E8B8D8BAB81BC811496BC8379
:10B38000AB83B3E02B16310409F009CF66960FB6F4
:10B39000F894DEBF0FBECDBFDF91CF911F910F910B
:10B3A000FF90EF90DF90CF90BF90AF909F908F90E5
:10B3B0007F906F905F904F903F902F9008952F92C5
:10B3C0003F924F925F926F927F928F929F92AF9235
:10B3D000BF92CF92DF92EF92FF920F931F93CF9382
:10B3E000DF93CDB7DEB7C756D1090FB6F894DEBFED
:10B3F0000FBECDBF1C01A4966FAFA4976F965FAF31
:10B400004EAF6F9769963FAF2EAF69972896EFAE14
:10B410002897FFAE60960FAF609764961FAF649752
:10B42000CFAAA196BFAEAEAEA197DA014D915D91C4
:10B430006D917C918091CE059091CF05A091D00522
:10B44000B091D1058A019B01081B190B2A0B3B0BFC
:10B450000BA31CA32DA33EA36F96AEADBFAD6F97FC
:10B4600014964D915D916D917C9117978091D205C5
:10B470009091D305A091D405B091D5058A019B0187
:10B48000081B190B2A0B3B0B0FA318A729A73AA7D8
:10B490006F96AEADBFAD6F9718964D915D916D9162
:10B4A0007C911B978091D6059091D705A091D805E6
:10B4B000B091D9058A019B01081B190B2A0B3B0B84
:10B4C0000FA718AB29AB3AAB6F96AEADBFAD6F9778
:10B4D0001C96CD90DD90ED90FC901F978091DA0541
:10B4E0009091DB05A091DC05B091DD0526013701C7
:10B4F000481A590A6A0A7B0A09F497C06091C50480
:10B500007091C6048091C7049091C80420918E0464
:10B5100021112AC00E947FAA2091190230911A029B
:10B52000621773070CF5C092DA05D092DB05E09242
:10B53000DC05F092DD056996EEADFFAD6997848577
:10B540009585A685B7858093AD059093AE05A093AC
:10B55000AF05B093B0050E94121684EF94E10E94EB
:10B560000416412C512C3201C301B2010E94B2AA2F
:10B570001FA904E0109FF0011124E45BFD4F20811E
:10B580003181428153810E944EAC6B017C0120E0ED
:10B5900030E0A9010E9413AC87FF04C0F7FAF094D1
:10B5A000F7F8F09460915F067091600680916106F3
:10B5B000909162060E947FAA9B01AC01A8ECB0E0CA
:10B5C0000E9496AD0E94B2AA9B01AC01C701B601D0
:10B5D0000E9413AC18164CF56F96EEADFFAD6F9749
:10B5E00084859585A685B7858093DA059093DB05DC
:10B5F000A093DC05B093DD056996EEADFFAD6997CC
:10B6000084859585A685B7858093AD059093AE0515
:10B61000A093AF05B093B0050E94121685ED94E19A
:10B620000E940416412C512C32018BA19CA1ADA18A
:10B63000BEA18827B7FD83959927AA27BB27182F76
:10B640002FA138A549A55AA557FD12608FA598A925
:10B65000A9A9BAA9B7FD146077FC1860C301B201AB
:10B660000E94B2AABFA9A4E0BA9FF0011124E45B32
:10B67000FD4F20813181428153810E944EAC4B01AC
:10B680005C0120E030E0A9010E9413AC87FF04C0F8
:10B69000C501B401905802C0C501B40120E030E0FA
:10B6A00040E05FE30E9437A90E9484AA6BAF7CAFA1
:10B6B0008DAF9EAFF101108215AB2BA13CA14DA126
:10B6C0005EA12BA73CA74DA75EA757FF0BC05095C7
:10B6D0004095309521953F4F4F4F5F4F2BA73CA78B
:10B6E0004DA75EA78BA59CA5ADA5BEA5F101858B39
:10B6F000968BA78BB08F2FA138A549A55AA52BAB48
:10B700003CAB4DAB5EAB57FF0BC0509540953095B1
:10B7100021953F4F4F4F5F4F2BAB3CAB4DAB5EABDB
:10B720008BA99CA9ADA9BEA9F101818F928FA38F8E
:10B73000B48F2FA538A949A95AA92F962CAF3DAF90
:10B740004EAF5FAF2F9757FF0DC050954095309586
:10B7500021953F4F4F4F5F4F2F962CAF3DAF4EAFD0
:10B760005FAF2F972F968CAD9DADAEADBFAD2F9730
:10B77000F101858F968FA78FB0A36BA17CA18DA1BE
:10B780009EA10E94B2AA20911F06309120064091EE
:10B790002106509122060E944EAC27966CAF7DAFD9
:10B7A0008EAF9FAF2797698B7A8B8B8B9C8B6FA10A
:10B7B00078A589A59AA50E94B2AA20912306309166
:10B7C000240640912506509126060E944EAC6B013E
:10B7D0007C016D8B7E8B8F8B988F6FA578A989A943
:10B7E0009AA90E94B2AA209127063091280640917A
:10B7F000290650912A060E944EAC6D966CAF7DAF23
:10B800008EAF9FAF6D97698F7A8F8B8F9C8F2091B2
:10B810002B0630912C0640912D0650912E06C50125
:10B82000B4010E944EAC4B015C016D8F7E8F8F8FF7
:10B8300098A32BA53CA54DA55EA526303105410555
:10B84000510544F58BA99CA9ADA9BEA90697A105F0
:10B85000B10504F52F962CAD3DAD4EAD5FAD2F97E4
:10B860002630310541055105ACF420E030E0A90156
:10B87000C501B4010E9413AC87FF04C0B7FAB094AD
:10B88000B7F8B094D1011D968D929D92AD92BC9265
:10B89000509759C0A196EEADFFADA19780809180E1
:10B8A000A280B38020E030E0A901C501B4010E946C
:10B8B00010AA882341F0D1011D968D929D92AD92E0
:10B8C000BC92509731C027962CAD3DAD4EAD5FADCB
:10B8D0002797CA01B9010E944EAC4B015C01A70138
:10B8E0009601C701B6010E944EAC9B01AC01C50197
:10B8F000B4010E9437A94B015C016D962CAD3DADA2
:10B900004EAD5FAD6D97CA01B9010E944EAC9B016F
:10B91000AC01C501B4010E9437A90E94BBACF10182
:10B92000658776878787908B5101C12EEFA4F8A891
:10B9300009A91AA92FA138A549A55AA56BA17CA1CF
:10B940008DA19EA1B4DB0BAD1CAD2DAD3EADD101E3
:10B9500091960D931D932D933C93949755964D91ED
:10B960005D916D917C9158975D960D911D912D91F2
:10B970003C91909759968D919D910D90BC91A02DE1
:10B9800080179107A207B30710F4D901C8018417E3
:10B990009507A607B70710F4DB01CA010BAD1CAD74
:10B9A0002DAD3EAD80179107A207B30710F4D90162
:10B9B000C801F10185A396A3A7A3B0A70697A10587
:10B9C000B105A8F18091C004EF5AFF4F8083452B49
:10B9D000462B472B09F01798F101818D928DA38D8D
:10B9E000B48D892B8A2B8B2B09F01698F101858D4C
:10B9F000968DA78DB0A1892B8A2B8B2B09F01598DA
:10BA00000BAD1CAD2DAD3EAD012B022B032BD1F0A8
:10BA10008091B505882319F081508093B5051FA941
:10BA2000111107C0149880E28093B50502C080E030
:10BA3000FEC7E0907F06F09080060091810610918D
:10BA4000820608C0E0908306F09084060091850687
:10BA5000109186069701A80128966FAD28977FADB3
:10BA600060968FAD609764969FAD64970E9410AA10
:10BA700087FFD2C7D1011D962D913D914D915C91CB
:10BA800050976D962CAF3DAF4EAF5FAF6D9760E0B6
:10BA900070E080E89FE30E9417AA2B966CAF7DAF01
:10BAA0008EAF9FAF2B979B01AC01B701C8010E94DD
:10BAB0004EAC4B015C0180918D0690918C06891BE8
:10BAC0008F7024968FAF2497A501940160E074E2F3
:10BAD00084E799E40E9417AA0E941EAC6B017C01C6
:10BAE00024968FAD249782508630C0F580914F0602
:10BAF00090915006A0915106B0915206C816D906F1
:10BB0000EA06FB0658F58C199D09AE09BF09BC0170
:10BB1000CD01660F771F881F991F2496BFAD24970C
:10BB20000B2F10E020E030E0A90198010E943BAD0E
:10BB3000CA01B9010E94B0AA0E941EAC6C0D7D1D05
:10BB40008E1D9F1D0E94B0AA9B01AC0160E074E2B3
:10BB500084E799E40E9417AA4B015C01A5019401B6
:10BB60006D966CAD7DAD8EAD9FAD6D970E944EAC68
:10BB70009B01AC010E944EAC23966CAF7DAF8EAFA3
:10BB80009FAF2397F101618372838383948305A11F
:10BB900016A127A130A50FA718AB29AB3AABC90155
:10BBA000B8010E94B0AA6FAB78AF89AF9AAFA50178
:10BBB00094010E944EAC0E94FDA90E9484AA639643
:10BBC0006CAF7DAF8EAF9FAF6397F101EF5BFF4F1F
:10BBD00060837183828393838E010F5E1F4F1CA746
:10BBE0000BA7005111092D961FAF0EAF2D9703E63D
:10BBF00016E0A1961FAF0EAFA1978E010F5D1F4FEC
:10BC00001AA309A32D960EAD1FAD2D971CAB0BAB40
:10BC10001BA21FA200E81FE3ABA5BCA56D917D91FF
:10BC20008D919D91BCA7ABA7A50194010E944EAC3C
:10BC30006B017C01EBA9FCA96193719381939193B2
:10BC4000FCABEBAB20E030E0A9010E9413AC87FF16
:10BC500004C0F7FAF094F7F8F094A196AEADBFAD3A
:10BC6000A1972D913D914D915D91A196BFAFAEAF42
:10BC7000A19767962CAF3DAF4EAF5FAF6797C701F7
:10BC8000B6010E9413AC1816C4F4A701960167967A
:10BC90006CAD7DAD8EAD9FAD67970E9417AA6B010D
:10BCA0007C019B01AC016BA17FA1C8010E9413AC78
:10BCB00018161CF4CBA2DFA28701EBA5FCA529A1D5
:10BCC0003AA1E217F30709F0A7CF20E030E040E8FF
:10BCD0005FE36BA17FA1C8010E9410AA87FF4BC040
:10BCE0006E0131E1C30ED11C2D96EEACFFAC2D9749
:10BCF0002BA13FA1A801D7016D917D918D919C91C0
:10BD00000E944EACF70161937193819391937F01EF
:10BD1000EC15FD0569F77101F1E4EF0EF11C639676
:10BD20006CAD7DAD8EAD9FAD63970E94B0AA2BA187
:10BD30003FA1A8010E944EAC0E9484AAD7016D9336
:10BD40007D938D939C9313972BA13FA1A8016BA189
:10BD50007FA1C8010E944EAC9B01AC0123966CAD43
:10BD60007DAD8EAD9FAD23970E944EACF1016183F6
:10BD70007283838394832B962CAD3DAD4EAD5FAD26
:10BD80002B976FA978AD89AD9AAD0E944EAC6BAB85
:10BD90007CAB8DAB9EABD10155960D911D912D9134
:10BDA0003C9158970BA31CA32DA33EA35D960D9128
:10BDB0001D912D913C9190970FA318A729A73AA701
:10BDC00059960D911D912D913C915C970BA71CA745
:10BDD0002DA73EA70BA11CA12DA13EA1012B022B3B
:10BDE000032B41F52BA53CA54DA55EA5232B242BAC
:10BDF000252B01F58FA198A5A9A5BAA5892B8A2B7A
:10BE00008B2BC1F42091770630917806409179060A
:10BE100050917A066BA97CA98DA99EA90E944EAC6F
:10BE20000E94FDA90E9484AA4B015C01D101D69613
:10BE30001C92F0C20BAD1CAD2DAD3EAD012B022B03
:10BE4000032B49F06091730670917406809175061A
:10BE50009091760608C060917B0670917C06809177
:10BE60007D0690917E062BA93CA94DA95EA90E9452
:10BE70004EAC0E94FDA90E9484AA4B015C012BAD2F
:10BE80003CAD4DAD5EAD232B242B252BA9F020E03E
:10BE900030E0A9016091B1057091B2058091B305C0
:10BEA0009091B4050E9410AA882331F081E0141407
:10BEB0001504160417040CF080E0D101D6968C937B
:10BEC000882309F4BAC02091A1053091A2054091C0
:10BED000A3055091A4056996EEADFFAD6997608109
:10BEE0007181828193810E9436A92B013C012091AE
:10BEF000A5053091A6054091A7055091A805699622
:10BF0000AEADBFAD699714966D917D918D919C9169
:10BF100017970E9436A96BAF7CAF8DAF9EAF209173
:10BF2000A9053091AA054091AB055091AC056996E1
:10BF3000EEADFFAD699760857185828593850E941E
:10BF400036A96B017C01A3019201C301B2010E94D9
:10BF50004EAC2B013C012BAD3CAD4DAD5EADCA01ED
:10BF6000B9010E944EAC9B01AC01C301B2010E9419
:10BF700037A92B013C01A7019601C701B6010E9418
:10BF80004EAC9B01AC01C301B2010E9437A90E94D3
:10BF9000BBAC6B017C012091AD053091AE054091A9
:10BFA000AF055091B0056996AEADBFAD69971C96CF
:10BFB0006D917D918D919C911F970E9436A9A7014B
:10BFC00096010E9417AA6B017C01F101FD96608326
:10BFD00071838283938320E030E040E450E40E9448
:10BFE00013AC18161CF4F10116AA27C02091B10554
:10BFF0003091B2054091B3055091B405C701B60127
:10C000000E944EAC9B01AC0160911B0670911C0616
:10C0100080911D0690911E060E9417AA2BA93CA98B
:10C020004DA95EA90E944EAC0E9484AA68157905AC
:10C030008A059B0510F44B015C018091CA05909123
:10C04000CB05A091CC05B091CD05F10141A052A046
:10C0500063A074A00FA518A929A93AA98017910770
:10C06000A207B30708F4CDC02BA13CA14DA15EA14E
:10C07000232B242B252B61F120912F0630913006A4
:10C080004091310650913206281539054A055B0565
:10C09000F8F46FA578A989A99AA90E9418AD6B0137
:10C0A0007C01A50194016BA17CA18DA19EA10E94A0
:10C0B00018ADC616D706E806F90650F4C701B60152
:10C0C0002BA13CA14DA15EA10E943BAD49015A01AB
:10C0D0008BA59CA5ADA5BEA5892B8A2B8B2B61F1C9
:10C0E0002091330630913406409135065091360642
:10C0F000281539054A055B05F8F46FA578A989A9C3
:10C100009AA90E9418AD6B017C01A50194016BA551
:10C110007CA58DA59EA50E9418ADC616D706E8067B
:10C12000F90650F4C701B6012BA53CA54DA55EA5A7
:10C130000E943BAD49015A010FA118A529A53AA5B6
:10C14000012B022B032B61F1209137063091380629
:10C150004091390650913A06281539054A055B0584
:10C16000F8F46FA578A989A99AA90E9418AD6B0166
:10C170007C01A50194016FA178A589A59AA50E94CB
:10C1800018ADC616D706E806F90650F4C701B60181
:10C190002FA138A549A55AA50E943BAD49015A01D6
:10C1A000411451046104710409F434C120913B0627
:10C1B00030913C0640913D0650913E0628153905C8
:10C1C0004A055B0508F026C16FA578A989A99AA937
:10C1D0000E9418AD6B017C01A5019401C301B2015D
:10C1E0000E9418ADC616D706E806F90608F012C177
:10C1F000C701B601A30192010E943BAD49015A015A
:10C2000009C12BA13CA14DA15EA1232B242B252BE1
:10C21000E9F160912F06709130068091310690917E
:10C220003206681579058A059B0580F50E94B0AA3B
:10C230002FA938AD49AD5AAD0E944EAC6B017C01BF
:10C240006BA17CA18DA19EA10E94B0AA6BA37CA32F
:10C250008DA39EA3C501B4010E94B0AA2BA13CA14D
:10C260004DA15EA10E944EACA70196010E9413ACA5
:10C27000181664F42BA13CA14DA15EA1C701B60123
:10C280000E9417AA0E9484AA4B015C018BA59CA561
:10C29000ADA5BEA5892B8A2B8B2BE9F160913306C6
:10C2A00070913406809135069091360668157905AF
:10C2B0008A059B0580F50E94B0AA2FA938AD49AD2B
:10C2C0005AAD0E944EAC6B017C016BA57CA58DA57F
:10C2D0009EA50E94B0AA6BA37CA38DA39EA3C501BB
:10C2E000B4010E94B0AA2BA13CA14DA15EA10E9465
:10C2F0004EACA70196010E9413AC181664F42BA152
:10C300003CA14DA15EA1C701B6010E9417AA0E94DF
:10C3100084AA4B015C010FA118A529A53AA5012B00
:10C32000022B032BE9F1609137067091380680915A
:10C33000390690913A06681579058A059B0580F5BE
:10C340000E94B0AA2FA938AD49AD5AAD0E944EAC9B
:10C350006B017C016FA178A589A59AA50E94B0AA5E
:10C360006BA37CA38DA39EA3C501B4010E94B0AAB8
:10C370002BA13CA14DA15EA10E944EACA70196014C
:10C380000E9413AC181664F42BA13CA14DA15EA130
:10C39000C701B6010E9417AA0E9484AA4B015C0142
:10C3A0004114510461047104A9F160913B0670913C
:10C3B0003C0680913D0690913E06681579058A05F8
:10C3C0009B0540F50E94B0AA2FA938AD49AD5AADE2
:10C3D0000E944EAC6B017C01C301B2010E94B0AA65
:10C3E0002B013C01C501B4010E94B0AAA301920136
:10C3F0000E944EACA70196010E9413AC181654F48B
:10C40000A3019201C701B6010E9417AA0E9484AA43
:10C410004B015C01F101E35BFF4F80829182A282BC
:10C42000B382C501B4010E94B0AA6B017C012BA9A3
:10C430003CA94DA95EA90E9417AA2B966CAF7DAFAF
:10C440008EAF9FAF2B97D10151966D937D938D93B6
:10C450009C9354972DEB37E346E051E4C701B601B6
:10C460000E944EAC0E9484AAF10161AB72AB83AB17
:10C4700094AB86A9882381F1FD9620813181428188
:10C4800053816091B1057091B2058091B30590918F
:10C49000B4050E944EAC2B962CAD3DAD4EAD5FADBC
:10C4A0002B970E944EAC20915F0630916006409120
:10C4B0006106509162060E944EAC9B01AC0160E0A7
:10C4C00074E284EF99E40E9417AA0E9484AAD10121
:10C4D000D8967C936E93D797D10111960D911D91AB
:10C4E0002D913C91149763960CAF1DAF2EAF3FAFCB
:10C4F0006397C901B8010E94BBAC6FA77BAF8FAB3C
:10C500009BA70FE016E065961FAF0EAF65973E0143
:10C5100011E1610E711C0FE016E021961FAF0EAF06
:10C5200021972D964EAC5FAC2D976BA37FA3182F50
:10C53000092F1BAAD201CD90DD90ED90FD902D0129
:10C5400020E030E0A901C701B6010E9413AC87FFCB
:10C5500004C0F7FAF094F7F8F0942196EEADFFAD31
:10C56000219781909190A190B1902196FFAFEEAF6D
:10C570002197A5019401C701B6010E9413AC1816BA
:10C580000CF03FC0FBA9FF2329F1A50194016FA581
:10C590007BAD8FA99BA50E944EAC4B015C012BA1EA
:10C5A0003FA1412F502FC701B6010E944EACA501FB
:10C5B00094010E9413AC181614F5A7019601C50149
:10C5C000B4010E9417AA6BA37FA3182F092F21E0A3
:10C5D0002BAB17C0A7019601C501B4010E9417AA91
:10C5E0009B01AC016BA17FA1812F902F0E944EACCB
:10C5F0006BA37FA3182F092F31E03BAB02C041E0B2
:10C600004BAB4614570409F095CF5BA1A5965FAFDD
:10C61000A5978FA1A6968FAFA697A7961FAFA797AE
:10C62000A8960FAFA89724969FAD2497992309F455
:10C630004CC1C090B605D090B705E090B805F09019
:10C64000B9052DEB37E346E855E3C701B6010E9473
:10C6500010AA87FD3AC1C701B6010E94BBAC6B01AD
:10C660007C019B01AC016FA57BAD8FA99BA50E94AE
:10C6700010AA87FD04C0CFA6DBAEEFAAFBA69601E9
:10C68000A7016FA57BAD8FA99BA50E9417AAA396B2
:10C690006CAF7DAF8EAF9FAFA397AAEBB5E02196AD
:10C6A000BFAFAEAF219720E030E040E85FE32BABB7
:10C6B0003CAB4DAB5EAB24961FAE24972196AEAD3E
:10C6C000BFAD21976D917D918D919D912196BFAFC9
:10C6D000AEAF2197A3962CAD3DAD4EAD5FADA39708
:10C6E0000E944EAC6B017C012D96EEADFFAD2D97F7
:10C6F00081909190A190B1902D96FFAFEEAF2D97C4
:10C700002496FFAD2497FF2391F02BA93CA94DA9B6
:10C710005EA90E944EAC6B017C012BA93CA94DA9DE
:10C720005EA9C501B4010E944EAC4B015C01A5019C
:10C730009401C701B6010E9413AC20E030E0A901CA
:10C7400018164CF5C501B4010E9413AC18164CF034
:10C7500020E030E0A901C701B6010E9410AA87FFBE
:10C7600009C0A5019401C701B6010E9436A92B0199
:10C770003C0139C02401350177FA709477F8709440
:10C78000A3019201C701B6010E9413AC18165CF513
:10C790002601370128C0C501B4010E9410AA87FDF7
:10C7A00009C020E030E0A901C701B6010E9413AC26
:10C7B00018164CF4A7019601C501B4010E9436A9D0
:10C7C0002B013C0110C02601370177FA709477F8ED
:10C7D0007094A5019401C301B2010E9413AC181614
:10C7E00014F0240135016596AEADBFAD6597CD90CF
:10C7F000DD90ED90FD906596BFAFAEAF6597A70158
:10C800009601C301B2010E9413AC1816CCF4A30127
:10C810009201C701B6010E9417AA9B01AC016BA946
:10C820007CA98DA99EA90E944EAC6BAB7CAB8DAB55
:10C830009EAB2496BFAD2497BF5F2496BFAF2497CD
:10C840002196EEADFFAD2197EA5CF54009F036CFB9
:10C8500024963FAD2497332371F02BA93CA94DA911
:10C860005EA96FA57BAD8FA99BA50E944EAC6FA75B
:10C870007BAF8FAB9BA724EA30E74DE75FE36FA563
:10C880007BAD8FA99BA50E944EAC6B017C019B01E7
:10C89000AC0160918C0570918D0580918E05909111
:10C8A0008F050E9413AC181654F4A70196016BA1D2
:10C8B0007FA1812F902F0E9413AC181634F00FA582
:10C8C0000BA31BAD1FA31FA90BA5A5968FADA59705
:10C8D000A6969FADA697A796AFADA797A896BFAD12
:10C8E000A89780938C0590938D05A0938E05B093A7
:10C8F0008F052BA13FA1412F502F6BA17FA1812F2D
:10C90000902F0E944EAC7B018C01CB01D801F1012C
:10C9100081879287A387B4872B966CAD7DAD8EAD52
:10C920009FAD2B9790589B01AC010E9437A96D9643
:10C930002CAD3DAD4EAD5FAD6D970E944EAC9B01F1
:10C94000AC016BE077ED83E29BE30E9436A95B01CB
:10C950006C01A496FFADA497FF2361F09B01AC018D
:10C96000B701C8010E9410AA87FD09C09A2D8B2D1E
:10C97000860107C09BE087ED03E21BE302C09E2D0A
:10C980008F2D492F582FB801D10115964D935D93E6
:10C990006D937C9318971C919501A60163966CADDD
:10C9A0007DAD8EAD9FAD63970E9410AA181614F44A
:10C9B00081E001C083E0182BF101108380E1FE01CA
:10C9C0003196AAEBB5E001900D928A95E1F7F1015D
:10C9D00081819281A381B4818093B6059093B7053C
:10C9E000A093B805B093B90580E16F96EEADFFADA9
:10C9F0006F97AEECB5E001900D928A95E1F780E17A
:10CA00006996EEADFFAD6997A1EAB5E001900D9290
:10CA10008A95E1F781E00BC02896EFAC2897FFAC30
:10CA200060960FAD609764961FAD649723C8C9598F
:10CA3000DF4F0FB6F894DEBF0FBECDBFDF91CF91B1
:10CA40001F910F91FF90EF90DF90CF90BF90AF902C
:10CA50009F908F907F906F905F904F903F902F901E
:10CA600008956F927F928F929F92AF92BF92CF92D2
:10CA7000DF92EF92FF920F931F93CF93DF9300D03B
:10CA80001F92CDB7DEB74C013B0180918806909193
:10CA90008906892BD9F590918D0680918A06981B7D
:10CAA0009F709F3059F429833A834B835C830E94A3
:10CAB00097A85C814B813A812981EDCFD0908D067A
:10CAC00080918D0666E5869FC00111245701C02E16
:10CAD00079018A019301A40160E08257994F0E9475
:10CAE000DF598823A9F020918D0690918A06291399
:10CAF00003C094E69093870691E09D0D9F709093FC
:10CB00008D0689830E948056898103C080E001C020
:10CB100081E00F900F900F900F90DF91CF911F91B8
:10CB20000F91FF90EF90DF90CF90BF90AF909F90CC
:10CB30008F907F906F90089580918D0690918A06D6
:10CB4000891B8F708F3019F40E9497A8F5CF8091C0
:10CB50008D068F5F8F70E0918D0696E59E9FF001A8
:10CB60001124E257F94FDF011D929A95E9F798E0F9
:10CB700090834091CE055091CF056091D005709182
:10CB8000D105458B568B678B708F4091D2055091A4
:10CB9000D3056091D4057091D505418F528F638F75
:10CBA000748F4091D6055091D7056091D80570914A
:10CBB000D905458F568F678F70A34091DA05509144
:10CBC000DB056091DC057091DD0541A352A363A3F1
:10CBD00074A320918D0690918A06291303C094E6D0
:10CBE0009093870680938D060C94772F2F923F9217
:10CBF0004F925F926F927F928F929F92AF92BF926D
:10CC0000CF92DF92EF92FF920F931F93CF93DF9318
:10CC1000CDB7DEB7A9970FB6F894DEBF0FBECDBF74
:10CC2000F801A0918806B0918906AB2B09F0A7C046
:10CC300016010E2DF8A7EFA33EA32DA36A017B01D9
:10CC4000FC014080518062807380209153063091B6
:10CC500054064091550650915606C301B2010E94F8
:10CC60004EAC0E941EAC698B7A8B8B8B9C8BD70150
:10CC70008D909D90AD90BC902091570630915806B4
:10CC80004091590650915A06C501B4010E944EAC1C
:10CC90000E941EAC6D8B7E8B8F8B988FD6012D9151
:10CCA0003D914D915C9129A33AA34BA35CA32091A4
:10CCB0005B0630915C0640915D0650915E0669A16D
:10CCC0007AA18BA19CA10E944EAC0E941EAC698FE0
:10CCD0007A8F8B8F9C8FEDA1FEA1C080D180E280E6
:10CCE000F38020915F06309160064091610650917B
:10CCF0006206C701B6010E944EAC0E941EAC6D8F49
:10CD00007E8F8F8F98A349825A826B827C828D821C
:10CD10009E82AF82B88629A13AA14BA15CA1298746
:10CD20003A874B875C87CD86DE86EF86F88A20912E
:10CD3000850323FF10C06093DA057093DB058093B1
:10CD4000DC059093DD05C092AD05D092AE05E09272
:10CD5000AF05F092B005AFA1B8A52D913D914D91D1
:10CD60005C917101BE016F5F7F4FCE01419679DE0C
:10CD7000882331F089A70E94772F89A501C080E020
:10CD8000A9960FB6F894DEBF0FBECDBFDF91CF914D
:10CD90001F910F91FF90EF90DF90CF90BF90AF90D9
:10CDA0009F908F907F906F905F904F903F902F90CB
:10CDB0000895AF92BF92CF92DF92EF920F931F939D
:10CDC000CF93DF93CDB7DEB764970FB6F894DEBF8D
:10CDD0000FBECDBFA98ABA8ACB8ADC8AFC018081CA
:10CDE0009181A281B38189839A83AB83BC83FB0148
:10CDF00080819181A281B3818D839E83AF83B88727
:10CE0000FA0180819181A281B38189879A87AB875A
:10CE1000BC87F90180819181A281B3818D879E8732
:10CE2000AF87B88BAE01475F5F4FBE016B5F7F4F2F
:10CE3000CE0101960E940A57CE0141966C019E01D7
:10CE4000235F3F4FAE01475F5F4FBE016B5F7F4F78
:10CE50004097CCDE64960FB6F894DEBF0FBECDBF10
:10CE6000DF91CF911F910F91EF90DF90CF90BF9006
:10CE7000AF9008958F929F92AF92BF92EF92FF92E0
:10CE80000F931F93CF93DF937B018A01E901FC018C
:10CE900080809180A280B380209153063091540607
:10CEA0004091550650915606C501B4010E944EAC02
:10CEB0000E941EAC6093CE057093CF058093D00581
:10CEC0009093D1052091570630915806409159060C
:10CED00050915A06F70160817181828193810E948D
:10CEE0004EAC0E941EAC6093D2057093D305809324
:10CEF000D4059093D50520915B0630915C06409156
:10CF00005D0650915E06F801608171818281938196
:10CF10000E944EAC0E941EAC6093D6057093D7055C
:10CF20008093D8059093D90520915F0630916006D3
:10CF30004091610650916206688179818A819B8166
:10CF40000E944EAC0E941EAC6093DA057093DB0524
:10CF50008093DC059093DD058092A1059092A20557
:10CF6000A092A305B092A405F70180819181A281CE
:10CF7000B3818093A5059093A605A093A705B093D0
:10CF8000A805F80180819181A281B3818093A905D0
:10CF90009093AA05A093AB05B093AC0588819981C5
:10CFA000AA81BB818093AD059093AE05A093AF0598
:10CFB000B093B00590918D0680918A06981759F02C
:10CFC000DF91CF911F910F91FF90EF90BF90AF90A5
:10CFD0009F908F90B1CD0E94475880916F0081FB48
:10CFE000CC27C0F981FF05C080916F008D7F8093B1
:10CFF0006F002AED35E046ED55E062ED75E08EEC10
:10D0000095E00E94A732CC2329F080916F008260C6
:10D0100080936F00DF91CF911F910F91FF90EF9060
:10D02000BF90AF909F908F900895CF93DF93CDB72F
:10D03000DEB760970FB6F894DEBF0FBECDBFFC0120
:10D0400080819181A281B38189839A83AB83BC83E0
:10D05000FB0180819181A281B3818D839E83AF8307
:10D06000B887FA0180819181A281B38189879A87EB
:10D07000AB87BC87F90180819181A281B3818D87C3
:10D080009E87AF87B88BAE01475F5F4FBE016B5F76
:10D090007F4FCE0101960E940A579E01235F3F4FAA
:10D0A000AE01475F5F4FBE016B5F7F4FCE010196C0
:10D0B000E1DE60960FB6F894DEBF0FBECDBFDF9104
:10D0C000CF910895CF92DF92EF92FF92FC01C08042
:10D0D000D180E280F38020915F063091600640911C
:10D0E000610650916206C701B6010E944EAC0E94D3
:10D0F0001EAC6093DA057093DB058093DC0590939A
:10D10000DD05C092AD05D092AE05E092AF05F0927C
:10D11000B00590918D0680918A06981729F0FF90AE
:10D12000EF90DF90CF9008CD0E94475880916F001C
:10D1300081FB992790F981FF05C080916F008D7F59
:10D1400080936F004091DA055091DB056091DC051A
:10D150007091DD054093E3045093E4046093E5048B
:10D160007093E604992329F080916F008260809388
:10D170006F00FF90EF90DF90CF900895CF92DF92F5
:10D18000EF92FF920F931F93CF93DF93CFE3D6E0FD
:10D190000FE216E0C12CD12C7601C39469917991EC
:10D1A000899199910E94B0AA288939894A895B8915
:10D1B0000E944EAC0E9484AAF801619371938193FE
:10D1C00091938F01C616D706E806F90610F46B0195
:10D1D0007C01F6E0CF34DF0709F76FEF7FEFCB017B
:10D1E000A70196010E943BAD2093CA053093CB0561
:10D1F0004093CC055093CD05DF91CF911F910F91B6
:10D20000FF90EF90DF90CF9008950F931F93CF93EF
:10D21000DF9303E516E0CFE1D6E0F80121913191EB
:10D22000419151918F0160E070E080E89FE30E949E
:10D2300017AA6993799389939993F6E0CF32DF0720
:10D2400061F725E835E041E855E06DE775E089E7ED
:10D2500095E0EBDEDF91CF911F910F918FCF8EEE96
:10D260009BE00C94845181548A3108F041C0A82F6E
:10D27000B0E04091170C5091180C6091190C70910E
:10D280001A0C04C076956795579547958A95D2F7FD
:10D2900040FF2EC0E091220CF091230CA350B44F1C
:10D2A0008C918823E9F0E80FF11D808190ED980FB3
:10D2B0009A3098F08E3211F481810CC08D3211F0C9
:10D2C0008B3271F4818190ED980F9A3030F08E326C
:10D2D00039F4828180538A3018F49E2F8F2F02C038
:10D2E00090E080E090931E0C80931F0C81E00895E5
:10D2F00080E00895B8DF882341F081E020911E0C82
:10D3000030911F0C232B09F480E008950F931F9395
:10D31000CF9380911E0C90911F0C009711F1FC018E
:10D320008F01C1912C2F2F7DA9F0C53411F0C53686
:10D33000B9F7F801108260E070E080911E0C9091C6
:10D340001F0C0E94A0ADF801C083562F472F382F25
:10D35000292F0BC060E070E0CF911F910F910C94CA
:10D36000A0AD50E040E030E020E0652F742F832F27
:10D37000922FCF911F910F91089580911E0C909143
:10D380001F0C009731F04AE050E060E070E00C9430
:10D3900006AF60E070E0CB010895CF9384E5AADF8B
:10D3A000882359F1EADF97FD24C0E7DF6F3F71055D
:10D3B0008105910509F0FCF4E0DFC62F1616FCF498
:10D3C0000E9412168DE40E9494186AE070E0809129
:10D3D0001B0C90911C0C0E9487196C2FCC0F770BA3
:10D3E00087E695E10E9435168AE00E9494188FEF37
:10D3F00007C0C0E004C0CFEF02C080E001C08C2FA6
:10D40000CF910895BF92CF92DF92EF92FF920F9348
:10D410001F93CF93DF9389E6E82E85E0F82E09E786
:10D4200015E094EFC92E9BE0D92EC9E2D3E0BC2EC3
:10D4300084E0B80E899117DF8823B1F067DFF60129
:10D440002081211104C020918905222339F0F8019F
:10D4500020813181428153810E9437A9F701608385
:10D460007183828393830AC0F80180819181A281B4
:10D47000B381F70180839183A283B383F4E0EF0E3D
:10D48000F11C0C5F1F4F8FEFC81AD80ABC12D2CF05
:10D4900086E430DF8823B9F039DF20E030E0A901ED
:10D4A0000E9413AC18167CF431DF20E030E040E736
:10D4B00052E40E9417AA6093480270934902809335
:10D4C0004A0290934B02DF91CF911F910F91FF90F1
:10D4D000EF90DF90CF90BF900895CF92DF92EF92C0
:10D4E000FF926B017C010E948711C60ED71EE81EB9
:10D4F000F91E0E948711DC01CB018C199D09AE0930
:10D50000BF09B7FF03C00E9497A8F3CFFF90EF9029
:10D51000DF90CF9008956F927F928F929F92AF92FB
:10D52000BF92CF92DF92EF92FF920F931F93CF9310
:10D53000DF93CDB7DEB73C01A090220CB090230C56
:10D54000CDB6DEB66AE070E0C3010E9473B17C0123
:10D55000009721F08C010619170904C0C3010E942D
:10D560007EB18C01C80101962DB73EB7281B390B3F
:10D570000FB6F8943EBF0FBE2DBF8DB79EB7019674
:10D580004C01A801B3010E949FB1F401E00FF11F0B
:10D590001082C40148D581E034D0E114F10451F087
:10D5A00037019FEF691A790A0FB6F894DEBE0FBEF5
:10D5B000CDBEC6CF0FB6F894DEBE0FBECDBEC50140
:10D5C000DF91CF911F910F91FF90EF90DF90CF905F
:10D5D000BF90AF909F908F907F906F9024C5CF9316
:10D5E000C3E00E943785882341F0C15019F00E94A2
:10D5F00081A7F7CFCF910C94AEA780E595E1CF91AD
:10D600008ACFCF93C82F41E04093F30B90911D0C2C
:10D610009D3409F45EC0943509F4F7C1973409F0DC
:10D62000F8C120911B0C30911C0C2B31310509F4F1
:10D630003EC0CCF42430310544F42230310564F589
:10D6400037FDE7C10E94DC94E7C12C30310561F160
:10D650002531310509F4E0C12430310509F0D9C183
:10D660000E94E594D9C12A35310551F154F42D3188
:10D67000310521F1FCF02E31310509F0CAC151D23A
:10D68000CBC12C35310511F1F4F0293A314009F0C4
:10D69000C0C10E94ED82C0C181E02230310509F095
:10D6A00080E00E940D99B8C10E94F68FB5C10E941A
:10D6B000FA8FB2C180E00E94EB78AEC190DFACC1BE
:10D6C00010928905A9C140938905A6C10E941777C8
:10D6D000A3C120911B0C30911C0C2937310509F492
:10D6E0005DC10CF083C02836310509F42AC10CF065
:10D6F00044C02C34310509F421C104F5223131052F
:10D7000009F43EC164F437FD84C1223031050CF4C4
:10D710000DC12131310509F07CC19FD77DC12A326D
:10D72000310509F405C12B34310509F404C12F3149
:10D73000310509F06EC10E94F8756EC123353105BF
:10D7400009F41BC16CF42135310509F411C10CF049
:10D7500011C12D34310509F05CC10E9436755CC1E0
:10D760002535310509F40EC10CF40AC12C353105FB
:10D7700009F04FC10E9483914FC12037310509F450
:10D780004BC1CCF42C36310509F446C15CF42A3681
:10D79000310509F4E7C00CF0E8C00E94509F1092D8
:10D7A000F30B41C12E36310509F4CEC00CF0CFC0C9
:10D7B0000E94DD9E31C12537310509F4E8C06CF4C3
:10D7C0002237310509F4E0C00CF4C3C0233731051A
:10D7D00009F01FC10E94B1761FC12737310509F436
:10D7E000D8C00CF0D9C00E94657616C12E3581E0F4
:10D7F000380709F408C10CF04BC0233D310509F48A
:10D80000D8C01CF5293C310509F4CAC07CF42B3979
:10D81000310509F4A4C02E3B310509F49DC02C3814
:10D82000310509F0F6C00E94349EF6C02C3C31054B
:10D8300009F4B9C02D3C310509F4B8C02B3C3105C1
:10D8400009F0E7C00E941D93E7C02D3281E0380740
:10D8500009F4B6C07CF42D3D310509F4ACC0223E7C
:10D86000310509F4ABC02C3D310509F0D2C00E944E
:10D870003291D2C02F3281E0380709F4A7C00CF4EE
:10D88000A2C02033314009F0C4C00E94C090C4C07F
:10D89000243F81E0380709F4A8C014F5223981E05B
:10D8A000380709F49AC06CF4203981E0380709F48C
:10D8B00090C00CF090C02F35314009F0AAC0ACD513
:10D8C000ABC0243A81E0380709F489C0293A81E0E5
:10D8D000380709F487C02A39314009F09AC09CC042
:10D8E000283F81E0380709F486C04CF4263F81E0E8
:10D8F000380709F47CC00CF07CC012D58DC02438E8
:10D9000083E0380709F479C034F42335334009F053
:10D9100080C040D281C02B3883E0380709F470C042
:10D92000273E334009F075C091D776C0ACD274C0A1
:10D930000E94D37471C00E9432756EC00E9434750B
:10D940006BC00E94BA9E68C00E94FD7665C00BD76E
:10D9500063C00E94237660C00E944D9E5DC00E94FD
:10D96000739E5AC00E94339F57C00E94499F54C063
:10D970005FD752C00E94D5944FC00E94D8944CC02B
:10D980006ED64AC019D648C00E94617645C07AD288
:10D9900043C00E94597640C07FD73EC080D73CC06C
:10D9A0000E94EE9239C00E94429336C00E94B89302
:10D9B00033C07AD731C00E9465902EC0C1D52CC02B
:10D9C0000E943E9429C00E94579226C00E947F9DCB
:10D9D00023C068D721C09BD01FC09ED01DC00E940D
:10D9E0001D841AC00E94A67717C098D415C09AD477
:10D9F00013C09AD411C0BCD40FC00E94758F0CC044
:10DA00000E94469009C0D3D407C080911B0C1FD63A
:10DA100003C08CEF9BE072D41092F30BC11103C0D2
:10DA2000CF910C94999BCF910895CF93DF93C091A0
:10DA3000BE0E80E6C89FE0011124C352D34F8091EF
:10DA4000850380FF05C00E941216CE010E94EB18CC
:10DA5000CE01E9D280E0DF91CF91D3CDCF92DF929A
:10DA6000EF92FF920F931F930E9487116B017C012D
:10DA70008091DE0E81112FC080915202882359F1CE
:10DA80008091F30B882339F14091EF0B5091F00B0B
:10DA90006091F10B7091F20B97018601041B150B3D
:10DAA000260B370B37FD2CC0833079F03CF48130E6
:10DAB00094F00E9412168EE395E10BC0843059F465
:10DAC0000E9412168FE095E104C00E94121687E2B0
:10DAD00095E10E9404162091520230E0A8EEB3E0D6
:10DAE0000E9481ADDC01CB018C0D9D1DAE1DBF1DC3
:10DAF0008093EF0B9093F00BA093F10BB093F20B8C
:10DB00001F910F91FF90EF90DF90CF90089581E0EB
:10DB10000E94B1480C94F54B80E00E94B1480C94EF
:10DB2000F54B8F929F92AF92BF92CF92DF92EF927E
:10DB3000FF920F931F93CF93DF93CDB7DEB7289754
:10DB40000FB6F894DEBF0FBECDBFC0907905D09060
:10DB50007A05E0907B05F0907C0588E5CBDB8111B0
:10DB600008C020E030E0A901C701B6010E9437A932
:10DB700001C0CCDB6D837E838F839887C0907D0549
:10DB8000D0907E05E0907F05F090800589E5B2DBBE
:10DB9000811108C020E030E0A901C701B6010E9450
:10DBA00037A901C0B3DB6B017C0169837A838B8366
:10DBB0009C838D809E80AF80B88422ED30E040EE63
:10DBC00050EC0E9413AC87FDD2C027E030E04EE35A
:10DBD00053E4C701B6010E9410AA18160CF4C7C07E
:10DBE00023EA31E040E450ECC501B4010E9413ACDB
:10DBF00087FDBDC027E030E042E253E4C501B40137
:10DC00000E9410AA18160CF4B2C027E030E041E2DE
:10DC100053E4C501B4010E9410AA18160CF4A7C061
:10DC200027E030E041E253E4C701B6010E9410AAA8
:10DC300018160CF49CC080E00E94881A0E94584E6E
:10DC400085E458DB182F8823B1F080911E0C909149
:10DC50001F0C892B09F489C090DB97FD0FC08DDB69
:10DC60006F3F71058105910509F04CF486DB611168
:10DC70007CC040E005C085E4F6DA77C010E0412FB3
:10DC800001E021E0BE016F5F7F4FCE0105960E944B
:10DC900052496B017C019B01AC010E94FCAC8111DB
:10DCA0005FC08D809E80AF80B88420E030E0A90105
:10DCB000C501B4010E9410AA87FD05C027E137EB1A
:10DCC00041E558E304C027E137EB41E558EBC501D6
:10DCD000B4010E9437A9AB01BC0184E895E10E9420
:10DCE0004F1689809A80AB80BC8020E030E0A9018B
:10DCF000C501B4010E9410AA87FD05C027E137EBDA
:10DD000041E558E304C027E137EB41E558EBC50195
:10DD1000B4010E9437A9AB01BC018FE795E10E94D5
:10DD20004F1620E030E0A901C701B6010E9410AAF9
:10DD300087FD05C027E137EB41E558E304C027E143
:10DD400037EB41E558EBC701B6010E9437A9AB019B
:10DD5000BC018AE795E10E944F168AE00E94941860
:10DD60000E94774E0E94F54B02C041E089CF289671
:10DD70000FB6F894DEBF0FBECDBFDF91CF911F91DC
:10DD80000F91FF90EF90DF90CF90BF90AF909F905A
:10DD90008F900895EF92FF920F931F93CF93DF938D
:10DDA0008AE561DA882309F456C080911E0C9091AF
:10DDB0001F0C009709F44FC0FC017F01C1912C2F6B
:10DDC0002F7D89F0C53411F0C536B9F7F7011082FF
:10DDD00060E070E080911E0C90911F0C0E94A0AD3D
:10DDE000F701C08304C060E070E00E94A0AD8B0129
:10DDF000D82FC92F20E030E040E050EC0E9413AC57
:10DE000087FD1DC020E030E040EA50E4B8018D2FCE
:10DE10009C2F0E9410AA181694F0C801AD2FBC2F99
:10DE20008093530590935405A0935505B0935605E0
:10DE3000DF91CF911F910F91FF90EF9008950E9475
:10DE400015168DE995E1DF91CF911F910F91FF900C
:10DE5000EF900C9404160E941216409153055091B5
:10DE6000540560915505709156058CE895E10E9426
:10DE70004F168AE0DF91CF911F910F91FF90EF90A5
:10DE80000C9494180895CF92DF92EF92FF920F9323
:10DE90001F93CF93DF93C091200CD091210C80E58C
:10DEA00029DA8823D1F080911E0C90911F0C0097E5
:10DEB00049F04AE050E060E070E00E942EB06B0153
:10DEC0007C0103C0C12CD12C760111E0C114D10416
:10DED000E104F10431F410E004C010E0C12CD12CB5
:10DEE000760183E507DA882309F486C080911E0C49
:10DEF00090911F0C009701F1FC017F010191202FEF
:10DF00002F7D89F0053411F00536B9F7F70110823D
:10DF100060E070E080911E0C90911F0C0E94A0ADFB
:10DF2000F701008304C060E070E00E94A0ADB62F4E
:10DF3000A72FF82FE92F04C0B0E0A0E0F0E0E0E068
:10DF400020E030E04AE754E46B2F7A2F8F2F9E2F8A
:10DF50000E944EAC0E9484AA6B017C01111109C081
:10DF6000672B682B692B29F4209719F08881811180
:10DF700002C010E001C011E00E944758112329F0AF
:10DF80000E941216CE010E94EB1883E08093F30BDF
:10DF900081E08093DF0EC114D104E104F10429F182
:10DFA0000E948711C60ED71EE81EF91E0E94871117
:10DFB000DC01CB018C199D09AE09BF09B7FD0EC06C
:10DFC0001092DF0E81E08093F30BDF91CF911F91D0
:10DFD0000F91FF90EF90DF90CF9008958091DF0E2A
:10DFE000882371F30E9497A8E1CF8091DF0E8823E8
:10DFF00039F30E9497A8F9CF1111BBCFB5CF10927A
:10E00000210C1092200C8FE380931D0C10921C0C9D
:10E0100010921B0C1092170C1092180C1092190CE5
:10E0200010921A0C08953F924F925F926F927F92D6
:10E030008F929F92AF92BF92CF92DF92EF92FF9218
:10E040000F931F93CF93DF931F921F92CDB7DEB72D
:10E0500089839A83D4DF8981282F9A81392FF90106
:10E0600080812F5F3F4F8032D1F38E34B1F48181B4
:10E0700090ED980F9A3020F08D3211F08B3269F4C8
:10E080003296DF0131962C9120532A30D0F3CD0106
:10E09000FC01019620812032D9F3F093230CE09308
:10E0A000220C8F010F5F1F4F30806AE270E0C801C1
:10E0B0000E94D5B1009731F0FC0131978081803208
:10E0C000E1F311828DE4381631F0E4E53E1619F0E3
:10E0D000F7E43F12FFC0F80180810F5F1F4F8032CD
:10E0E000D1F380538A3008F0F5C030921D0C1092A5
:10E0F0001C0C10921B0C4AE020911B0C30911C0C44
:10E10000429FC001439F900D112490931C0C80935B
:10E110001B0C3196DF0111972C91022E000C330B52
:10E1200020533109280F391F30931C0C20931B0CEE
:10E13000808180538A3000F3DF0131968C918032E8
:10E14000D9F38DE438121AC02E31310591F03CF428
:10E150002731310571F02C31310581F40AC02537A2
:10E16000310564F02737310524F0203AE3E03E071B
:10E1700029F4B093210CA093200CACC01092210C78
:10E180001092200C5091220CC12CD12C7601C394FA
:10E19000FD0131964C91442309F49CC04132A9F40D
:10E1A0008DE4381212C02032310579F4F093210C3D
:10E1B000E093200C63E270E0CF010E94D5B100979C
:10E1C00009F488C0FC01108285C041544A3108F02E
:10E1D00055C0BF01FB0180816F5F7F4F8032D1F35B
:10E1E00090ED980F9A3008F18E3211F481810CC0B5
:10E1F0008D3211F08B3259F4818190ED980F9A3065
:10E20000A0F08E3221F4828180538A3070F08091A8
:10E21000200C9091210C892B09F059C0CF01019756
:10E220009093210C8093200C52C0CF01A42FB0E01A
:10E230004601570104C0880C991CAA1CBB1C4A95B6
:10E24000D2F74090170C5090180C6090190C7090F9
:10E250001A0C84289528A628B7288092170C90922B
:10E26000180CA092190CB0921A0C009711F0851B93
:10E2700001C080E0A350B44F8C930AC08091200C61
:10E280009091210C892B21F4B093210CA093200CA8
:10E29000808181548A3130F4DF017ACF80ED890F9B
:10E2A0008A3040F44E2F6F2F91919111F7CF842F28
:10E2B000962F07C083ED890F8230A0F39B3291F334
:10E2C000F6CFFC01019640814032D9F3E5CF80E0E2
:10E2D00090E0ACCF0F900F90DF91CF911F910F91F5
:10E2E000FF90EF90DF90CF90BF90AF909F908F9076
:10E2F0007F906F905F904F903F9008950E9412160C
:10E300006091220C7091230C88EB95E10E94181605
:10E3100082E20E9494188AE00C9494180C94AF3B0B
:10E320000C94AA480C943C3FCF9383E50E94336938
:10E33000C82F8823B9F080911E0C90911F0C892B57
:10E34000A9F01BD897FD0BC018D86F3F7105810548
:10E35000910509F02CF411D8611108C003C0C0E088
:10E3600081E0C8278C2FCF910C947F40C0E0FACF7A
:10E370000E94A348882331F00E9412168BEC95E18D
:10E380000C94041608950E94BD6997FD0CC00E946C
:10E39000BD696F3F71058105910509F034F40E9454
:10E3A000BD69862F089580E008958FEF08950F933B
:10E3B0001F93CF9383E50E943369811104C00DE25E
:10E3C00013E0C0E00DC0C0E0DEDF682F8C2F0E949C
:10E3D0002A3ACF5FC530C1F7F2CFCF5FC43069F0C2
:10E3E000F80181918F010E9433698823B1F3CBDF5B
:10E3F000682F8C2F0E942A3AF0CF82E40E94336962
:10E40000882329F0C0DF682F84E00E942A3ACF9148
:10E410001F910F910C94D43A0F931F93CF9383E5E0
:10E420000E947A69882309F465C0ADDF823029F142
:10E43000833009F43FC0813009F05CC00DE213E085
:10E44000C0E0F80181918F010E947A69882339F038
:10E450009ADF2FEF4FEF682F8C2F0E94D339CF5FB9
:10E46000C43079F782E40E947A69882309F442C0B3
:10E470008ADF2FEF4FEF682F3AC00DE213E0C0E0C4
:10E48000F80181918F010E947A69882339F07BDF3E
:10E490002FEF482F6FEF8C2F0E94D339CF5FC430FE
:10E4A00079F782E40E947A69882321F16CDF2FEFEB
:10E4B000482F1CC00DE213E0C0E0F80181918F01EC
:10E4C0000E947A69882339F05EDF282F4FEF6FEFC3
:10E4D0008C2F0E94D339CF5FC43079F782E40E9439
:10E4E0007A69882339F04FDF282F4FEF6FEF84E0F0
:10E4F0000E94D339CF911F910F910C94D43ACF93AE
:10E50000DF931F921F92CDB7DEB769837A830E9493
:10E51000336969817A81882361F080911E0C909122
:10E520001F0C009731F04AE050E060E070E00E947C
:10E5300006AF972F862F0F900F90DF91CF91089500
:10E540001F93CF93DF9380E50E943369882381F185
:10E5500060E070E080E5D3DF182F6FEF7FEF83E599
:10E56000CEDFEC010196039718F517FD21C00E943C
:10E570004758CF3F8FEFD80729F0219771F4C1E0BA
:10E58000D0E00DC0812F0E94DB1331E020E0892B09
:10E5900009F030E0C32FD22F02C0C0E0D0E0812FBD
:10E5A0000E94DB138C179D0719F00E9497A8F7CFE4
:10E5B000DF91CF911F9108950F931F93CF9383E520
:10E5C0000E943369882309F43EC080911E0C90910B
:10E5D0001F0C009701F1FC018F01C1912C2F2F7DA1
:10E5E00089F0C53411F0C536B9F7F801108260E042
:10E5F00070E080911E0C90911F0C0E94A0ADF8015C
:10E60000C08304C060E070E00E94A0ADB62FA72FC9
:10E61000F82FE92F04C0B0E0A0E0F0E0E0E020E057
:10E6200030E04AE754E46B2F7A2F8F2F9E2F0E9401
:10E630004EAC0E9484AA6093DA0E7093DB0E809336
:10E64000DC0E9093DD0ECF911F910F91089520E085
:10E6500040E050E0BA010C94262F0C9467A70F936A
:10E660001F93CF9383E50E943369882391F18091B2
:10E670001E0C90911F0C009761F1FC018F01C1915C
:10E680002C2F2F7D89F0C53411F0C536B9F7F8016C
:10E69000108260E070E080911E0C90911F0C0E942F
:10E6A000A0ADF801C08304C060E070E00E94A0AD9E
:10E6B00020E030E04AE754E40E944EAC0E9484AA75
:10E6C00060935702709358028093590290935A02B4
:10E6D00046C088E50E943369811114C089E50E9413
:10E6E000336981110FC08AE50E94336981110AC024
:10E6F00085E40E943369811105C0CF911F910F916C
:10E700000C9422580E94475888E50E943369882358
:10E7100031F0179A80918A058E7F80938A0589E56A
:10E720000E943369882331F0169A80918A058D7F83
:10E7300080938A058AE50E943369882331F0159A0F
:10E7400080918A058B7F80938A0585E40E943369D6
:10E75000882329F0CF911F910F910C946CA7CF9132
:10E760001F910F910895FF920F931F93CF93DF9303
:10E7700083E50E9433698823F1F083E50E943369C1
:10E78000811102C060E015C080911E0C90911F0C99
:10E79000892BC1F30E94BD6997FDF4CF0E94BD692A
:10E7A0006F3F71058105910511F00CF03FC00E948B
:10E7B000BD69609385030E9412168AE096E10E946B
:10E7C000041680918503882329F100E016E1C0E05A
:10E7D000D0E020E08091850390E00C2E02C095955A
:10E7E00087950A94E2F780FF0EC0FF24F394F20E9F
:10E7F000222319F08CE20E949418F80185919491DB
:10E800000E9404162F2D21960E5F1F4FC530D10593
:10E8100009F704C08CEF95E10E9404168AE0DF91AD
:10E82000CF911F910F91FF900C9494186FEFC1CF6F
:10E830000E94AB200E94B7A40E9422581092C004EC
:10E8400068EE73E080E090E00C94C21581E0809364
:10E850005C0283E50E943369882331F080911E0CAD
:10E8600090911F0C892B39F483E50E943369811143
:10E8700012C00C94F89B0E94BD6997FDFACF0E94CC
:10E88000BD696F3F71058105910509F024F40E946F
:10E89000BD69662371F3089581E00C94C32D80E077
:10E8A0000C94C32D0C944758CF930E94121681E309
:10E8B00096E10E94041683E50E943369C82F8823DD
:10E8C000D1F080911E0C90911F0C892B91F00E9429
:10E8D000BD6997FD0DC00E94BD696F3F710581053F
:10E8E000910509F034F40E94BD69C1E0611101C0D5
:10E8F000C0E0C0934102809141020E94891689E2E2
:10E9000096E10E94041640913502509136026091C2
:10E9100037027091380287E296E10E944F164091CB
:10E92000390250913A0260913B0270913C0284E2BC
:10E9300096E10E944F1640913D0250913E02609137
:10E940003F027091400281E296E10E944F1689E1F8
:10E9500096E10E9404164091290250912A0260918A
:10E960002B0270912C0287E196E10E944F16409194
:10E970002D0250912E0260912F027091300284E19D
:10E9800096E10E944F1640913102509132026091FF
:10E9900033027091340281E196E10E944F168AE0C1
:10E9A000CF910C9494180F931F93CF93DF9383E52B
:10E9B0000E947A69882309F450C0E5DC182F80E5AD
:10E9C0000E947A6981110AC081E0111101C080E0C2
:10E9D000DF91CF911F910F910C94AC1580E50E94AF
:10E9E0007A69882331F00E94BD69EB0177FD35C05B
:10E9F00002C0CDE0D0E00C2F89E40E947A69882320
:10EA000051F080911E0C90911F0C892B49F0BBDCBA
:10EA1000811106C017C089E40E943369882391F0F0
:10EA200061E08C2F0E947013612F8C2F0E94AC1319
:10EA3000612F70E08C2F0E945312083071F41093F4
:10EA4000C0040BC0802F0E9430A7882349F3DF91B8
:10EA5000CF911F910F910C9458A7DF91CF911F91E7
:10EA60000F9108950C9430A50C94CCA40C94B7A4E9
:10EA70004F925F926F927F92AF92BF92CF92DF924E
:10EA8000EF92FF92CF93DF93EB01FC0160817181E4
:10EA9000828193812CE3C22ED12CE12CF12CA70191
:10EAA00096010E943BADB62EA72ECA01B901A7015F
:10EAB00096010E943BAD6B017C01CA01B90128E1BE
:10EAC00030E040E050E00E943BAD2B013C01C90129
:10EAD0006DE671E00E9427AD61157105D9F0AF9226
:10EAE000BF92DF92CF925F924F929F938F937F93CB
:10EAF0006F9389E696E19F938F93DF93CF930E9464
:10EB000000B28DB79EB70E960FB6F8949EBF0FBE9B
:10EB10008DBF61C00097C9F0AF92BF92DF92CF92D4
:10EB20005F924F929F938F9389E596E19F938F9386
:10EB3000DF93CF930E9400B2EDB7FEB73C960FB6BD
:10EB4000F894FEBF0FBEEDBF46C0411451046104EE
:10EB50007104B9F0AF92BF92DF92CF925F924F9261
:10EB60008DE496E19F938F93DF93CF930E9400B241
:10EB70008DB79EB70A960FB6F8949EBF0FBE8DBF95
:10EB80002AC0C114D104E104F104A9F0AF92BF92EC
:10EB9000DF92CF9285E496E19F938F93DF93CF939B
:10EBA0000E9400B2EDB7FEB738960FB6F894FEBFDC
:10EBB0000FBEEDBF10C0AF92BF9281E496E19F936C
:10EBC0008F93DF93CF930E9400B20F900F900F901E
:10EBD0000F900F900F90DF91CF91FF90EF90DF900B
:10EBE000CF90BF90AF907F906F905F904F900895BF
:10EBF000CF93DF93CDB7DEB769970FB6F894DEBF3A
:10EC00000FBECDBF0E94FCA46E8B7F8B888F998F27
:10EC1000BE016F5F7F4FCE0146962ADF0E9412161B
:10EC2000BE016F5F7F4F8DE796E10E9418168AE064
:10EC30000E94941869960FB6F894DEBF0FBECDBF40
:10EC4000DF91CF91089583E50E943369882331F0E5
:10EC500080911E0C90911F0C892B71F40E9412164A
:10EC60004091520250E060E070E08AE896E10E9434
:10EC700079168AE00C9494180E94BD6997FD17C01C
:10EC80000E94BD696F3F71058105910509F01CF473
:10EC90000E94BD6901C06FEF862F90E0CD971CF4F4
:10ECA0006093520208958CE380935202089560E0CD
:10ECB000F3CF81E00E94AC150E942A2E80E00C94D4
:10ECC000AC150E9447580C94F54B1F93CF93DF93DC
:10ECD000C091200CD091210C83E010E040E08150E5
:10ECE000C9F09881292F2B7F2134C9F7298121333D
:10ECF000B1F7913421F0953419F441E001C011E0ED
:10ED00009E012E5F3F4FE9012F5F3F4F9881903268
:10ED1000D1F3E5CF41110E941216112321F081E9B0
:10ED200096E10E940416CE01DF91CF911F910C94C1
:10ED3000EB180F931F93CF938C01C62F85E996E1B3
:10ED40000E940416C8010E9404168AE30E949418C7
:10ED50006AE070E08C2F90E0CF911F910F910C949E
:10ED60008D1985E997E10E94041660E085E897E136
:10ED7000E0DF61E08EE797E1DCDF60E083E797E1C9
:10ED8000D8DF61E083E697E1D4DF60E08AE597E1D0
:10ED9000D0DF61E080E597E1CCDF61E086E497E1D8
:10EDA000C8DF61E08EE397E1C4DF61E080E397E1D3
:10EDB000C0DF60E082E297E1BCDF60E083E197E1E1
:10EDC000B8DF60E085E097E1B4DF60E08FEE96E1C8
:10EDD000B0DF61E08EED96E1ACDF60E08FEC96E1B4
:10EDE000A8DF60E08AEB96E1A4DF61E087EA96E1C4
:10EDF000A0DF60E08AE996E19CCF8EE40E9433694F
:10EE00008823A1F080911E0C90911F0C009771F047
:10EE10004AE050E060E070E00E9406AF6093C00EF0
:10EE20007093C10E8093C20E9093C30E08954F92BB
:10EE30005F926F927F929F92AF92BF92CF92DF923A
:10EE4000EF92FF920F931F93CF93DF9381E3E82E0E
:10EE500083E0F82E09E715E0B12C912CA12CF701E5
:10EE600081917F010E943369882309F450C0809109
:10EE70001E0C90911F0C009709F449C0FC013F0142
:10EE8000C1912C2F2F7D89F0C53411F0C536B9F70B
:10EE9000F301108260E070E080911E0C90911F0CD5
:10EEA0000E94A0ADF301C08304C060E070E00E9446
:10EEB000A0AD6B01D82FC92FF8012081318142818B
:10EEC00053810E9436A92B013C012DEB37E346E824
:10EED00055EB0E9413AC87FD0AC02DEB37E346E8E3
:10EEE00055E3C301B2010E9410AA181684F4F3E09E
:10EEF000BF1619F09924939402C0AA24A394A601E2
:10EF00006D2F7C2FF8014083518362837383B39408
:10EF10000C5F1F4FF4E0BF12A2CF992019F00E949E
:10EF20001D4C03C0A1100E94274CDF91CF911F916F
:10EF30000F91FF90EF90DF90CF90BF90AF909F9098
:10EF40007F906F905F904F900C94F54BBF92CF9253
:10EF5000DF92EF92FF920F931F93CF93DF9325E3FE
:10EF6000E22E23E0F22E04E21CE06701C0E0D0E0D4
:10EF7000BB24B394F60181916F010E943369882309
:10EF800051F10E944758F8016081662389F070E0D2
:10EF900080E090E00E94B2AA9B01AC01FE01E95D15
:10EFA000F34F60817181828193810E9417AA03C00F
:10EFB00060E070E0CB0120911E0C30911F0C232BE0
:10EFC00011F00E948669FE01E95CF34F6083718352
:10EFD00082839383B12C24960F5F1F4FCC30D105D1
:10EFE00049F686E40E943369882371F10E944758EC
:10EFF0000E9486698B01D82FC92F20E030E040E8BD
:10F000005FE30E9413AC18167CF020E030E0A90109
:10F01000B8018D2F9C2F0E9410AA87FF09C000E025
:10F0200010E0D0E0C0E004C000E010E0D0E8CFE3A2
:10F03000C801AD2FBC2F8093330C9093340CA09358
:10F04000350CB093360CB12C83E50E9433698823CC
:10F0500069F00E9447580E9486696093530270933A
:10F0600054028093550290935602ABC0BB2009F422
:10F07000A8C089E599E10E94041620E030E0A901CA
:10F080006091330C7091340C8091350C9091360C5A
:10F090000E9410AA811104C086E599E10E9404161D
:10F0A0008DE499E10E9404164091330C5091340C88
:10F0B0006091350C7091360C89E299E10E944F16EF
:10F0C00088E099E10E94041686EE98E10E940416F9
:10F0D00007E31CE0C5E3D3E093E0D92EDE0C80E229
:10F0E0000E94941889910E949418F801619171917D
:10F0F000819191918F0142E050E00E94121A8AE0C2
:10F100000E949418DC12EBCF4091530250915402AC
:10F11000609155027091560282EC98E10E944F1660
:10F120008AE00E94941880EA98E10E94041687E21F
:10F13000C82E8CE0D82EC4E2DCE013E01C0F8881DE
:10F140008823D1F080E20E949418F70180810E9408
:10F150009418688170E080E090E00E94B2AA9B0160
:10F16000AC01F60160817181828193810E9417AAAE
:10F1700042E050E00E94121A2196FFEFEF1AFF0AB8
:10F1800084E0C80ED11C1C13DACF8091240C8111AD
:10F190000CC08091250C811108C08091260C811132
:10F1A00004C08CE898E10E9404168AE0DF91CF91B8
:10F1B0001F910F91FF90EF90DF90CF90BF900C9434
:10F1C0009418DF91CF911F910F91FF90EF90DF90F6
:10F1D000CF90BF9008952F923F924F925F926F927F
:10F1E0007F928F929F92AF92BF92CF92DF92EF92D7
:10F1F000FF920F931F93CF93DF93CDB7DEB76A973C
:10F200000FB6F894DEBF0FBECDBF182F81E00E946D
:10F21000AC158FE40E947A698823B9F080911E0CA6
:10F2200090911F0C892BB1F00E94BD6997FD18C009
:10F230000E94BD696F3F71058105910509F054F485
:10F240000E94BD69611106C00BC08FE40E94336942
:10F25000882331F090918B059770973009F40FC295
:10F260000E94475820910E06288F80E00E94881A3D
:10F270000E94584E81E00E94D62D111119C088E5D8
:10F280000E943369382E89E50E943369182F8AE578
:10F290000E943369282E311006C0111110C081114F
:10F2A0000EC0312E0AC0112351F0312E082F08C094
:10F2B00011E0332433942224239401E001C000E0C0
:10F2C00080E1E9E7F5E0A9E6B5E001900D928A95C5
:10F2D000E1F7011102C0222019F082E00E94FC50E7
:10F2E00082E50E947A69882371F180911E0C9091C9
:10F2F0001F0C009709F457C0FC015F012191322FC8
:10F300003F7D99F0253411F02536B9F7D5011C92CF
:10F3100060E070E080911E0C90911F0C2A8F0E947B
:10F32000A0AD2A8DF501208304C060E070E00E944A
:10F33000A0AD6B017C0120E030E0A9010E9410AA81
:10F34000882389F106C0C12CD12C20E8E22E30E4BC
:10F35000F32E011105C0311003C0112309F410C1AF
:10F36000C601D7018093710590937205A093730530
:10F37000B0937405209181053091820540918305F9
:10F3800050918405B601C7010E9413AC18165CF4B5
:10F3900019821A821B821C82BE016F5F7F4F81E738
:10F3A00095E00E94DF4D01110CC0332009F4FCC030
:10F3B000111107C080E00E94FC50002309F47EC1B7
:10F3C000DCC010927D0510927E0510927F05109290
:10F3D00080051092790510927A0510927B051092A3
:10F3E0007C050E941D4CE6E9F4E12491298FE5EAB1
:10F3F000F4E185909590A590B490E9EAF4E1459008
:10F40000559065907490A3019201C501B4010E94CA
:10F4100013AC18162CF4A5019401C301B20104C069
:10F42000A3019201C501B4010E9417AA6B017C01DE
:10F43000EEE8F4E185919591A591B4918D879E8731
:10F44000AF87B88BEAE8F4E185919591A591B491E5
:10F45000898B9A8BAB8BBC8B2D853E854F855889CC
:10F46000BC01CD010E9410AA87FD09C09D859D8B1E
:10F47000AE85AE8BBF85BF8BE889ED8708C0F98963
:10F48000FD8B2A892E8B8B898F8B9C899D87A70169
:10F490009601C701B6010E944EAC20E030E040E882
:10F4A0005FE30E9437A90E94BBAC9B01AC016D8950
:10F4B0007E898F899D850E944EAC69877A878B876C
:10F4C0009C87E7E9F4E1F49020E030E040EC5FE372
:10F4D000C301B2010E944EAC2B013C016F2DFF0C09
:10F4E000770B880B990B0E94B2AA9B01AC01C30158
:10F4F000B2010E944EAC69837A838B839C8320E0A7
:10F5000030E040EC5FE3C501B4010E944EAC6B01FA
:10F510007C01A98D6A2FAA0F770B880B990B0E948B
:10F52000B2AA9B01AC01C701B6010E944EAC6D832B
:10F530007E838F839887AE01475F5F4FBE016F5F09
:10F540007F4FCE0105960E94FD4D0E949D2D109289
:10F550007D0510927E0510927F0510928005109215
:10F56000790510927A0510927B0510927C050111A5
:10F5700021CF3110A0C0112319F081E00E94FC506E
:10F580000E941D4CF090D10480E00E94C32D812C7C
:10F59000912C90EAA92E90E4B92E89829A82AB82AE
:10F5A000BC82011115C0A8C01111E7CF0E941D4CEB
:10F5B000F090D10480E00E94C32D80E090E0A0EAAA
:10F5C000B0E489839A83AB83BC83222009F48BC087
:10F5D00080E090E0ADE1B3E48D839E83AF83B88794
:10F5E000BE016F5F7F4FCE0105960E94DF4D80E028
:10F5F00090E0A0EAB0E489839A83AB83BC830111D5
:10F600000BC0111109C080917D0590917E05A091DC
:10F610007F05B091800504C080E090E0A9E3B3E4E9
:10F620008D839E83AF83B88701110BC0311009C051
:10F630008091790590917A05A0917B05B0917C0528
:10F6400004C080E090E0A0EAB0E489879A87AB87A5
:10F65000BC87AE014F5F5F4FBE016B5F7F4FCE0136
:10F6600009960E94FD4D8F2D0E94C32D0E94982D5A
:10F67000888D0E94881A0E94774E0E94F54B80E088
:10F680000E94AC156A960FB6F894DEBF0FBECDBFD0
:10F69000DF91CF911F910F91FF90EF90DF90CF906E
:10F6A000BF90AF909F908F907F906F905F904F90A2
:10F6B0003F902F90089580E00E94FC5011115DCF83
:10F6C0000E941D4CF090D10480E00E94C32D812C3B
:10F6D000912C80EAA82E80E4B82E89829A82AB828F
:10F6E000BC8221101FC08091810590918205A0915C
:10F6F0008305B091840570CF2220A9F380E090E0CB
:10F70000ADE1B3E48D839E83AF83B887BE016F5FA5
:10F710007F4FCE0105960E94DF4D89829A82AB828F
:10F72000BC826FCF80E090E0ADE1B3E48D839E8337
:10F73000AF83B887BE016F5F7F4FCE0105960E94F1
:10F74000DF4D89829A82AB82BC825DCF80E1E9E79E
:10F75000F5E0A9E6B5E001900D928A95E1F70895EC
:10F760004F925F926F927F928F929F92AF92BF92D1
:10F77000CF92DF92EF92FF920F931F93CF93DF937D
:10F78000CDB7DEB72E970FB6F894DEBF0FBECDBF54
:10F79000270138012E874A875B876C877D87898799
:10F7A000D5DF89852E854A855B856C857D858F3F74
:10F7B00051F094E0899FF0011124E759FA4F4083FA
:10F7C0005183628373832F3F51F0A4E02A9FF0019D
:10F7D0001124E759FA4F4082518262827382BFEF4F
:10F7E000CB1651F084E0C89EF0011124E759FA4F7E
:10F7F00080829182A282B3828090690590906A058E
:10F80000A0906B05B0906C0520E030E042E253E43C
:10F81000C501B4010E9410AA87FF11C020E030E0AA
:10F8200040E450ECC501B4010E9413AC18166CF012
:10F83000812C912C30E4A32E30ECB32E06C0812C09
:10F84000912C22E2A22E23E4B22E8092690590929E
:10F850006A05A0926B05B0926C0540906D055090C2
:10F860006E0560906F057090700520E030E04EE30B
:10F8700053E4C301B2010E9410AA87FF11C020E027
:10F8800030E040EE50ECC301B2010E9413AC1816F8
:10F890006CF0412C512C90EE692E90EC792E06C024
:10F8A000412C512C8EE3682E83E4782E40926D0516
:10F8B00050926E0560926F0570927005809171058F
:10F8C00090917205A0917305B09174058D839E830C
:10F8D000AF83B88720E030E04FE153E4BC01CD01B5
:10F8E0000E9410AA87FF11C020E030E040E050ECF9
:10F8F0006D817E818F8198850E9413AC18166CF003
:10F9000080E090E0A0E0B0EC04C080E090E0AFE1E7
:10F91000B3E48D839E83AF83B8878D819E81AF8151
:10F92000B8858093710590937205A0937305B09389
:10F93000740580E090E0A8E4B2E489839A83AB8305
:10F94000BC83DE0111966D01ED80FE800F8118856C
:10F95000A3019201C501B4010E94034D2E960FB67A
:10F96000F894DEBF0FBECDBFDF91CF911F910F91F5
:10F97000FF90EF90DF90CF90BF90AF909F908F90CF
:10F980007F906F905F904F9008958F929F92AF926B
:10F99000BF92CF92DF92EF92FF920F931F93CF937C
:10F9A000DF93EC016A017B0120E030E040E45FE39B
:10F9B000688579858A859B850E9437A9A70196016C
:10F9C0000E9437A9AB01BC01812C912C5401CC249D
:10F9D000CA94850174012FEF82E0C2DEEC80FD80C5
:10F9E0000E811F81488159816A817B8121E080E0FD
:10F9F000B7DEDF91CF911F910F91FF90EF90DF90D5
:10FA0000CF90BF90AF909F908F9008952F923F928C
:10FA10004F925F926F927F928F929F92AF92BF921E
:10FA2000CF92DF92EF92FF920F931F93CF93DF93CA
:10FA3000CDB7DEB72E970FB6F894DEBF0FBECDBFA1
:10FA400089878B014A87222359F0812C912C90E8D9
:10FA5000A92E9EE3B92E80E090E0A0EAB1E40CC0AC
:10FA60008AE0882E87ED982E83E2A82E8CE3B82EAC
:10FA700080E090E0A0E8BFE389839A83AB83BC83F6
:10FA8000211105C080E090E0A0EAB0E404C080E06D
:10FA900090E0A8E4B2E48D839E83AF83B88756DEFE
:10FAA000412C512C3201B985A4E0BA9FC001112428
:10FAB000FC01E759FA4F1F01C801110FAA0BBB0B3C
:10FAC0008B879C87AD87BE872D813E814F8158856E
:10FAD000C301B2010E9410AA87FF3FC06B857C85DD
:10FAE0008D859E850E94B2AAA50194010E944EAC0C
:10FAF0009B01AC01D1016D917D918D919C910E94F2
:10FB000037A9F1016083718382839383E09071054B
:10FB1000F0907205009173051091740520916D05A8
:10FB200030916E0540916F055091700560916905A7
:10FB300070916A0580916B0590916C05DE011196BC
:10FB40006D010E94034D0E94475883B182958170D8
:10FB5000B1E08B27EA858E1324C0398524E0329FDB
:10FB6000F0011124E759FA4F6081718182819381FC
:10FB70002E960FB6F894DEBF0FBECDBFDF91CF91AA
:10FB80001F910F91FF90EF90DF90CF90BF90AF90BB
:10FB90009F908F907F906F905F904F903F902F90AD
:10FBA0000895A5019401C301B2010E9437A92B0158
:10FBB0003C018ACF4F925F926F927F928F929F9279
:10FBC000AF92BF92CF92DF92EF92FF920F931F936B
:10FBD000CF93DF93CDB7DEB728970FB6F894DEBF8B
:10FBE0000FBECDBFB82E6B01A42E4901C801B701CD
:10FBF000FF24F39420E030E040EA50E40E9410AA91
:10FC00008111F12CA3DD84E0B89E80011124F8015C
:10FC1000E759FA4F80819181A281B3818D839E83C0
:10FC2000AF83B8872F2D4A2DB6018B2DEFDE2B0128
:10FC30003C018114910411F1F11020C041E04A25EA
:10FC4000662777276C197D0920E08B2DDFDEA30165
:10FC500092010E9436A96B017C0120E030E0A901ED
:10FC60000E9413AC87FF04C0F7FAF094F7F8F09401
:10FC7000D401CD92DD92ED92FC921397F801E759F1
:10FC8000FA4F8D819E81AF81B88580839183A28355
:10FC9000B38380E090E0A8E4B2E489839A83AB83E5
:10FCA000BC83E0907105F09072050091730510918E
:10FCB000740520916D0530916E0540916F0550914E
:10FCC00070056091690570916A0580916B0590914E
:10FCD0006C05DE0111966D010E94034DC301B20156
:10FCE00028960FB6F894DEBF0FBECDBFDF91CF913F
:10FCF0001F910F91FF90EF90DF90CF90BF90AF904A
:10FD00009F908F907F906F905F904F9008952F926B
:10FD10003F924F925F926F927F928F929F92AF929B
:10FD2000BF92CF92DF92EF92FF920F931F93CF93E8
:10FD3000DF93CDB7DEB769970FB6F894DEBF0FBE7D
:10FD4000CDBF3C014C8B5D8B6E8B7F8B2D878CE008
:10FD5000EDEEF2E0DE01119601900D928A95E1F749
:10FD60004C895D896E897F89C3010FDE2D85223024
:10FD7000D1F060F42223F1F0213009F073C1212C7D
:10FD8000312C60E8462E6FEB562E46C03D85333051
:10FD9000C9F1343009F066C1212C312C70E8472EAE
:10FDA0007FEB572E36C0212C312CF0E84F2EFFE38D
:10FDB0005F2E2FC09301205E3F4FEC88FD880E8997
:10FDC0001F8941E06FEF7FEF82E0F4DE6B017C0181
:10FDD00020E030E040E05FE369857A858B859C8593
:10FDE0000E944EAC9B01AC01C701B6010E9436A92E
:10FDF000F3016087718782879387C486D586E686FC
:10FE0000F78630C1212C312CE0E84E2EEFE35E2E38
:10FE100003C0DD24D39401C0D12C2D2D30E03F87C9
:10FE20002E87002309F463C0C901880F991F880F2A
:10FE3000991F7301E80EF91EE1E0F0E0EC0FFD1FE1
:10FE4000E80FF91F20E030E040E05FE3608171815E
:10FE5000828193810E944EACF701E05CFF4F2081CC
:10FE60003181428153810E9436A99B01AC01C201BC
:10FE7000B10190580E944EACF7012081318142813E
:10FE800053810E9437A9AB01BC01812C912C5401F4
:10FE9000CC24CA94850174012FEF8D2D61DCEC8890
:10FEA000FD880E891F899301205E3F4F41E06FEF6F
:10FEB0007FEF82E07FDE4B015C01F3016487758791
:10FEC0008687978720E030E040E05FE369857A85A8
:10FED0008B859C850E944EAC9B01AC01C501B40191
:10FEE0000E9436A9F30160877187828793878E8588
:10FEF0009F85880F991F880F991F9301280F391F1D
:10FF00003F872E87E1E0F0E0EC0FFD1FE80FF91FBF
:10FF100020E030E040E05FE3608171818281938185
:10FF20000E944EAC688B798B8A8B9B8B520141016E
:10FF3000B7FAB094B7F8B0948E859F85805C9F4FD8
:10FF4000998F888F20E030E040E05FE3FC01608122
:10FF50007181828193810E944EAC9B01AC016889C2
:10FF600079898A899B890E9437A92C893D894E8984
:10FF70005F890E9437A99B01AC01C501B4010E94B1
:10FF80004EACEE85FF8520813181428153810E94F4
:10FF900037A9AB01BC01812C912C5401CC24CA940B
:10FFA000850174012FEF8D2DDBDB23E333E343E386
:10FFB0005FE3F30164857585868597850E9436A980
:10FFC000AB01BC012FEF82E0CBDBFD85AF2EB12C66
:10FFD000450128E0820E911C880C991C880C991C04
:10FFE000860C971CC201B1010E947FAAEC88FD8893
:10FFF0000E891F89940141E08D2DDCDD6B017C01B0
:020000021000EC
:1000000020E030E040E05FE3E88DF98D60817181B0
:10001000828193810E944EAC9B01AC0168897989F1
:100020008A899B890E9437A99B01AC01C201B10159
:100030000E944EAC9B01AC01C701B6010E9437A9DA
:10004000EE85FF856083718382839383F501339608
:10005000EE0FFF1FEE0FFF1FE60DF71DC082D182CE
:10006000E282F38269960FB6F894DEBF0FBECDBF71
:10007000DF91CF911F910F91FF90EF90DF90CF9084
:10008000BF90AF909F908F907F906F905F904F90B8
:100090003F902F900895CF92DF92EF92FF920F93AF
:1000A000CF93DF93EC016A017B0100E020E02FDEBB
:1000B00022E0B701A601CE012ADE23E0B701A601A6
:1000C000CE0125DEB701A601CE015FDC1CAA1DAA68
:1000D0001EAA1FAA18AE19AE1AAE1BAE2885398506
:1000E0004A855B8560E070E0CB010E9436A96CAF69
:1000F0007DAF8EAF9FAFDF91CF910F91FF90EF90CB
:10010000DF90CF9008958F929F92AF92BF92CF923F
:10011000DF92EF92FF920F931F93CF93DF93EC0147
:10012000C090330CD090340CE090350CF090360C2D
:1001300080E090E0A0E8BFE38093330C9093340C10
:10014000A093350CB093360C8090530290905402DB
:10015000A0905502B0905602109253021092540291
:100160001092550210925602CE0195DF0E94475818
:1001700009E715E02CAD3DAD4EAD5FADF8016085F2
:100180007185828593850E9437A9F8016087718700
:1001900082879387188619861A861B861CAE1DAE29
:1001A0001EAE1FAE0E941D4C8092530290925402CC
:1001B000A0925502B0925602C092330CD092340CE9
:1001C000E092350CF092360CDF91CF911F910F9198
:1001D000FF90EF90DF90CF90BF90AF909F908F9067
:1001E00008952F923F924F925F926F927F928F92DB
:1001F0009F92AF92BF92CF92EF92FF920F931F9375
:10020000CF93DF93CDB7DEB728970FB6F894DEBF54
:100210000FBECDBF5C018091330C9091340CA09146
:10022000350CB091360C8D839E83AF83B8871092C6
:10023000330C1092340C1092350C1092360C8091C5
:10024000530290915402A0915502B09156028983B5
:100250009A83AB83BC831092530210925402109283
:10026000550210925602C50116DFE7E3FCE0D50106
:100270009C964D915D916D917C919F9740835183A8
:100280006283738398964D915D916D917C919B975C
:10029000448355836683778390964D915D916D91EC
:1002A0007C919397408751876287738780E090E0C5
:1002B000A0E8BFE38093330C9093340CA093350CEB
:1002C000B093360C109253021092540210925502C1
:1002D0001092560289E7282E85E0382E20E030E083
:1002E00040E450E4F10160857185828593850E9428
:1002F00037A94B015C0120E030E040E450E4D1013B
:1003000014966D917D918D919C9117970E9437A9BC
:100310002B013C0120E030E040E450E4F101608139
:100320007181828193810E9437A9AB01BC0192E067
:10033000C92E8301720121E080E012DA20E030E072
:1003400040E450E4D10118966D917D918D919C917E
:100350001B970E9436A94B015C0120E030E040E48D
:1003600050E4F10164817581868197810E9436A9EC
:100370002B013C0120E030E040E450E4D1016D91DC
:100380007D918D919C910E9436A9AB01BC018301A6
:10039000720121E080E0E4D989819A81AB81BC813E
:1003A0008093530290935402A0935502B093560247
:1003B0008D819E81AF81B8858093330C9093340CEE
:1003C000A093350CB093360C28960FB6F894DEBF88
:1003D0000FBECDBFDF91CF911F910F91FF90EF9096
:1003E000CF90BF90AF909F908F907F906F905F90D5
:1003F0004F903F902F9008958F929F92AF92BF920F
:10040000CF92DF92EF92FF92C090330CD090340CD9
:10041000E090350CF090360C812C912C20E8A22E27
:100420002FE3B22E8092330C9092340CA092350CB4
:10043000B092360C8090530290905402A0905502D6
:10044000B09056021092530210925402109255022C
:100450001092560258DE8092530290925402A0925B
:100460005502B0925602C092330CD092340CE092F6
:10047000350CF092360CFF90EF90DF90CF90BF904C
:10048000AF909F908F9008959C018CE0E9EFF2E08F
:10049000D90101900D928A95E1F798E0E5E0F3E04B
:1004A000D901A05CBF4F01900D929A95E1F7089594
:1004B0004F925F926F927F928F929F92AF92BF9274
:1004C000CF92EF92FF920F931F93CF93DF93CDB70D
:1004D000DEB7CC54D1090FB6F894DEBF0FBECDBF46
:1004E000CE010196D1DF4090330C5090340C6090D7
:1004F000350C7090360C80E090E0A0E8BFE380936C
:10050000330C9093340CA093350CB093360C80913F
:10051000530290915402A0915502B09156022D962B
:100520008CAF9DAFAEAFBFAF2D971092530210921C
:100530005402109255021092560240E050E060EAD8
:1005400070E4CE01019658DF40E050E060E87FE3C0
:10055000CE01019646DE40E050E060E87FE3CE0148
:1005600001964ADF812C912C5401CC24CA94850138
:1005700074012FEF40E050E066E173E480E0F0D8D2
:100580002D968CAD9DADAEADBFAD2D978093530232
:1005900090935402A0935502B09356024092330CAC
:1005A0005092340C6092350C7092360CC45BDF4F65
:1005B0000FB6F894DEBF0FBECDBFDF91CF911F9174
:1005C0000F91FF90EF90CF90BF90AF909F908F9042
:1005D0007F906F905F904F9008959F92AF92BF92DF
:1005E000CF92DF92EF92FF920F931F93CF93DF93FF
:1005F000CDB7DEB7C854D1090FB6F894DEBF0FBE31
:10060000CDBF81E00E94AC150091410210924102E1
:1006100090900E0680E00E94881A41E061E081E03F
:100620000E94A84F8111EEC0CE0101962DDF85E515
:100630000E943369882341F120911E0C30911F0CD8
:100640002115310509F1F9015F011191812F8F7D8C
:1006500099F0153411F01536B9F7F501108260E004
:1006600070E080911E0C90911F0C0E94A0AD6B0158
:100670007C01F50110830EC060E070E0C9010E94AA
:10068000A0AD6B017C0106C0C12CD12C80E8E82E06
:100690008FE3F82E82E40E943369882331F0B7019A
:1006A000A601CE0101969DDDADC084E50E943369AF
:1006B000882391F080911E0C90911F0C009731F0CF
:1006C0004AE050E060E070E00E9406AFB701A6018A
:1006D000CE01019618DD96C086E50E943369882315
:1006E00009F48FC0B701A601CE010196D4DC8AE0DF
:1006F0000E94941883EF99E10E9404164D855E854F
:100700006F8578898BEE99E10E944F168AE00E94EE
:100710009418498D5A8D6B8D7C8D82EE99E10E94E3
:100720004F168AE00E9494184D895E896F89788DF2
:1007300088ED99E10E944F168AE00E9494188AE0A1
:100740000E9494188FEC99E10E94041649855A85FD
:100750006B857C858CEC99E10E944F168AE00E94A3
:1007600094188AE00E94941881EC99E10E94041682
:100770004DA55EA56FA578A988EB99E10E944F165B
:100780008AE00E94941849A55AA56BA57CA58EEA1B
:1007900099E10E944F168AE00E94941849A15AA13B
:1007A0006BA17CA186EA99E10E944F168AE00E9423
:1007B00094188AE00E94941888E899E10E9404162F
:1007C0008AE00E94941884E50E9494186AE070E020
:1007D00080E090E00E94871984E799E10E94041666
:1007E00021964CAD5DAD6EAD7FAD219781E799E16E
:1007F0000E944F168AE00E9494188AE00E94941882
:1008000001C056DE892D0E94881A0093410280E0C3
:100810000E94AC15C85BDF4F0FB6F894DEBF0FBE69
:10082000CDBFDF91CF911F910F91FF90EF90DF909F
:10083000CF90BF90AF909F9008951F93CF93DF9379
:10084000CDB7DEB72C970FB6F894DEBF0FBECDBF85
:1008500083E50E9433698823B9F080911E0C909142
:100860001F0C892BC9F00E94BD6997FD10C00E9422
:10087000BD696F3F71058105910509F06CF40E9417
:10088000BD69611109C003C010910E0606C080E069
:100890000E94881A10E001C011E0809179059091C2
:1008A0007A05A0917B05B0917C0589839A83AB83FF
:1008B000BC8380917D0590917E05A0917F05B091CC
:1008C00080058D839E83AF83B88780918105909149
:1008D0008205A0918305B091840589879A87AB87AB
:1008E000BC8786E50E943369882331F068E27AE1AB
:1008F0008AEE95E00E94E3A3812F0E94881A1123BB
:1009000051F080910E06811106C00E94151689E0F3
:100910009AE10E9404160E9412168BEF99E10E9440
:10092000041680910E060E9491164CE050E069E793
:1009300075E0CE0101960E94C8B1892B59F02C9622
:100940000FB6F894DEBF0FBECDBFDF91CF911F91E0
:100950000C94F54B2C960FB6F894DEBF0FBECDBFAE
:10096000DF91CF911F9108958F929F92AF92BF9286
:10097000CF92DF92EF92FF92CF934B015C0169011E
:100980007A0122ED30E040EE50ECC701B6010E9442
:1009900013AC87FD33C027E030E04EE353E4C701DA
:1009A000B6010E9410AA18164CF123EA31E040E487
:1009B00050ECC501B4010E9413AC87FD1FC027E0B5
:1009C00030E042E253E4C501B4010E9410AA1816B7
:1009D000ACF027E030E041E253E4C501B4010E94ED
:1009E00010AA18165CF0C1E027E030E041E253E4C1
:1009F000C701B6010E9410AA18160CF4C0E08C2F93
:100A0000CF91FF90EF90DF90CF90BF90AF909F90ED
:100A10008F900895CF93DF93D82FC62F0E947A69C5
:100A20008823D1F080911E0C90911F0C892B11F41A
:100A300081E01AC00E94BD6997FD15C00E94BD6982
:100A40006F3F71058105910509F094F70E94BD691A
:100A500081E0611109C007C08D2F0E9433698111A7
:100A6000E7CF8C2F01C080E0DF91CF9108952F92C6
:100A70003F924F925F926F927F928F929F92AF922E
:100A8000BF92CF92DF92EF92FF920F931F93CF937B
:100A9000DF93CDB7DEB7CB51D1400FB6F894DEBFB0
:100AA0000FBECDBF81E00E94AC1541E061E081E066
:100AB0000E94A84F81111AC080910E06882329F048
:100AC00060E08FE4A7DF811111C0FE0131968CE355
:100AD000DF011D928A95E9F730900E068AE40E94A4
:100AE0003369982E882329F00E94A71A912C0C9420
:100AF000488F60E070E086E50E947F72C351DF4F4F
:100B000099838883CD5ED040059718F08BE09CE1F7
:100B100036C160E084E47EDFC950DF4F8883C75F61
:100B2000D040C351DF4F28813981CD5ED040233082
:100B300031054CF460E084E56DDFC450DF4F8883FD
:100B4000CC5FD04006C031E0C450DF4F3883CC5F6B
:100B5000D04062E070E088E50E947F72182F62E06A
:100B600070E089E50E947F72082F80E50E947A6913
:100B7000811103C0612F802F03C00E94BD69862FA1
:100B8000623019F082EE9BE1FAC0823019F089EBF5
:100B90009BE1F5C083E50E947A69882319F00E94E1
:100BA000866904C060E070E88BEB95E420E030E0FB
:100BB00040E752E40E9417AA6093420270934302F6
:100BC000809344029093450288E40E94336988230D
:100BD00091F10E9486690E947FAA8B0177FF02C073
:100BE0000F5F1F4F15950795119501951109035B2F
:100BF0001F4F0E3F4FEF14072CF44DEFA42EBB24D4
:100C0000BA9401C058016501C60ED71E51EAC51637
:100C1000D1041CF031EAC32ED12C0A3FAFEF1A07E2
:100C200014F409EF1FEF7801E60EF71EB1EAEB1698
:100C3000F104CCF135C08CE40E947A69882331F04C
:100C40000E9486690E947FAA5B0104C02DEFA22E3C
:100C5000BB24BA9482E50E947A69882331F00E940D
:100C600086690E947FAA6B0103C091EAC92ED12C2C
:100C700086E40E947A69882331F00E9486690E9486
:100C80007FAA8B0102C009EF1FEF82E40E947A69FC
:100C9000882331F00E9486690E947FAA7B0103C0ED
:100CA00081EAE82EF12CB801012E000C880B990B7B
:100CB0000E94B2AAC250DF4F688379838A839B83E4
:100CC000CE5FD040B5010B2C000C880B990B0E9415
:100CD000B2AACE5FDE4F688379838A839B83C2503A
:100CE000D140C250DF4F288139814A815B81CE5F7C
:100CF000D0403ADE882309F440C0B7010F2C000C25
:100D0000880B990B0E94B2AA9B01AC01B6010D2C75
:100D1000000C880B990BC85EDE4F2883C851D14068
:100D2000C75EDE4F3883C951D140C65EDE4F48836F
:100D3000CA51D140C55EDE4F5883CB51D1400E948D
:100D4000B2AAC85EDE4F2881C851D140C75EDE4FCF
:100D50003881C951D140C65EDE4F4881CA51D14069
:100D6000C55EDE4F5881CB51D140FEDDCA50DF4F0A
:100D70008883C65FD040811106C08DE99BE10E9447
:100D800004160C94488FB6016A197B09072E000CD3
:100D9000880B990B0E94B2AAC65FDE4F68837983E5
:100DA0008A839B83CA50D140B701601B710B072E09
:100DB000000C880B990B0E94B2AAC25FDE4F6883B9
:100DC00079838A839B83CE50D140C351DF4FE88122
:100DD000F981CD5ED040EF2B91F087E89BE10E9436
:100DE0000416C950DF4FE881C75FD040EE2321F0E1
:100DF0008DE79BE10E9404168AE00E9494180E94ED
:100E0000475880E00E94881A81E00E94B1488823F8
:100E100029F0832D0E94881A0C94488F0E94584E06
:100E200060E085E4F7DD811107C0F2E0C350DF4FD9
:100E3000F883CD5FD04006C021E0C350DF4F288348
:100E4000CD5FD040C151DF4F19821882CF5ED040B4
:100E5000C752DF4F188219821A821B82C95DD040A7
:100E6000C850DF4F188219821A821B82C85FD04097
:100E7000C751DF4F1882C95ED0404FEF5FEFC352BA
:100E8000DF4F59834883CD5DD0405FEFCB50DF4FBC
:100E90005883C55FD0408FEFCD50DF4F8883C35F4D
:100EA000D04091E0CB52DF4F9883C55DD040C35214
:100EB000DF4F88819981CD5DD0400196880F991FC1
:100EC000880F991F4DE350E04C0F5D1F480F591FCD
:100ED000CB51DF4F59834883C55ED040DC01149766
:100EE000C85FDE4FB983A883C850D1408CE0C3529D
:100EF000DF4F28813981CD5DD040829FF001839FF3
:100F0000F00D1124CA5FDE4FF983E883C650D1404B
:100F1000CF51DF4F19821882C15ED040C151DF4FDF
:100F200088819981CF5ED040092E000CAA0BBB0BA3
:100F3000CE5EDE4F88839983AA83BB83C251D140A2
:100F4000C151DF4FA881B981CF5ED040AA0FBB1F2E
:100F5000CA5EDE4FB983A883C651D140CB52DF4F62
:100F60005881C55DD040CD50DF4F8881C35FD040F0
:100F7000581709F497C2CE5EDE4F688179818A8165
:100F80009B81C251D1400E94B2AA9B01AC01C65FB5
:100F9000DE4F688179818A819B81CA50D1400E944D
:100FA0004EAC9B01AC01CE5FDE4F688179818A81B6
:100FB0009B81C250D1400E9437A94B015C01CB52AA
:100FC000DF4FB881C55DD0406B2FBB0F770B880B0F
:100FD000990B0E94B2AA9B01AC01C25FDE4F6881EF
:100FE00079818A819B81CE50D1400E944EAC9B0179
:100FF000AC01C250DF4F688179818A819B81CE5FCD
:10100000D0400E9437A96B017C0120E030E0A901AB
:10101000C501B4010E9410AA87FD05C020E030E0A0
:1010200040E05FE303C020E030E0A901C501B40166
:101030000E9437A90E94EDAAC355DF4F68837983C8
:101040008A839B83CD5AD04020E030E0A901C701BC
:10105000B6010E9410AA87FD05C020E030E040E004
:101060005FE303C020E030E0A901C701B6010E94A0
:1010700037A90E94EDAAC755DF4F688379838A8319
:101080009B83C95AD040C352DF4FE881F981CD5DBF
:10109000D0403196C352DF4FF983E883CD5DD04015
:1010A000CA5EDE4FE881F981C651D140CB52DF4F95
:1010B0002881C55DD040E20FF11D27FDFA95EE0FA6
:1010C000FF1F41EA50E04C0F5D1FE40FF51FC352B4
:1010D000DF4F88819981CD5DD0409183808301E08D
:1010E000C351DF4F2881CD5ED040C350DF4F4881D0
:1010F000CD5FD040BE0167557F4FCE0183559F4FD6
:101100000E945249C752DF4F688379838A839B8349
:10111000C95DD0409B01AC010E94FCAC882321F04A
:10112000832D0E94881AD5C1C752DF4F288139818B
:101130004A815B81C95DD040C850DF4F68817981A9
:101140008A819B81C85FD0400E9437A9C850DF4F79
:10115000688379838A839B83C85FD040CF51DF4FF8
:10116000E881F981C15ED040C85FDE4FA881B981B6
:10117000C850D140EA0FFB1F2DE630E02C0F3D1F79
:10118000E20FF31FC752DF4F88819981AA81BB818B
:10119000C95DD04084839583A683B783C355DF4F51
:1011A000488059806A807B80CD5AD040CB51DF4F38
:1011B000A881B981C55ED0404D925D926D927D92BD
:1011C000CB51DF4FB983A883C55ED040CF51DF4FED
:1011D000E881F981C15ED0403496CF51DF4FF98369
:1011E000E883C15ED040C755DF4F88809980AA80D0
:1011F000BB80C95AD0401C968D929D92AD92BC92F4
:101200001F9720E030E040E85FE35C962D933D932C
:101210004D935C935F97A301920169817A818B81E1
:101220009C810E9437A969837A838B839C83A50163
:1012300094016D817E818F8198850E9437A96D838D
:101240007E838F839887C752DF4F288139814A81F7
:101250005B81C95DD04069857A858B859C850E94BC
:1012600037A969877A878B879C87A3019201C3017D
:10127000B2010E944EAC9B01AC016D857E858F85CD
:1012800098890E9437A96D877E878F87988BA501E3
:101290009401C501B4010E944EAC9B01AC01698967
:1012A0007A898B899C890E9437A9698B7A8B8B8B71
:1012B0009C8BC752DF4F288139814A815B81C95D90
:1012C000D040CA01B9010E944EAC9B01AC016D89AE
:1012D0007E898F89988D0E9437A96D8B7E8B8F8B2D
:1012E000988FA5019401C301B2010E944EAC9B01ED
:1012F000AC01698D7A8D8B8D9C8D0E9437A9698F89
:101300007A8F8B8F9C8FC752DF4F288139814A811A
:101310005B81C95DD040C301B2010E944EAC9B010C
:10132000AC016D8D7E8D8F8D98A10E9437A96D8F38
:101330007E8F8F8F98A3C752DF4F288139814A81D2
:101340005B81C95DD040C501B4010E944EAC9B01D8
:10135000AC0169A17AA18BA19CA10E9437A969A3C4
:101360007AA38BA39CA31DA10EA13FA028A420E0DB
:1013700030E0A901C301B2010E9413AC7301620104
:1013800087FF04C0F7FAF094F7F8F094212F302F7C
:10139000432D522DC701B6010E9413AC181624F03C
:1013A000C12ED02EE32CF22CCDA2DEA2EFA2F8A605
:1013B00019A50AA53BA42CA420E030E0A901C50191
:1013C000B4010E9413AC7501640187FF04C0F7FAF1
:1013D000F094F7F8F094212F302F432D522DC701B0
:1013E000B6010E9413AC181624F0C12ED02EE32CA7
:1013F000F22CC9A6DAA6EBA6FCA620E030E040E875
:101400005FE369AD7AAD8BAD9CAD0E9437A969AF42
:101410007AAF8BAF9CAFC752DF4FC880D980EA80CC
:10142000FB80C95DD04095018401B301A201CE01CA
:1014300083589F4F0E94719FCF51DF4FA881B98180
:10144000C15ED040AA0FBB1FCF51DF4FE881F981A9
:10145000C15ED040AE0FBF1FCA5FDE4F2881398109
:10146000C650D140A20FB31FAD5BB34FFE01E3588E
:10147000FF4F8CE001900D928A95E1F70E9497A8AA
:10148000CB52DF4F3881C55DD040CB50DF4F488114
:10149000C55FD040340FCB52DF4F3883C55DD0409D
:1014A000312C5CCDC151DF4FA881B981CF5ED040D6
:1014B000119779F0C752DF4F288139814A815B81CA
:1014C000C95DD040CA01B9010E94FCAC882309F46F
:1014D000A4C480E00E94B148882381F0832D0E943B
:1014E000881A20E030E040EC5FE7C752DF4F2883E6
:1014F00039834A835B83C95DD04071C4C752DF4FD3
:10150000288139814A815B81C95DD040CA01B90116
:101510000E94FCAC811163C4CE0101960E9452A5C9
:101520008DA59EA5AFA5B8A9C352DF4F8883998327
:10153000AA83BB83CD5DD04029A93AA94BA95CA958
:10154000CF51DF4F288339834A835B83C15ED0400C
:101550008DA99EA9AFA9B8ADCB51DF4F88839983E0
:10156000AA83BB83C55ED04020E030E040E85EE364
:10157000C850DF4F688179818A819B81C85FD040E4
:101580000E944EACC151DF4F688379838A839B836D
:10159000CF5ED040C351DF4FA881B981CD5ED0402E
:1015A000AB2B09F480C14BE55CE06FE47CE0CE013D
:1015B00083589F4F0E9443A04FE45CE063E47CE0CB
:1015C000CE0187579F4F0E9443A0AE0143585F4F03
:1015D000BE0167577F4FCE018B569F4F0E948B9F56
:1015E000CB56DF4F488059806A807B80C559D040F8
:1015F000C756DF4F88809980AA80BB80C959D040E8
:10160000C356DF4F288139814A815B81CD59D04053
:10161000CB52DF4F288339834A835B83C55DD0403B
:101620002091670C3091680C4091690C50916A0CC4
:10163000C301B2010E944EAC6B017C0120916B0C86
:1016400030916C0C40916D0C50916E0CC501B40141
:101650000E944EAC9B01AC01C701B6010E9437A9A4
:101660006B017C0120916F0C3091700C4091710CDA
:101670005091720CCB52DF4F688179818A819B81B6
:10168000C55DD0400E944EAC9B01AC01C701B601C4
:101690000E9437A96B017C018091430C9091440C0E
:1016A000A091450CB091460CBC01CD019058A3010E
:1016B00092010E944EACC751DF4F688379838A83C1
:1016C0009B83C95ED0402091470C3091480C4091DB
:1016D000490C50914A0CC501B4010E944EAC9B01CB
:1016E000AC01C751DF4F688179818A819B81C95ED6
:1016F000D0400E9436A9C751DF4F688379838A831F
:101700009B83C95ED04020914B0C30914C0C409192
:101710004D0C50914E0CCB52DF4F688179818A81FC
:101720009B81C55DD0400E944EAC9B01AC01C7516E
:10173000DF4F688179818A819B81C95ED0400E9498
:1017400036A99B01AC01C701B6010E9437A96B0104
:101750007C0120E030E0A9010E9413AC181624F0AF
:10176000F7FAF094F7F8F094A3019201C301B201E3
:101770000E944EAC2B013C01A5019401C501B401AE
:101780000E944EAC9B01AC01C301B2010E9437A97B
:101790004B015C01CB52DF4F288139814A815B814B
:1017A000C55DD040CA01B9010E944EAC9B01AC019D
:1017B000C501B4010E9437A90E94BBAC9B01AC01DA
:1017C000C701B6010E9417AAAB01BC0186E59BE1E7
:1017D0000E944F168AE00E94941809E313E0D80192
:1017E0008D918D01882319F00E949418F8CF48E05C
:1017F00050E0C352DF4F688179818A819B81CD5D42
:10180000D04090580E94121A0FE413E0F801819121
:101810008F01882319F00E949418F8CF48E050E017
:10182000CF51DF4F688179818A819B81C15ED04031
:1018300090580E94121A04E513E0D8018D918D0191
:10184000882319F00E949418F8CFCB51DF4F68819C
:1018500079818A819B81C55ED040905848E050E0F4
:101860000E94121AC351DF4FE881F981CD5ED0404A
:101870003397B4F009E513E0D8018D918D018823E9
:1018800019F00E949418F8CF48E050E0C151DF4FA2
:10189000688179818A819B81CF5ED0400E94121A33
:1018A0008AE00E949418C950DF4FB881C75FD040CA
:1018B000B1112DC0C12CD12C70E8E72E7FE3F72E9B
:1018C000CF51DF4F088119812A813B81C15ED04011
:1018D000C352DF4F488159816A817B81CD5DD04001
:1018E000CE0183589F4F0E94719FBE0163587F4F66
:1018F000CE018F549F4F0E94F5A284E2FE01EF5467
:10190000FF4FAAEEB5E001900D928A95E1F7C45021
:10191000DF4FE881CC5FD040EE2309F4BBC183E9FF
:101920009AE10E9404166E01F3EACF0ED11CCB524D
:10193000DF4FD982C882C55DD04022E0C751DF4F5A
:101940002883C95ED040212C30ECC352DF4F38834E
:10195000CD5DD04049E7CF51DF4F4883C15ED040D5
:1019600054E4CB51DF4F5883C55ED04000E010E017
:10197000CB52DF4FE881F981C55DD040E00FF11F08
:10198000E080F180C701880F991F880F991FCD5003
:10199000DF4F99838883C35FD040EDE6F0E0EC0F22
:1019A000FD1FE80FF91F4080518062807380C15194
:1019B000DF4F288139814A815B81CF5ED040C301EE
:1019C000B2010E9436A94B015C01E1E0F0E0EC0FAE
:1019D000FD1FCD50DF4FA881B981C35FD040EA0F12
:1019E000FB1F84AD95ADA6ADB7ADCB56DF4F888359
:1019F0009983AA83BB83C559D040F7013496EE0F73
:101A0000FF1FEE0FFF1F21E030E02C0F3D1FE20F04
:101A1000F31F84AD95ADA6ADB7ADC757DF4F888333
:101A20009983AA83BB83C958D040C358DF4F18821B
:101A300019821A821B82CD57D0409E0123583F4FF6
:101A4000AE0147575F4FBE016B567F4F8AEE95E060
:101A50000E9403A2C358DF4F288139814A815B81EC
:101A6000CD57D040C301B2010E9436A97B013C0191
:101A70009B01AC01622DC352DF4F7881CD5DD04018
:101A8000CF51DF4F8881C15ED040CB51DF4F98816D
:101A9000C55ED0400E9413AC181684F42E2CC3529D
:101AA000DF4FF882CD5DD040CF51DF4F6882C15EFD
:101AB000D040CB51DF4F7882C55ED04020E030E08F
:101AC000A901C501B4010E9413AC87FD05C080E9DE
:101AD0009AE10E94041603C080E20E94941845E037
:101AE00050E0C501B4010E94121A0C5F1F4F08306C
:101AF000110509F03DCF8AE00E949418CB52DF4FC8
:101B000048815981C55DD04042505109CB52DF4FC9
:101B100059834883C55DD040C751DF4F5881C95EA6
:101B2000D040513039F081E0C751DF4F8883C95E22
:101B3000D0401CCF8AE00E949418C351DF4FA88187
:101B4000B981CD5ED040149709F0A4C087E69AE130
:101B50000E94041642E0742E00E010E0F601E00F4F
:101B6000F11F808191817C01EE0CFF1CEE0CFF1CAB
:101B7000E1E0F0E0EC0FFD1FEE0DFF1D44AD55ADB3
:101B800066AD77ADCB56DF4F488359836A837B833D
:101B9000C559D040FC013496EE0FFF1FEE0FFF1F1A
:101BA00021E030E02C0F3D1FE20FF31F84AD95AD17
:101BB000A6ADB7ADC757DF4F88839983AA83BB8390
:101BC000C958D040C358DF4F188219821A821B822D
:101BD000CD57D0409E0123583F4FAE0147575F4F2E
:101BE000BE016B567F4F8AEE95E00E9403A2EDE6A0
:101BF000F0E0EC0FFD1FEE0DFF1DC358DF4F2881F5
:101C000039814A815B81CD57D04060817181828169
